:020000040800F2
:1000000000000420457F0008652E0008672E0008C8
:10001000692E00086B2E00086D2E000800000000FD
:10002000000000000000000000000000813B01080B
:100030006F2E000800000000093C0108693C01081F
:10004000957F0008957F0008957F0008957F000840
:10005000957F0008957F0008712E0008772E000814
:10006000957F0008957F00089D0E0008091C000878
:10007000311C0008591C0008957F0008811C0008ED
:100080008D1C0008957F0008957F0008957F00086B
:10009000957F0008957F0008957F000809320008C9
:1000A000957F0008957F0008957F0008957F0008E0
:1000B000957F0008957F0008957F0008591B000870
:1000C000651B0008711B00087D1B0008891B0008C8
:1000D000951B0008957F0008A11B0008957F00086C
:1000E0007D2E0008957F0008957F0008ED2E000802
:1000F000052F00081D2F0008957F0008B51C00087B
:1001000000000000957F0008957F0008957F00089B
:100110000000000000000000957F0008957F0008A7
:10012000DD1C0008E91C00081D1D0008312F000817
:10013000957F0008957F0008957F0008957F00084F
:10014000957F0008957F0008957F0008957F00083F
:10015000957F00083D2F0008291D0008BD1B0008E1
:10016000957F0008957F0008000000000000000057
:10017000000000000000000000000000000000007F
:10018000957F0008957F0008000000000000000037
:10019000957F0008957F0008000000000000000027
:1001A000000000000000000000000000000000004F
:1001B000957F00080000000000000000957F000807
:1001C000957F000810B5034B0360044613F0B8FA9E
:1001D000204610BDE088010810B50446FFF7F2FF85
:1001E0002046082114F043FF204610BD08B5244CDA
:1001F0002368BFF35B8FD9070ED4204600F07EFC46
:1002000050B1204800F060FB1F4A20491D4800F013
:100210007EFC204600F077FC1D4C2368BFF35B8F0B
:10022000DA070FD4204600F069FC58B11549194887
:1002300000F0D0F8144A1849164800F068FC20462F
:1002400000F061FC154C2368BFF35B8FDB070FD414
:10025000204600F053FC58B10A49114800F0C0F99B
:10026000094A10490E4800F052FC204600F04BFCB1
:100270000D4B01221A7014F079FB04F003F900BF52
:10028000180400201C040020350B0008C1020008DF
:1002900090020020940200201D03000808020020A4
:1002A0000C020020090300086CD90120837910B5E5
:1002B00004461BB1006808B114F0DBFE204610BDF7
:1002C00038B5044600F5B56500F5B760FFF7EEFFF9
:1002D0002846FFF7EBFF04F5B360FFF7E7FF04F2F2
:1002E0008440FFF7E3FF204638BD000010B5054B02
:1002F000044640F8783BFFF765FF204613F036FBD5
:10030000204610BDFC88010810B5034B036004466D
:10031000FFF7ECFF204610BDCC89010810B5034B58
:1003200003600446FFF7E2FF204610BDB8890108CC
:1003300010B50446FFF7DAFF2046802114F097FE3F
:10034000204610BD10B50446FFF7E8FF20464FF4E5
:10035000C27114F08CFE204610BD10B50446FFF7A4
:10036000D3FF2046842114F082FE204610BD08B53C
:1003700004460021204613F081FB60B9204613F0AB
:100380008BFB062805D1D4F88000032102F0AEFAD9
:10039000EFE704F077F8022003F070F8E9E773B5AF
:1003A000531A0F2B04460D461646019306D9002218
:1003B00001A914F067FE019B2060A3603246294624
:1003C000206814F09AFE019B226863600021D154DA
:1003D00002B070BD30B50F4A87B0044602AB0D467F
:1003E0006846A2F10A010093FFF7D9FF4FF480623B
:1003F00069460323204613F025FB684614F064FE8B
:10040000054B2360C4F88051204613F077FA20464C
:1004100007B030BD12890108B88901082DE9F04103
:10042000D0F88041204600F0ABFA421E18BF0122EE
:1004300005460321204602F08FFA2A460121204674
:1004400002F08AFA04F5987002F0C4FE0EF020FD66
:100450004C480DF061FE4C48082278210EF04EFB0E
:100460004A48C82278210EF049FB4948DC2278210D
:100470000EF044FB47481E2278210EF03FFB464811
:100480000DF04AFE012D49D100200DF029FE434810
:10049000502278210EF032FB04200DF021FE6E2256
:1004A00078213F483D4FDFF8F8800EF027FB002011
:1004B0000DF016FE3B48962278210EF01FFB01221C
:1004C0000021204602F048FA0021204602F024FBD9
:1004D000022806464BD004282DD001281AD1024606
:1004E0000321204602F038FA00223146204602F06D
:1004F00033FA04200DF0F4FD5022782138460EF036
:10050000FDFA00200DF0ECFD6E22782140460EF041
:10051000F5FA0025FA2003F0EDFFD5E704200DF0F1
:10052000DFFD1E48502278210EF0E8FA281E18BF81
:1005300001208000B1E700220321204602F00CFADE
:1005400001221146204602F007FA00200DF0C8FDF6
:100550005022782138460EF0D1FA30460DF0C0FD19
:100560006E22782140460EF0C9FA0125D2E7FA2022
:1005700003F0C0FF2046294600F005FA2846BDE8F2
:10058000F08100BF48D801081389010829890108B2
:100590002E8901084289010830C8010858890108DC
:1005A0006D8901088489010830B595B00446FFF7CC
:1005B00035FF0323019302230546029301A9062375
:1005C0002046039313F074FA6421204613F066FA70
:1005D000D4F88001294600F05BFA15B030BD000068
:1005E00030B50F4A87B0044602AB0D466846A2F10B
:1005F0000E010093FFF7D3FE4FF400726946022309
:10060000204613F01FFA684614F05EFD054B236088
:10061000C4F88050204613F071F9204607B030BD71
:10062000AF890108CC89010802484FF4DC310FF092
:1006300085B800BFE81100204FF0C043C0B2188059
:1006400070474FF0C0435880704700EB41014FF0B6
:10065000C043884200D1704730F8022B5A80F8E737
:1006600000EB41014FF0C043884200D170475A88E7
:1006700020F8022BF8E7000010B5A0B014220021EA
:1006800001A817F059F96822002106A817F054F9BB
:1006900000231A46144915480EF05EFB04460CF080
:1006A0004FFBF022114600200CF0CCFAF02211464C
:1006B00000200CF0AFFA032100200DF029FE01A963
:1006C00020460CF046FA0A4B0E930A4B0F930A4B46
:1006D00011930A4B15930A4A0A4B06A920460CF0BF
:1006E00056FA20B010BD00BF50E601089CE4010896
:1006F00039060008430600084B060008610600089A
:10070000BDBE000859C500084FF0FF30704700001B
:1007100030B589B01D4B1E48002400941A6B42F07E
:1007200008021A631A6B02F008020092009A019400
:100730001A6B42F040021A631A6B02F040020192F7
:10074000019A02941A6B42F020021A631B6B059403
:1007500003F020030293029B4FF4006303930125EF
:10076000022303A90693049504F042F9082303A980
:1007700008480393049404F03BF9202306480393AC
:1007800003A9049504F034F909B030BD00380240E3
:10079000000C0240001802400014024008B500F2AC
:1007A00064450223194604460122284600F0E9FA6E
:1007B00004F27C46284600F00BFB0221304600F094
:1007C000BBFB04F5B564284600F038FB284600F072
:1007D0003DFB0121284600F05DFB40F30F21204640
:1007E00000F0E9F947F6FF7382B20221304600F0CB
:1007F000CEFBE8E783B5DFED2E8A9FED2E9ADFED85
:100800002E9A9FED2EAA06460025F0EE68AA68EE05
:10081000897A87EEA90A07EE905AF8EEE77A20EE79
:10082000270A14F091FC60EE0A7AB0EE408AFDEEE1
:10083000E77AD6F8400617EE903A19B207F06AFF49
:10084000BEEEC98A06F5B56018EE103A1CB2214614
:1008500000F0B1F9C0EB0011090144BF01F57F417F
:10086000FF3107460914D6F8440607F053FF06F295
:10087000D45023462A46CDE9005711490446013594
:1008800017F020F82146002003F0BAFDB5F5817F6E
:100890000BD178EEAA8ADFED0B7AF4EEE78AF1EE5F
:1008A00010FAC8BFDFED028A00250DF079FDAEE732
:1008B0000000C842DB0FC94000007A4500007042CA
:1008C000D889010800007A4430B56021044687B019
:1008D00001F044FA04F294430025C4F884348122E0
:1008E000C4F88C34C4F89034224BA4F8882404F55E
:1008F000B361C4F89835A4F89C25C4F8A03504F277
:100900008442C4F8A43584F88A544FF4005384F820
:100910009E5504F5B56000F028F92846C4F838560D
:10092000C4F83C5603F04CFC2946204600F0ECFB92
:100930002046012100F002FC2046012100F008FCC5
:100940000D4B00951A6B0D4842F001021A631B6BA8
:10095000039503F001030093009B4FF48063019320
:100960000123029301A90223049304F041F82046D5
:1009700007B030BDAE8A01080038024000000240D6
:10098000032102F0E6B80A46032102F0D9B80000BC
:10099000F0B5D0F83C5685B004460E462DB1284639
:1009A00005B0BDE8F04008F0AABB08F081FE4FF4A6
:1009B000087303930223CDE90003F0231A46294666
:1009C0000295284608F05EFA2A46C4F83C066FF005
:1009D0007F4108F0ABFA2C49D4F83C06012208F01C
:1009E000A5FA03222949D4F83C0608F09FFAD4F866
:1009F0003C06012108F0B7FA334604F24C624FF48A
:100A0000F0714FF47F0007F04BFE334604F60C22E2
:100A1000C4F840064FF4F0714FF4004007F040FE78
:100A2000D4F84076C4F8440606463946D4F83C0665
:100A300008F038FA38463C2107F087FED4F83C0627
:100A4000314608F02FFA3046B42107F07EFE142319
:100A500001221146184607F017FDB7EE000AC4F848
:100A6000480607F03FFDD4F84816D4F83C0608F0D5
:100A70003BFA0095D4F83C062B462A46142108F090
:100A80008AFA05B0F0BD00BF808080004040400081
:100A900008B505460C46C0F83816B1B90EF0F8F99D
:100AA0001149204603F0ACFC1049204603F0A8FC95
:100AB0000F48502278210EF021F80E486E2278213E
:100AC0000EF01CF82846FFF769FE4FF4F071FFF7AF
:100AD0005FFF0949002003F093FC0449002003F064
:100AE0008FFC2846FFF786FEEF8901080D8A010872
:100AF000508A01086C8A01088B8A01080078B0FAD4
:100B000080F0400970470123037070477047002050
:100B100070477047FEE70000044A1168034609B9B0
:100B2000034911601068034413607047E8C901204D
:100B3000881802200020704738B58B7904460D468E
:100B40008BB18888400014F096FAAB79AA882060AF
:100B5000A280A371A060E0601BB12968520016F06A
:100B600087FF204638BD0868EFE7F8B5044617460A
:100B70000E461D46FFF7E0FF394604F11000FFF76F
:100B8000DBFFB2882585930802F0030223626262CC
:100B90002046F8BD816803468A1E8260B1F90000D4
:100BA00019688A4206D29A8802F10042013A01EBA2
:100BB000420199607047C3692DE9F74F044683618C
:100BC00000F11007981CE0611980A28A236903EBE9
:100BD0004202904218BFE369E361236A4FF0000AC2
:100BE0001D464FF000084FF0000926680193384673
:100BF00036F90AB0FFF7CEFFCBFB808906EB0A0B74
:100C00003846BBF902200092FFF7C4FF009AC2FBEE
:100C10008089BBF9042000923846FFF7BBFF009A99
:100C2000BBF906B0C2FB80893846FFF7B3FF013D30
:100C3000019BCBFB80890AF1080AD6D106EBC306DB
:100C4000636AAB420AD8B4F928204046D317494614
:100C500015F046FC00B203B0BDE8F08F384636F917
:100C600002ABFFF797FF0135CAFB8089E8E7000078
:100C700010B5034B0360044612F0B8FD204610BDCA
:100C8000B88B010810B50446FFF7F2FF2046082193
:100C900014F0EDF9204610BD2DE9F041044640F86E
:100CA0000C1B022788B06060A7600822002116F0A4
:100CB00043FE00251B4B01951A6B25753A431A63B9
:100CC0001A6BDFF86C803A400192019A02951A6B18
:100CD00042F004021A631B6B059503F0040301261E
:100CE000029303A94046029B03960496069503F0DF
:100CF0007FFE1023039303A90B4B0C480493059626
:100D0000069703F075FE2A4609210A2003F018FC15
:100D100040463246314603F057FF204608B0BDE852
:100D2000F08100BF0038024000002110000802409E
:100D30000004024070B504460D4616462A460021BE
:100D4000206800F0A9F900222068114600F0A4F9FB
:100D500035B183B2B34203D00A2003F0CBFBEDE7F9
:100D600070BD10B54031044601EB0222006800213D
:100D700000F092F9002220681146BDE8104000F012
:100D80008BB9F8B50E461746002140F2FF221D46EA
:100D90000446FFF7CFFF45F2065211462046FFF703
:100DA000C9FF760038220B212046FFF7DAFF06F054
:100DB000FE020D212046FFF7D4FF05EB4712D2B209
:100DC0000E212046FFF7CDFF01232375F8BD00005B
:100DD00010B503220F210446FFF7C3FF4FF44C5216
:100DE00011462046FFF7A6FF45F205521146204660
:100DF000FFF7A0FF034812F01AFD034B4FF4806287
:100E00001A6010BDF0C9012000E100E007B50A48F2
:100E100001A912F017FD019B012B09D14FF0E0232E
:100E20004FF08052C3F8042DBFF34F8FBFF36F8F85
:100E300003B05DF804FB00BFF0C9012002484FF089
:100E4000FF3112F0E9BC00BFF0C9012010B588B035
:100E500005AA0F4B019304460323039201A903AA99
:100E600000680293049300F0F5F8039B206859682A
:100E700001F075FE6368000A1860039B206899689A
:100E800001F06DFE6368000A586008B010BD00BF35
:100E9000C08B0108436853F82100704708B5102043
:100EA00003F09EFEBDE80840FFF7B0BFF0B589B083
:100EB0001E4B0160002601961A6B42F002021A6373
:100EC0001A6B02F002020192019A02961A6B42F02A
:100ED00004021A631B6B03F004030293029B4FF49A
:100EE00080430125044603930227114B11480493C4
:100EF00003A90595069703F07BFD324609212820BA
:100F000003F01EFB059606F1804606F5023603A99E
:100F1000304603950495069703F06AFD30462A464D
:100F2000294603F051FE204609B0F0BD00380240CA
:100F300000002110000402401FB503238022C94392
:100F400019408DF8062001AACDE902238DF805107D
:100F500000688DF8043002AA012100F0BFF805B046
:100F60005DF804FB1FB503AB0193303103230293FB
:100F70008DF80C10130A8DF80E2000688DF80D30D6
:100F800001AA012100F0AAF805B05DF804FB1A449B
:100F900092B2FFF7E7BF01607047000010B5064C42
:100FA00000220121204612F055FC2046034A044944
:100FB000BDE81040FFF7ABBDF0C90120350B0008BC
:100FC000710C0008054810B5044654F808391B6830
:100FD00098472046FFF74CFE10BD00BFA0CF012070
:100FE000054810B5044654F808391B689847204650
:100FF000FFF73EFE10BD00BF90CF0120054810B5A1
:10100000044654F808391B6898472046FFF730FE1D
:1010100010BD00BF80CF0120054810B5044654F82C
:1010200008391B6898472046FFF722FE10BD00BF15
:1010300070CF0120064838B50624013CA0F1080510
:1010400005D0036A20301B6898472846F5E738BD6D
:1010500040CF012008B54B681268096805489B001D
:101060009BB206F0A7F9BDE8084003484FF0FF31F6
:1010700012F0D2BB10D00120B0CF012021B904481A
:101080004FF0FF3112F0C8BB02484FF0FF31F9E7D3
:10109000B0CF0120A8CF012030B585B00546019220
:1010A0000C4669B904230B4803AA0DEB030106F0B3
:1010B00081F928462146FFF7E1FF039805B030BDCE
:1010C0000548022201A906F009F941F234230393ED
:1010D000EFE700BF10D00120B8CF012038B513468C
:1010E0000C1E1968064B92880546064818BF18461C
:1010F00006F0F4F821462846BDE83840FFF7BEBFA9
:10110000B8CF012010D0012038B5094B094C5D5CE7
:10111000094B20465A5C4FF4806103F055FD2A4686
:1011200020464FF40051BDE8384003F04DBD00BFEC
:10113000328C010800140240358C01080A1E034855
:1011400018BF0122202103F03FBD00BF0010024064
:101150000A1E034818BF0122402103F035BD00BF1D
:101160000010024000B58BB0254B264800220192AA
:10117000196B41F008011963196B01F00801019125
:1011800001990292196B41F010011963196B01F07A
:101190001001029102990392196B41F02001196329
:1011A000196B01F02001039103990492196B41F02E
:1011B000400119631B6B079203F040030493049BE7
:1011C00008924FF44053059305A90123069303F0B9
:1011D0000FFC602305A90C48059303F009FC42F2BB
:1011E0000C4305A90948059303F002FC4FF498430A
:1011F0000748059305A903F0FBFB0BB05DF804FB62
:1012000000380240000C024000100240001402406E
:10121000001802402DE9F04F8FB04FF0000ABD4C8E
:10122000CDF808A0236BBC48BC4D43F001032363F9
:10123000236B03F001030293029BCDF80CA0636CB7
:1012400043F480536364636C03F480530393039B00
:101250000226A02309A94FF003084FF005090993BE
:101260000A960B96CDF83080CDF8349003F0C0FB91
:101270001023A94809930127122309A90A930B9760
:1012800003F0B6FB4023A448099309A9CDF82CA08C
:1012900003F0AEFBA24B2B604FF482736B604FF4F4
:1012A0008023AB610823EB6128460A23C5F808A018
:1012B000C5F80CA0C5F810A06F61C5F820A0C5F84E
:1012C00024A0C5F828A0EB6205F0C6FF08B103F022
:1012D000D9F80490236BDFF86CA2924A43F48003A0
:1012E0002363236BCAF8002003F480030493049B58
:1012F000CAF80C004023CAF808304FF480634FF05E
:101300008062CAF81030CAF81400CAF81800CAF887
:101310001C004FF40033CAF82C00CAF830004FF01C
:10132000040B5046CAF80420CAF82030CAF824B08A
:10133000CAF8288003F088F902460028C7D1394648
:1013400001903A2003F0FCF83A2003F02BF9C5F89D
:1013500048A0CAF83850DFF8F0A17349CAF8001065
:101360004FF0C061019ACAF804104FF480634FF443
:1013700040315046CAF824B0CAF80820CAF80C20F8
:10138000CAF81030CAF81420CAF81820CAF81C206D
:10139000CAF82010CAF82880CAF82C20CAF83020D1
:1013A00003F052F98346002891D10246394638208D
:1013B00003F0C6F8382003F0F5F85A4631462320EA
:1013C000C5F84CA0CAF8385003F0BAF8232003F04F
:1013D000E9F8CDF814B0236B5448554D43F002039F
:1013E0002363236B03F002030593059BCDF818B02C
:1013F000236B43F004032363236B03F0040306937E
:10140000069BCDF81CB0236C43F480432364236C0B
:101410000A9603F480430793079B0B96082309A9B8
:101420000993CDF83080CDF8349003F0E1FA4FF411
:1014300000534048099309A9CDF82CB0CDF8349059
:1014400003F0D6FA4FF480533A48099309A91223BE
:101450000A930B97CDF8349003F0CAFA364B2B6001
:101460004FF482736B604FF40043AB604FF4802302
:10147000AB610823EB6128460A23C5F80CB02E6146
:10148000C5F814B0C5F820B0C5F824B0C5F828B028
:10149000EB6205F0E1FE00287FF419AF0890236BA2
:1014A00043F400132363236B244C03F400130893C9
:1014B000089B234B23604023A3604FF4806360604C
:1014C000E06023616061A061E0614FF4003360621D
:1014D000E06220632046C4F82880236203F0B4F859
:1014E000804600287FF4F3AE024639460F20AC64F4
:1014F000A56303F025F80F2003F054F84246314667
:10150000242003F01DF8242003F04CF80FB0BDE8B0
:10151000F08F00BF003802400000024010D00120D0
:101520000030014040640240106402400008024064
:10153000B8CF0120000402400038004020CC012038
:1015400070600240E0CD012080CD01202DE9F04FF8
:101550008DB0844C8448854F002502950995236CF5
:1015600043F400132364236C03F400130293029BDF
:101570000395236C43F480032364236C03F48003FA
:101580000393039B0495236B43F002032363236BB4
:1015900003F002030493049B4FF0120BC0234FF09F
:1015A000020A4FF0040907A90793CDF820B0CDF83F
:1015B00028A0CDF82C9003F01BFA6D4B6D4ABD604E
:1015C000C7E900234FF480486E233846FB60C7F814
:1015D00010807D61BD61FD613D6203F0EDFC08B1ED
:1015E00002F050FF0590226B634E42F4001222631A
:1015F000226BB06002F400120592059A5F4A3260D5
:10160000F0604FF000727061B061F0614FF48033B0
:1016100070624FF48065304672603561336203F06A
:1016200013F802460028DBD101900C210B20BE6389
:10163000B76302F085FF52495248019A086040267C
:1016400008464A60CA604A618A61CA610A624A629F
:101650008E600D6102F0F8FF02460028C0D14849B3
:1016600079638F6301900D210C2002F069FF012343
:101670003D48099307A9CDF82C900795CDF820B0E7
:10168000CDF828A003F0B4F94FF40073DFF80C9103
:101690003548079307A909230B9303F0A9F93A4B9F
:1016A000C9F80030324B019AC9F8043048466E231D
:1016B000C9F80820C9F80C30C9F81080C9F81420FE
:1016C000C9F81820C9F81C20C9F8202003F074FCC0
:1016D000002885D10690236B43F400132363236B0A
:1016E0002A4C03F400130693069B294BA0604FF08D
:1016F0006068C4E90038E0606061A061E0614FF4B7
:101700008033606220462561236202F09DFF074618
:1017100000287FF465AF0246C9F83840C4F8389015
:101720000C211C4C0D2002F00BFF1B4BA660204629
:10173000C4E90038E76025616761A761E761276256
:10174000676202F081FF024600287FF449AF0C2156
:101750002F20C9F83440C4F8389002F0F1FE0DB0E3
:10176000BDE8F08F00380240000402404CCA01205E
:10177000801A06000054004060CB01201060024037
:10178000C0CB01202860024000580040A0CA0120C0
:101790004060024000CB0120B8600240F8C901203F
:1017A0002DE9F04188B000263F4C0096236B3F4D59
:1017B0003F4843F001032363236B03F001030093CD
:1017C000009B0196236C43F400332364236C03F4E1
:1017D00000330193019B0223049301230C270593FB
:1017E000032306930DEB070107230793039703F0E9
:1017F000FFF8304B2B6028464FF4E1336B60AE604E
:10180000EE602E616F61AE61EE6106F0D2F908B153
:1018100002F038FE0290236B43F400132363236B22
:10182000254C03F400130293029B244BA060E0605C
:101830006061A061E061206260624FF000684FF477
:1018400080672046C4E90038276102F0FDFE0646A5
:101850000028DDD102460D2110206C63A56302F043
:101860006FFE102002F09EFE154C164BE660C4E998
:10187000003820464023A36027616661A661E661C7
:101880002662666202F0E0FE02460028C0D10D2109
:1018900011202C63A56302F053FE112002F082FE9A
:1018A00008B0BDE8F08100BF0038024040CD012003
:1018B000000002400044004080CC012088600240CB
:1018C000E0CC0120A06002402DE9F04F8BB0624CCB
:1018D000624800270197236B43F004032363236BC3
:1018E00003F004030193019B0297236B43F0400331
:1018F0002363236B03F040030293029B0397636C03
:1019000043F020036364636C03F020030825022680
:101910004FF0030803934FF0010A05A94FF0400967
:10192000039B0995CDF814900696CDF81CA0CDF830
:10193000208003F05DF84FF400734948059305A932
:1019400009950696CDF81CA0CDF8208003F050F83C
:101950004FF440534248099505A9424D0593069618
:101960000797CDF8208003F043F83F4B2B603F4BA7
:101970006B604FF44073AB614FF40043EB6128465A
:101980000C23AF60EF602F616B6106F012F908B1B4
:1019900002F078FD0490236B43F480032363236BF0
:1019A000334C03F480030493049B324BA0604FF04C
:1019B000206AC4E9003AE0606061A061E0614FF430
:1019C0000033E06220634FF4806804272046C4F8A7
:1019D000108023626762A66202F036FE834600280A
:1019E000D6D10246062139206C63A56302F0A8FD1A
:1019F000392002F0D7FD204C204BA662C4E9003A02
:101A000020464FF48033C4F80890C4F80CB0C4F8F2
:101A10001080C4F814B0C4F818B0C4F81CB0236225
:101A20006762C4F82CB0C4F830B002F00DFE064670
:101A30000028ADD10246062146202C63A56302F0A2
:101A40007FFD462002F0AEFD32460A21472002F01B
:101A500077FD0BB0BDE8F08F00380240000802406F
:101A60000018024000CF01200014014080841E00B5
:101A700040CE012028640240A0CE0120B86402407C
:101A800037B5044601F0E0FB40F20E2204F5AA70DF
:101A9000C4F850210021C4F84C01012515F04CFF79
:101AA00002F0EEFC14490095802304F559720020E1
:101AB00002F0B4FC00280DDB10490095802304F5EA
:101AC0007972284602F0AAFC002803DB0C490020AA
:101AD00002F096FC2046FFF745FB2046FFF79AFBF5
:101AE0002046FFF733FD2046FFF75AFE2046FFF75A
:101AF000EBFE204603B030BDCC8B0108DC8B010827
:101B0000EB8B01080268136823F040031360064B57
:101B1000984202D1054801F091B9054B984201D194
:101B20000448F8E7704700BF10D00120B0CF012073
:101B3000B8CF0120A8CF0120054B984207D10268F9
:101B40000448136823F04003136001F077B970472D
:101B500010D00120B0CF0120014803F003BE00BF28
:101B60004CCA0120014804F06BBA00BF4CCA0120E6
:101B7000014803F0F7BD00BFF8C90120014804F097
:101B80005FBA00BFF8C90120014805F09DBD00BF44
:101B900010D00120014805F097BD00BFB8CF01204B
:101BA00008B5044806F06EF8BDE80840024801F0A8
:101BB00045B900BF40CD012098CF012070B50F4C32
:101BC00094F83A6094F83950F6B2204606F05AF884
:101BD000222EEDB208D194F83A30202B0CD10848CF
:101BE000BDE8704001F02AB9212D05D194F83930B3
:101BF000202B01D10348F3E770BD00BF00CF0120C7
:101C000088CF012090CF012010B5074C204602F06C
:101C10002DFE94F83530012B04D1BDE81040034867
:101C200001F00CB910BD00BF60CB012078CF0120BE
:101C300010B5074C204602F019FE94F83530012B00
:101C400004D1BDE81040034801F0F8B810BD00BF52
:101C5000C0CB012080CF012010B5074C204602F0F8
:101C600005FE94F83530012B04D1BDE8104003483F
:101C700001F0E4B810BD00BFA0CA012068CF012068
:101C8000014802F0F3BD00BF20CC012010B5074C85
:101C9000204602F0EBFD94F83530012B04D1BDE86D
:101CA0001040034801F0CAB810BD00BF80CC01202D
:101CB00098CF012010B5074C204602F0D7FD94F8CC
:101CC0003530012B04D1BDE81040034801F0B6B80F
:101CD00010BD00BF00CB012070CF0120014802F0F1
:101CE000C5BD00BF80CD012010B5094C204602F0D3
:101CF000BDFD94F83530012B08D1064B0648202253
:101D0000BDE8104083F8392001F098B810BD00BF3D
:101D100040CE012000CF012088CF0120014802F0F1
:101D2000A5BD00BFE0CD012010B5094C204602F052
:101D30009DFD94F83530012B08D1064B0648202232
:101D4000BDE8104083F8392001F078B810BD00BF1D
:101D5000A0CE012000CF012090CF012010B5044675
:101D6000FFF78EFE214604F26440FEF795FF214600
:101D700004F27C40FFF79AF8214604F59060FFF7E3
:101D80000AF9204610BD000038B5002201212F4875
:101D90002F4D11F05FFD2F4A2F492C48FEF7B7FE5B
:101DA000002201212D4811F055FD2A4A2A492B48CD
:101DB000FEF7ADFE00220121294811F04BFD002263
:101DC0000121284811F046FD224A27490020FEF74C
:101DD0009EFE00220121254811F03CFD0022012138
:101DE000234811F037FD1B4A22490020FEF78FFEE1
:101DF00000220121204811F02DFD002201211F4861
:101E000011F028FD134A1E490020FEF780FE002233
:101E100001211C4811F01EFD002201211A4811F079
:101E200019FD0C4A19490020FEF771FE00242819FB
:101E300000220121083411F00DFD282CF7D1BDE856
:101E40003840044A12490020FEF761BEB0CF01209D
:101E500040CF0120350B0008710C0008A8CF0120ED
:101E600098CF0120A0CF0120C50F000888CF012006
:101E700090CF0120E10F000878CF012080CF012012
:101E8000FD0F000868CF012070CF01201910000855
:101E900035100008B420704730B5B328104C94BFFB
:101EA000054600252580B3290E4C94BF0D4600251C
:101EB00025801418B42CDCBF02F1FF3280180A4AC6
:101EC000D4BF80B2B32010805A18B42ADCBF03F10B
:101ED000FF33C918054BD4BF89B2B321198030BD77
:101EE0006AD0012068D001200200002000000020FC
:101EF00008B501F061FB4FF6FF7008BDB4207047D4
:101F000038B50C46154601F0DFFB2544AC4200D144
:101F100038BD14F8010B01F0D1FBF7E708B500223A
:101F200011462920FFF7ECFF0022BDE808401146CA
:101F30003820FFF7E5BF37B501F03EFB0024012252
:101F400001A935208DF80440FFF7DAFF06230122AE
:101F500001A93A208DF80430FFF7D2FF4FF6016354
:101F6000022201A9B020ADF80430FFF7C9FF42F208
:101F7000DE13022201A9B120ADF80430FFF7C0FF43
:101F800043F20533022201A9B720ADF80430FFF770
:101F9000B7FF022201A9B820FFF7B2FF4FF4417347
:101FA000022201A9C820ADF80430FFF7A9FF40F6CE
:101FB0005E03022201A9C9200225ADF80430FFF713
:101FC0009FFF40F60A43032201A9CA20ADF804305E
:101FD0008DF80650FFF794FF40F203432A4601A90B
:101FE000CC20ADF80430FFF78BFF0C23012201A9B0
:101FF000D0208DF80430FFF783FF012201A9B32020
:102000008DF80450FFF77CFF5323012201A9C02063
:102010008DF80430FFF774FF4FF48A432A4601A974
:10202000C520ADF80430FFF76BFF41F203232A46C9
:1020300001A9C220ADF80430FFF762FF012201A917
:10204000DD208DF80440FFF75BFF224601A9B42094
:10205000FFF756FF224601A91120FFF751FF9620F6
:1020600001F03DFB04221E230DEB02018DF805302B
:102070002A204FF45143ADF80630FFF741FF042208
:10208000B3230DEB02012B208DF805408DF80730AE
:10209000FFF736FF8323012201A936208DF8043093
:1020A000FFF72EFFFFF73AFF224601A92C20FFF78A
:1020B00027FF4BF6D854002001F000FB013CFAD179
:1020C000142003B0BDE8304001F009BB08B5002280
:1020D00011462820FFF714FF142001F000FB002216
:1020E00010201146FFF70CFFBDE80840962001F0D4
:1020F000F6BA13B5C0B200F11E028DF805202F38D4
:10210000042200230C468DF807000DEB02012A2063
:102110008DF804308DF80630FFF7F2FEE1B28DF84D
:10212000051004224D398DF807102B200DEB02010C
:10213000FFF7E6FE02B010BD38B5D50802F47843CB
:1021400005F0FC051D441446FFF7D3FF0022ADB295
:1021500011462C20FFF7D4FE284601F0AFFAE0022A
:1021600000F47840BDE8384001F0A8BA38B504461C
:102170000D46FFF7BEFF29462046FFF7BAFF0022B3
:1021800011462E20FFF7BCFE01F0A4FA01F0A2FADE
:10219000044601F09FFAC4F38502C0F3C42303EBA5
:1021A000421304F47844181980B238BD2DE9F8437D
:1021B000044604F01F0508461E461146C4F34513A5
:1021C0004FEAD428EF0004F4784404EB830407EBCF
:1021D0008327FFF78EFF002211462C204FEAC80804
:1021E000FFF78EFE08EBC528A4B21FFA88F8BFB22D
:1021F000002506F1FF39B54201D3BDE8F88320463A
:1022000001F05CFA404601F059FA4D4502D03846DB
:1022100001F054FA0235ADB2EDE7F8B50E460746C7
:102220001146304614461D46FFF763FF0022114653
:102230002C20FFF765FE2544ADB2AC4200D1F8BDBD
:1022400021463A4630460134FFF776FFA4B2F4E760
:102250002DE9F84F9046002206460F462C201146E5
:102260001D46FFF74DFE34464FF0000A08EB060905
:102270004C4501DBBDE8F88F1F4B1A88A24237D8C6
:102280001E4B1A88BA4233D81D4B1A88A2422FD34C
:102290001C4A1288BA422BD335F81AC04FEADC0028
:1022A0004FEA4A0B0CF4784C00F0FC0060440BF150
:1022B000020B80B201F002FA35F80BC035F81A00B3
:1022C0004FEADC2CC00200EBCC0080B201F0F6F942
:1022D00009F1FF31A14209D035F80B20D000C0B27E
:1022E000520900EB822080B201F0E8F90AF1020AFB
:1022F0000234A4B2BAE700BF6AD0012068D001203E
:102300000200002000000020184B2DE9F0471D8836
:10231000174B074617481B88048817480135ED1AE4
:1023200053889388538900880E4691899BB2013463
:10233000ADB2241A43EA014316FA84F44FEA450980
:1023400002EB0308A64201D3BDE8F087013C1FFA67
:1023500084FA51463846FFF7CCFE43462A4651469A
:102360003846FFF775FFC844ECE700BF02000020C5
:102370006AD001200000002068D001202DE9F0473C
:10238000DDF82080054616460C464FEA420ACF1873
:10239000A74201D8BDE8F0871FFA84F949462846CC
:1023A000FFF7A7FE4346324649462846FFF750FF4F
:1023B0000134D044ECE7F0207047000030B5EF283E
:1023C000104C94BF054600252580EF290E4C94BF84
:1023D0000D46002525801418F02CDCBF02F1FF32D9
:1023E00080180A4AD4BF80B2EF2010805A18F02A11
:1023F000DCBF03F1FF33C918054BD4BF89B2EF210D
:10240000198030BD6ED001206CD001203E0000202C
:102410003C000020F020704738B50C46154601F00E
:1024200053F92544AC4200D138BD14F8010B01F03A
:1024300045F9F7E7012813B504461DD002281DD140
:102440000F4B00930622002369463320ADF8043079
:10245000FFF7E2FF50232246694637208DF801300E
:10246000FFF7DAFFC0230122694636208DF80030DD
:10247000FFF7D2FF02B010BD0023F4E76023F2E7BC
:10248000000001F008B5002211462920FFF7C4FF23
:102490000022BDE8084011461120FFF7BDBF000033
:1024A00030B585B001F088F8002211461020FFF702
:1024B000B3FF0A2001F013F9002211460120FFF7B3
:1024C000ABFFC82001F00BF9002211461120FFF7E5
:1024D000A3FF782001F003F9002469460122362089
:1024E00005258DF80040FFF797FF694601223A2045
:1024F0008DF80050FFF790FF224621462120FFF77C
:102500008BFF4FF06F43694604222A200093FFF7A8
:1025100083FF694604222B20FFF77EFF40F60C4321
:10252000ADF800302A4633236946B2208DF80330D7
:102530008DF804303525FFF76FFF69460122B7207B
:102540008DF80050FFF768FF1F2369460122BB206A
:102550008DF80030FFF760FF2C2369460122C02070
:102560008DF80030FFF758FF4CF201336946022224
:10257000C220ADF80030FFF74FFF2023694601224B
:10258000C4208DF80030FFF747FF0F236946012272
:10259000C6208DF80030FFF73FFF4AF2A4136946CA
:1025A0000122D020ADF80030FFF736FF1E4B00931C
:1025B00003F12C5303F5201303F63C430193A3F1DD
:1025C000F953A3F5BB23A3F2BC630293694642F619
:1025D00029530E22E020ADF80C30FFF71DFF102329
:1025E0008DF8023040F20663ADF8043044238DF8D4
:1025F000073040F65133ADF80830162369468DF8A0
:102600000A300E2243F22F13E120ADF80C30FFF711
:1026100003FFFFF737FF0122694628468DF8004087
:10262000FFF7FAFE05B030BDD008110807B5FE234C
:1026300001A90122BD208DF80430FFF7EDFE002234
:1026400011461020FFF7E8FE0A2003B05DF804EB06
:1026500001F045B813B5C0B28DF805000422113859
:1026600000230C468DF807000DEB02012A208DF89F
:1026700004308DF80630FFF7CFFEE1B28DF805107B
:10268000042211398DF807102B200DEB0201FFF702
:10269000C3FE02B010BD10B51446FFF7DBFF0022E9
:1026A0002C201146FFF7B8FE2046BDE8104001F08F
:1026B00005B838B504460D46FFF7CCFF294620463D
:1026C000FFF7C8FF002211462E20FFF7A5FE01F0FC
:1026D00001F800F0FFFF044600F0FCFFC4F38502A0
:1026E000C0F3C42303EB421304F47844181980B2F6
:1026F00038BD70B50646084611461C46FFF7AAFFCE
:10270000002211462C20FFF787FE0025A54200D1AC
:1027100070BD304600F0D2FF0135F7E7F8B50E4640
:1027200007461146304614461D46FFF793FF002228
:1027300011462C20FFF770FE2544ADB2AC4200D10B
:10274000F8BD21463A4630460134FFF7A4FFA4B253
:10275000F4E700002DE9F84F1746002205460E4623
:102760002C2011469946DFF854A0DFF854B0FFF74B
:1027700053FE104A2C464FF000087B19A34201D8A3
:10278000BDE8F88FBAF80030A34211D8BBF800308A
:10279000B3420DD81388A3420AD3074B1B88B34218
:1027A00006D339F8180000F089FF024A08F1010841
:1027B0000134E2E73E0000203C0000206ED0012002
:1027C0006CD00120184B2DE9F0471D88174B0746A8
:1027D00017481B88048817480135ED1A53889388D9
:1027E000538900880E4691899BB20134ADB2241AF8
:1027F00043EA014316FA84F44FEA450902EB030861
:10280000A64201D3BDE8F087013C1FFA84FA514685
:102810003846FFF71FFF43462A4651463846FFF722
:1028200099FFC844ECE700BF3E0000206ED00120B5
:102830003C0000206CD001202DE9F047DDF820801D
:10284000054616460C464FEA420ACF18A74201D861
:10285000BDE8F0871FFA84F949462846FFF7FAFEDB
:102860004346324649462846FFF774FF0134D044B8
:10287000ECE708B500F028FF00F02CFF00F02AFF7D
:10288000C0B208BD08B500F097FE0420FFF7F1FFC5
:1028900008BD0000064838B50624013CA0F1080533
:1028A00005D0036A20301B6898472846F5E738BDF5
:1028B00030D10120012908B508D002290CD089B9EE
:1028C000094B185CBDE8084000F0CCBD064B185C15
:1028D000BDE8084000F0BABD034B185CBDE80840F5
:1028E00000F0CCBD01F0CEFD488C010810B599B1C7
:1028F00001291CD0164B174C33F81130E3604FF40C
:1029000048636360204600232361A36005F0B8F8A4
:10291000024680B101F0B6FD032000F0A3FD2C209B
:1029200001F04EFEBDE810400A4804F09BBF0320B2
:1029300000F08CFDF3E70E212C2001F001FE204673
:1029400004F080FFBDE810402C2001F02BBE00BF3A
:102950004C8C0108DCD10120032970B508461446CF
:102960000BDC1146FFF7A6FF70BD56F8040B21469D
:10297000FFF7A0FF013DF8D1F6E7014E0525F9E785
:10298000388C010870B54FF060434FF0E02501240A
:10299000D3F8000E04FA02F2D5F8FC4D44F080742E
:1029A000C5F8FC4D0F4CC3F8B04F0F4C002520EA82
:1029B000020001390226C3F8000EC3F8805EC4F895
:1029C000F06021610949C3F8405E094D0D604FF484
:1029D0008071C4F8041302430649C3F8801EC3F88B
:1029E000002E70BD55CEACC5000004E0001000E024
:1029F000FE0300400D000100F0B5A5B0364B0020ED
:102A000001901A6C42F080521A641B6C03F08053E0
:102A10000193019B314B02901A6842F440421A60C4
:102A20001B6803F4404302930D25029B4FF4A0233F
:102A30000224CDE908534FF480070123042508A898
:102A4000CDE90E47CDE91051CDE912450A930D931A
:102A5000149404F039F908B101F014FD0F26059023
:102A60004FF480530790032103A803960494069320
:102A700003F008FF0028EFD168231593482317932C
:102A8000032318934FF480731C931D904FF0006341
:102A9000229015A8199416951F9303F0D1FF0446B0
:102AA0000028D9D13946024603F06CFE03F0B6FE89
:102AB00003F082FF4FF47A73B0FBF3F001F08EFD68
:102AC000284601F09FFD224631464FF0FF3001F0CD
:102AD00037FD25B0F0BD00BF003802400070004057
:102AE00038B504462D200D4601F06AFD002001F0A6
:102AF00067FB7DB10121002003F048FB60212046E7
:102B0000FFF77AFF2D2001F04DFDBDE83840012090
:102B100001F056BB30BFF5E738B5FFF7E1FF074DD1
:102B20000124002105EBC40010F076FE08B1204618
:102B300038BD0134052CF4D10620F9E730D101204D
:102B4000132908B503D804F0DFFA002008BD0220DD
:102B5000FCE7132901D804F0DCBA0020704708BA5A
:102B60007047000070B588B0184C194800250195D1
:102B7000236B43F010032363236B069503F01003CC
:102B8000019303A90126019B04960F230393059645
:102B900001F02EFF284600F065FC304600F062FC94
:102BA000022000F05FFC032000F05CFC0295236C27
:102BB000084A43F080032364236C03F080030293EC
:102BC000029B054B1A6008B070BD00BF0038024080
:102BD00000100240001C0040DCD101202DE9F0472C
:102BE0008AB000243B4B01941A6B42F002021A6334
:102BF0001A6B02F002020192019A02941A6B42F0DF
:102C000020021A631A6B02F020020292029A0394C5
:102C10001A6B42F040021A631A6B02F040020392F0
:102C2000039A04949A6B42F002029A639B6B079496
:102C300003F002030493054602270326049B26485B
:102C40000697C0234FF0090A05A905934FF00A091A
:102C50000896CDF824A001F0CBFE4FF440731E4837
:102C6000059305A94FF00408069707940896CDF838
:102C7000249001F0BDFE1948CDF8148005A90697EF
:102C800007940896CDF824A001F0B2FE4023144822
:102C9000059305A9069707940896CDF8249001F0AE
:102CA000A7FE104B2B631023EB6317236C63C5F84F
:102CB00038802B646C64AC64EC642C6505F13000E6
:102CC00003F060FB08B101F0DDFB01F071F80AB020
:102CD000BDE8F087003802400014024000040240C2
:102CE00000180240001000A007B5002301930A4B12
:102CF0005A6B42F040025A635B6B03F0400301934E
:102D0000019B064B40F87C3F04F065F908B101F0E7
:102D1000B9FB03B05DF804FB003802400008065020
:102D20000A4A012108B5C2F83C1E094A02607F2107
:102D300000228160FF214260C160026142618261C4
:102D400004F094F908B101F09DFB08BD0000474272
:102D50000028004070B588B00026184B02961A6C07
:102D6000174C42F480721A641B6C03F480730D4696
:102D7000029301A903A8029B03F044FE03F022FE84
:102D8000104B236040F2E733E36040000E4BB0FB92
:102D9000F3F00138606020462661A66004F070FE02
:102DA000042229462D2001F0CBFB2D2001F0FAFB57
:102DB000204604F047FD08B070BD00BF0038024057
:102DC00058D101200020004040420F0038B5044691
:102DD0000D4601F033FA184B1A6842F400721A607B
:102DE0001A6842F480621A601A6842F480721A60AB
:102DF000032001F093FB0F212046FFF7ABFF29468C
:102E00002046FFF7F9FD03F009FD002208212046C6
:102E1000FFF7B8FD012000F03BFB2046FFF7A2FEC4
:102E20002046FFF7DBFE2046FFF75EFF2046FFF758
:102E300077FF204638BD00BF003C024007B501A91E
:102E400010F000FD58B1019B4BB14FF0E0234FF063
:102E50008052C3F8042DBFF34F8FBFF36F8F03B0C1
:102E60005DF804FBFEE7FEE7FEE7FEE7FEE77047DE
:102E7000012001F0B5BE022001F0B2BE08B54FF44A
:102E8000804001F0ADFEBDE808404FF4004001F085
:102E9000A7BE0000102808B51ED005D801280BD009
:102EA000022815D001F0EEFAB0F5804F12D0B0F53F
:102EB000004FF7D1094807E000F068FB084B0038E5
:102EC00018BF012003EB4010BDE80840FFF7B6BF74
:102ED0000448F9E70448F7E708BD00BF40D10120E6
:102EE00030D1012038D1012048D1012008B5034854
:102EF00004F0D2FC024B01221A7008BD9CD10120C3
:102F000098D1012008B5044804F0C6FCBDE808408B
:102F1000032000F0B3BA00BFDCD1012008B503489C
:102F200004F0BAFCBDE8084001F0D2BA58D1012043
:102F3000014801F09BBC00BF70D00120014801F0A6
:102F400095BC00BFD0D0012038B5084D0024281909
:102F500000220121083410F07DFC282CF7D1BDE8B7
:102F60003840034A03490020FDF7D1BD30D101208C
:102F7000350B00089528000810B54FF6FF7000F0DB
:102F8000E5FC002000F0FCFB4FF6FF7000F0FEFBBC
:102F9000084800F001FC084A01236421002000F0E9
:102FA0005FFCBDE81040054A01237821002000F0B5
:102FB00057BC00BF80000020588C0108648C0108B9
:102FC00070B504460D46204600F0B6FFE8B9B5B925
:102FD0002378D3B901F088FA86B2204600F0ACFF1E
:102FE0000028FAD1ADB92378013B012B16D8642013
:102FF00001F080FA6420BDE8704001F07BBA012D39
:1030000003D12378013B012BE4D9642001F072FA4B
:10301000D9E7012D02D12378002BE8D001F064FA22
:103020006438B0424FF06400E5D801F063FAD4E7A9
:10303000F8B51E46164B33F81150044600201746CB
:1030400000F09EFB29461422284600F007FD4FF6AB
:10305000FF7000F095FB0A222946284600F0FEFC8E
:1030600020460121FFF7ACFF63883B80E388338073
:1030700000212046FFF7A4FF4FF6FF7000F080FB11
:10308000294628461422BDE8F84000F0E7BC00BFFE
:10309000DE8C010838B500210446C068FFF759FDF1
:1030A000A8B36082000CA0820125E0680121FFF72F
:1030B00050FD70BB2046FFF75FFF00F051FB054657
:1030C00000F056FB012281B2A8B200F009FF0546CC
:1030D000002837D04FF6FF7000F058FB4FF47840CF
:1030E00000F04EFB294A01239121002000F0B8FB9B
:1030F000274A0123A021002000F0B2FB012D10D1AE
:10310000244A2B46AF21002000F0AAFB06E005462A
:10311000CBE7E082000C2083002DCBD0012020746F
:1031200038BD022D07D100F023FB1B4AA0F141015D
:10313000012389B2E7E700F01BFB184AA0F1410127
:103140000123F6E7234604F1120203F8140B0146AB
:103150002046FFF76DFF638AA28AE06843EA0242D5
:103160002946FFF7EDFC234604F1160203F8185B2D
:1031700020460121FFF75CFFE38A228BE06843EAE7
:1031800002420121FFF7DCFCC8E700BF708C010898
:10319000768C0108978C0108B38C0108C78C010854
:1031A00013B5002301930374094BC1601A6B42F4F9
:1031B00080521A631B6B03F4805301930446019BF6
:1031C00010F0A8FA042006F04BF8204602B010BD1B
:1031D0000038024038B504460BF094FE022000F09F
:1031E0009FFC00F0BDFA054600F0C2FA022281B24F
:1031F000A8B200F075FE30B92046FFF74BFFBDE8DE
:10320000384000F02FBF38BD0D4B13B55C6920204E
:1032100001F0E6FCA30610D50A4801A910F012FB44
:10322000019B012B09D14FF0E0234FF08052C3F8EE
:10323000042DBFF34F8FBFF36F8F02B010BD00BFDF
:10324000003C01401CD2012010B50446FFF7BEFD32
:10325000214604F59870FFF7A3FF204610BD00003B
:1032600010B5064C00220121204610F0F3FA20464A
:10327000034A0449BDE81040FDF749BC1CD20120B7
:10328000350B0008710C000870B58AB0064602F0D4
:1032900079FF002840F09C804E4B4F4C9E420CBF63
:1032A0004E4A4F4A32604F4A726000254FF48042C6
:1032B0009E42B560F56032617561B561F561356258
:1032C00044D10195236B484843F002032363236BE9
:1032D000079503F002030193019B402305931223FA
:1032E00006930223089305A90423099301F080FBA8
:1032F00080233D48059305A901F07AFB0295236CD4
:1033000043F400132364236C03F400130293029B21
:10331000236A43F400132362236A23F40013236215
:103320002A460F211F2001F00BF91F2001F03AF966
:1033300020202A460F2101F003F9202001F032F964
:1033400030460AB0BDE8704001F036BE0395236BED
:10335000254843F002032363236B079503F0020320
:103360000393039B4FF48063059312230693022378
:10337000089305A90423099301F03AFB4FF4007365
:103380001948059305A90923099301F031FB049518
:10339000236C43F480032364236C03F480030493BD
:1033A000049B236A43F480032362236A23F480038B
:1033B00023622A460F21212001F0C2F8212001F0CA
:1033C000F1F822202A460F2101F0BAF82220B5E7B1
:1033D0000AB070BD24D201200038024000540040E1
:1033E00000580040A08601000004024030B585B0BE
:1033F0004FF47A740294BDF824400194089C009420
:10340000054601F099FE044628B1284601F07BFEEE
:103410002846FFF739FF204605B030BD30B585B0EE
:103420004FF47A740294BDF824400194089C0094EF
:10343000054601F011FF044628B1284601F063FE5D
:103440002846FFF721FF204605B030BD034B002280
:1034500033F82010024801F0B7BB00BF088D010807
:1034600000100240034B012233F82010024801F003
:10347000ABBB00BF088D010800100240024B33F8BF
:103480002010024801F0A5BB088D01080010024081
:103490002DE9F0478AB000250223DFF8E880DFF845
:1034A000E890354C0795064608932F46032D42D8E1
:1034B000DFE805F002202B360097236B43F0010371
:1034C0002363236B03F001030093009B39F8023B55
:1034D0000593002E3AD1D8F80000069605A901F010
:1034E00087FA0135052D08F10408DFD100200AB064
:1034F000BDE8F0870197236B43F040032363236B00
:1035000003F040030193019BE0E70297236B43F034
:1035100020032363236B03F020030293029BD5E770
:103520000397236B43F020032363236B03F02003F3
:103530000393039BCAE70497236B43F04003236381
:10354000236B03F040030493049BBFE7012EC8D113
:103550000A4BD8F80000069305A901F049FA084B78
:1035600013F905A0002250460F2100F0E9FF504654
:1035700001F018F8B5E700BF003802400000211044
:10358000E28C0108F48C0108E88C010870B5084D44
:10359000084E002436F8021B55F8040B01F00EFB10
:1035A00008B1E0B270BD0134052CF3D12046F9E733
:1035B000F48C0108E88C010810B5ACB04FF0204342
:1035C000189303F582730124199307220923CDE987
:1035D0000A34139224231022CDE90C341D920023C7
:1035E0004FF48052CDE922234FF48042CDE92423C9
:1035F0004FF400120221CDE928232C4A1493CDE97F
:103600000E11CDE91034CDE91A33CDE91E33CDE9E1
:1036100020331591169117931C9326931294279398
:103620000193906B20439063906B20400190019830
:103630000293106B40F008001063106B00F008005C
:10364000029002980393106B40F010001063106B0F
:1036500000F01000039003980493136B144843F098
:1036600020031363136B069103F020030493049B60
:103670000794032308930C23099305A94CF2B37311
:10368000059301F0B5F94FF6807305A90948059334
:1036900001F0AEF905A90848059401F0A9F911AAAD
:1036A0000AA918A804F0A3F82CB010BD00380240F5
:1036B000000C024000100240001402404FF0C043D2
:1036C0005880BFF34F8F70474FF0C0431880BFF34F
:1036D0004F8F70474FF0C043588880B2704700F05A
:1036E00009BF00000148FFF7CFBD00BF24D2012071
:1036F000FFF7F8BF1FB501238DF80F200DF10F0262
:10370000009201930A4601460248FFF76FFE05B09A
:103710005DF804FB24D201201FB500230A468DF872
:103720000F300DF10F010123009101930146044870
:10373000FFF774FE9DF80F0005B05DF804FB00BFB5
:1037400024D2012007B5CDE900230A460123014612
:103750000248FFF763FE03B05DF804FB24D20120AA
:1037600008B5024B1B689B6A984708BD78D20120B8
:1037700008B5024B1B68DB6A984708BD78D2012068
:10378000014B1860704700BF7CD20120014B58608C
:10379000704700BF7CD20120014B9860704700BF8A
:1037A0007CD20120024B1B685B6903B1184770474C
:1037B00078D201202DE9F04F284B85B0203A0291B4
:1037C00099680190B1F804B0B1F806A00D680BF14A
:1037D0000706F6100AFB02F2CBEBC60006FB025509
:1037E0000BF1FF3252FA80F34FF000080393029B73
:1037F00003EB08091FFA89F3D045009302D305B003
:10380000BDE8F08F012E2C7806D0022E6A780CD1FC
:1038100044EA022464BAA4B2DFF840900027BB4512
:1038200009D808F101083544E1E7240444EA0224F8
:10383000AA781443F0E7019BD819039B0122D91BF6
:103840008A40224214BFB9F80020B9F80420009938
:1038500080B2FFF7A7FF0137E1E700BF7CD201206C
:103860002DE9F047054610469A460E46904614F05C
:103870000DF9224F8146FFF773FFBB68BAF1010FC4
:103880009B88B0FBF3F41ED0BAF1020F22D02BB20A
:10389000002BD8BF012508F1FF38002418F8019F3C
:1038A000B9F1000918BF4FF00109FFF759FFBB68D4
:1038B0009B8803FB140080B2984202D3B9F1000F39
:1038C0000ED1BDE8F087A4EB09045C4305EB54007E
:1038D00085B2DCE7A4EB090414FB03F4601BF7E7F3
:1038E000284698F800203146FFF764FFBB689B88A4
:1038F00001342B449DB2A4B2D0E700BF7CD201209A
:10390000104B1B682DE9F0411C6A06460F46154610
:10391000A4B113460A4601460B48A4460088BDE8F8
:10392000F04160473019B8F80020394680B2FFF7FF
:1039300039FF0134AC42F5D3BDE8F081DFF80880EF
:10394000F8E700BF78D201207CD20120F8B50A4DFB
:103950002E682860FFF70CFF00240746BC4202D106
:10396000B6B22E60F8BDFFF7FBFEA1B282B2002016
:10397000FFF7C6FF0134F1E77CD201202DE9F04FBB
:103980005400344F85B082468B461546C4F103047B
:103990004FF000091FFA85F81AFA89F39BB2ABEBD6
:1039A00008011FFA89F689B218463A8800930291F5
:1039B000FFF7F8FEAAEB06039BB218463A88029975
:1039C0000193FFF7EFFE08EB0A039BB2ABEB060196
:1039D00089B218463A8802930391FFF7E3FEAAEBF7
:1039E00008039BB2D844184603993A8803931FFAF8
:1039F00088F8FFF7D7FE5E443A8800984146FFF703
:103A0000D1FEB6B23A8801984146FFF7CBFE3A881C
:103A100002983146FFF7C6FE039B3A8818463146A6
:103A2000FFF7C0FE002C0C4BBB60B5BF0634A9EB02
:103A3000050304EB89040A34A8BF05F1FF3509F139
:103A40000109A8BF04EB83044D45A3D205B0BDE82E
:103A5000F08F00BF7CD20120780000202DE9F74FC5
:103A6000DFF8B8B05400BBF80030CBF80030814626
:103A70000E469246C4F1030417460025C7B11FFA4B
:103A800087F8A9EB08004FEA48081FFA88F816FAE9
:103A900085F180B2ABB2424689B201930090FFF744
:103AA0002FFF019B0098F11A424689B2FFF728FFC9
:103AB000BDB11FFA85F8BBB2A9EB08004FEA480870
:103AC000F11A1FFA88F880B2424689B20193009039
:103AD000FFF716FF019B00989919424689B2FFF73C
:103AE0000FFF002CB5BF0634EB1B04EB85040A3432
:103AF000A8BF07F1FF3705F10105A8BF04EB830458
:103B0000AF42BBD2BBF80030CBF800305246314652
:103B1000484603B0BDE8F04FFFF730BF7CD201202C
:103B2000F8B52A4D2A4BAB6000264FF6FF770446C6
:103B30002E606F60FCF7ECFD26480122202101F089
:103B400043F832464FF40061234801F03DF8052068
:103B500000F0D0FC01224FF400611F4801F034F85E
:103B60000A2000F0C7FC32464FF400611A481B4E91
:103B700001F02AF8142000F0BDFC01224FF400618E
:103B8000154801F021F80A2000F0B4FC736898474A
:103B900085280ED1124B1E60336898471CB9204609
:103BA000FEF748FC01E0022CF9D00E4BAB60002080
:103BB000F8BD0D4C63689847B84204D1084B1C60AF
:103BC00023689847F1E70120F2E700BF7CD201208B
:103BD0008800002000140240000C02404000002039
:103BE00078D20120780000200400002000B595B0B4
:103BF0004FF480720C92052206920022CDE9122227
:103C00000D920E920B921192009204924FF08071DD
:103C100010220F91029201214FF48002034601917C
:103C20000391059206A96A46044802F057FC003841
:103C300018BF012015B05DF804FB00BF88D2012039
:103C400000B595B04FF480730C9306230693174884
:103C5000002341F2883206A9CDE90E33CDE91233B3
:103C60000D930B93119302F0F3FBE0B90223CDE91E
:103C7000003301221023CDE902324FF48003059373
:103C8000052306934FF0807304900F93074841F289
:103C900088336A4606A902F021FC003818BF0120CB
:103CA00015B05DF804FB0120FAE700BF88D20120BF
:103CB0002DE9F0418AB03A4B3A4D3B48002401943B
:103CC0009A6B42F002029A639A6B02F0020201922E
:103CD000019A9A6942F002029A619A6922F00202FC
:103CE0009A6102941A6B42F040021A631A6B02F056
:103CF00040020292029A03941A6B42F002021A6383
:103D00001A6B02F002020392039A04941A6B42F0B7
:103D100020021A631B6B03F020030493049B02230D
:103D2000069301230A274FF04008079305A90323B0
:103D30000926CDF814800893099700F059FE042352
:103D400005A91A4805930794099600F051FE4FF40F
:103D5000807305A928460593099700F049FE4FF4A2
:103D6000007305A928460593099700F041FE8023BA
:103D700005A928460593099600F03AFE05A92846AC
:103D8000CDF81480099600F033FE22460F215C2006
:103D900000F0D6FB5C2000F005FC0AB0BDE8F08125
:103DA00000380240001402400018024000040240A3
:103DB00070B5494C494B236090B0204602F035FB6A
:103DC000054610B1012010B070BD01462046FFF736
:103DD0006FFF0423A36010236560E3604FF08076DB
:103DE00096FAA6F3B3FA83F3013B236120464FF41E
:103DF00080636361A561E561256202F0C3FA002872
:103E0000E0D1CDE90A00CDE90E004FF480756623BC
:103E1000099007900D9041F2883202A9204608953A
:103E2000029302F015FB08B10420CCE7992341F27C
:103E3000883202A92046029302F00AFB0028F3D13F
:103E400041F28830FFF7D2FE0028EDD1852302939E
:103E50000123CDE90A06CDE90C30CDE90E00099029
:103E6000079041F2883202A92046089502F0F0FA44
:103E70000028D9D141F288320DF10701204602F025
:103E80001EFC0028D0D1FFF7DBFE0028CCD1812317
:103E90000293F02292FAA2F29DF807300A21B2FAB8
:103EA00082F201FA02F203F00F03134302A941F276
:103EB000883220468DF8073002F0CAFA0028B3D1C4
:103EC00041F288320DF10701204602F099FB0028EB
:103ED0003FF479AFA8E700BF88D20120001000A00E
:103EE00070B5114C114E23683078154698476368B9
:103EF00070209847CD2814D18DB1022D0CBF082316
:103F00000C230B4A0B4D13707020A36830702C608B
:103F100098472B683078DB689847002070BD0623EF
:103F2000EFE70320FAE700BF94000020E4D201206D
:103F300090000020E8D201202DE9F04FDFF8D8B042
:103F4000DFF8D8A0DBF8003005461B699AF80000BE
:103F500085B09847287048B12C4E2D4FA94603AA2A
:103F600002AC4FF000082B78434503D8002005B081
:103F7000BDE8F08FDBF800309AF800005B69009232
:103F800021469847234B009A1B78019613F0080F9F
:103F90001FBF2188108820801180990742BF218887
:103FA000C1F1EF0121805B0748BF1388316834F805
:103FB00002CB44BFC3F1EF0313808BB28C458CBF9F
:103FC000ACEB0303A3EB0C039BB232F8020B0093A0
:103FD0003B6899B298428CBF411A091A009B89B27A
:103FE0000B44052B019BC8BFC6F800C01B68C8BFA7
:103FF0003860BE4629F8023FDEF80030A9F80430E8
:104000000436043708F10108ADE700BFDCD2012017
:10401000D4D2012090000020E8D20120E4D2012077
:104020007FB5002300930C4B0C481A6B42F0400202
:104030001A631B6B03F040030093009B2023019342
:10404000012303930223049301A9054B029300F07B
:10405000CFFC07B05DF804FB0038024000180240B6
:104060000000211008B5FFF7DBFF0F210022172009
:1040700000F066FA172000F095FA044B044A1B681A
:1040800010789B699847002008BD00BFE8D2012046
:10409000E4D2012070470020704710B50446FFF7B6
:1040A00027FBA821E0B2FFF737FB10BD13B50024B2
:1040B0000221C0B28DF80740FFF72EFB8DF80700F4
:1040C0009DF8073003F00F038DF807309DF8073097
:1040D000022B88BF8DF80740044B9DF807209DF800
:1040E00007005A7000229A7002B010BDECD2012075
:1040F00073B5154C1546A37862789A420E461FD9BF
:1041000003B3012B0CBF0921002104230DEB030293
:10411000C0B2FFF717FB9DF804309DF805201B0285
:1041200003F47063134333809DF806309DF8072035
:104130001B0203F4706313432B80A3780133A37035
:1041400002B070BD0321E0E7ECD201200122A421DE
:10415000C0B2FFF7CFBA0022A421C0B2FFF7CABA9B
:10416000FFF7F9BF70470000064A1378834208D072
:104170005178884205D00BB119B90123D054FFF70B
:10418000B7BA7047EFD20120012A82B009D10A4B99
:104190001B688B400093009B02681343036002B0CE
:1041A0007047064B1B6803FA01F1C9430191019B5B
:1041B00002681340F2E700BFC0000020BC000020EE
:1041C00008B5024600210248FFF7DEFF08BD00BF28
:1041D00010E000E008B50A4601460248FFF7D4FFA8
:1041E00008BD00BF24ED00E082B04AB1094B1B6856
:1041F0008B400093009B02681343036002B070473A
:10420000054B1B6803FA01F1C9430191019B026848
:104210001340F2E7C0000020BC00002038B5064D76
:1042200002460C4628460421FFF7DEFF2246032102
:104230002846FFF7D9FF38BD14ED00E010B5012185
:1042400004461120FFF7C6FF01211220FFF7C2FF2D
:1042500000210120FFF7E2FF204610BDF0B5C6683F
:10426000054600202C69AB68A64228BFE4189B1BBA
:10427000934204F1FF3428BF1346A41BA34228BF76
:1042800023466C68F718013E1844D21A26440B44A2
:104290008B4208D1AB68BB4214BF3E460026EE609D
:1042A000002ADFD1F0BD11F8014B06F8014FEFE70E
:1042B000F0B5C468876843683D1B234495421444A5
:1042C00003F1FF330ED80D440E46AE4214D14368BD
:1042D000E41B013B11448D4207D015F8012B03F874
:1042E000012FF8E70A44914201D1C460F0BD11F8F2
:1042F000015B03F8015FF6E716F801CB03F801CF85
:10430000E3E70369C26893429CBF81685B18013B85
:10431000981A704710B5114C114AA261032323610A
:104320006361104BE36122664FF480630E4A0F49CC
:104330002362626600231022E01DA3626362E362CF
:104340002367E3666367A26613F034FB08492046DF
:1043500013F030FB2023A37110BD00BF04D7012050
:104360001CBB010801D30120F1D2012025BB0108AB
:1043700029BB0108F8B5144B182700FB07751D442D
:1043800007FB00330E46DB6A012B14460AD0022BD2
:1043900014D023B92846FFF7B4FF844208D900247B
:1043A0002046F8BD2846FFF7ACFF844228BF0446EC
:1043B000224631462846FFF77BFFF1E72846BDE855
:1043C000F840FFF74BBF00BF04D70120F8B50B4BF7
:1043D0001B7804460D4616460BB9FFF79BFFEFF31B
:1043E00011874FF0200181F311883246294620467B
:1043F000FFF7C0FF87F31188F8BD00BF04D7012085
:1044000038B5054608460C4613F040FB21460246E7
:104410002846BDE83840FFF7D9BF00002DE9F0413C
:10442000164C1E4623780546884617460BB9FFF7FB
:1044300071FF2369AB421DD9EFF3118C4FF02001BE
:1044400081F3118865B1182005FB0003E21844F8D8
:104450000380576000FB054200231662936253629B
:10446000182303FB0544069BE3628CF311880020AC
:10447000BDE8F0814FF0FF30FAE700BF04D701201C
:10448000FFF748BFFEE7000038B50E4B1A784FF42F
:104490007A73B3FBF2F30C4A05461068B0FBF3F0F5
:1044A00000F09CF8044658B90F2D09D80246294659
:1044B0004FF0FF3000F044F8044B20461D6038BD3B
:1044C0000120FCE7C4000020CC000020C800002030
:1044D000034A044B11681B780B441360704700BFFC
:1044E000ACD70120C4000020014B1868704700BF02
:1044F000ACD7012038B50446FFF7F6FF631C1CBF9C
:10450000054B1B78054618BFE418FFF7EDFF431B6A
:10451000A342FAD338BD00BFC40000200749CA68CF
:1045200022F4E0620302120403F4E063120C13436A
:1045300043F0BF6343F40033CB60704700ED00E00D
:10454000164B30B5DC68C4F30224C4F10703251D03
:10455000042B28BF0423062D4FF0FF358CBF033CEE
:10456000002405FA03F321EA0303A54022EA050229
:10457000A340002843EA0203ACBF00F16040084AB0
:104580004FEA0313B8BF00F00F00DBB2AABF00F57B
:104590006140135480F8003330BD00BF00ED00E0EF
:1045A00014ED00E0002807DD4109044A00F01F0077
:1045B0000123834042F82130704700BF00E100E052
:1045C000002808DD4309044900F01F0001222033C0
:1045D000824041F82320704700E100E00138B0F14B
:1045E000807F0BD24FF0E023054A5861F02182F81A
:1045F00023100020072298611A617047012070473C
:1046000000ED00E04FF0E02304281A690CBF42F0EF
:10461000040222F004021A6170470000036810B51A
:10462000084C0246D9B210391820B1FBF0F0205CDA
:10463000D06523F47F7020F003005F2988BF043029
:10464000906510BD30BB010838B50446FFF74CFF3C
:104650000546002C72D00023226884F834300223EF
:1046600084F83530136823F00103136021680B6868
:10467000D80728D40B68354AA568A0691A40636832
:104680002B43E5682B4325692B4365692B43E5697B
:1046900003432B43256A2B431343626A042A1DD02C
:1046A0000B604B6923F0070313434B612046FFF770
:1046B000B5FFE26D3F2393408360002001236065D6
:1046C00084F8353009E0FFF70FFF401B0528CDD9EE
:1046D00020230320636584F8350038BDE26A256B2A
:1046E00015431D430D604B69A56A23F007032B4357
:1046F00043F00403002AD8D038B9012D16D035F084
:104700000200D2D1D201D0D513E0B0F5005F17D1AD
:10471000032DCAD801A050F825F000BF3347000888
:1047200005470008334700082D470008B2F1C07F55
:10473000BBD140236365012384F835300120CCE7E9
:10474000022DF6D9032DDDD0AFE700BF3F8010F07A
:1047500070B590F83440866D012C30D0012480F87B
:10476000344090F83540012C4FF0000425D102254B
:1047700080F8355044650468256825F48025256057
:1047800063608368402B0EBFA260A160E260C26DCF
:1047900008BFE1603F239340B360236843F01603F2
:1047A0002360036C1BB1236843F008032360236874
:1047B00043F001032360002070BD80F834400220E4
:1047C000FAE770B50446866DFFF78EFE94F8353033
:1047D000022B054606D080236365002384F834301D
:1047E000012070BD23681A6822F016021A605A6907
:1047F00022F080025A61226C0AB9A26C1AB11A68BE
:1048000022F008021A601A6822F001021A60236876
:10481000186810F0010009D1E26D3F239340B360A6
:10482000012384F8340084F83530DAE7FFF75CFEC2
:10483000401B0528EBD9202363650320002384F85F
:10484000343084F83500CCE790F83530022B03D0B3
:1048500080234365012070470268052380F83530C6
:10486000136823F00103136000207047F7B500239D
:1048700001935C4B856D1F68C36D2E6808229A40BA
:10488000324204460CD001680868400708D5086821
:1048900020F004000860AA60626D42F001026265C7
:1048A00001229A40324208D021684969090641BF75
:1048B000AA60626D42F00202626504229A403242AE
:1048C00008D021680968880741BFAA60626D42F07C
:1048D0000402626510229A40324210D0236819689F
:1048E00009070CD5AA601A68500337D51B6819034D
:1048F00001D4236C00E0A36C0BB120469847E16D16
:1049000020228A4032423AD023681868C60636D53B
:10491000AA6094F83520052A1A6827D122F01602D9
:104920001A605A6922F080025A61226C0AB9A26C9C
:104930001AB11A6822F008021A603F238B40AB605C
:10494000002384F83430012384F83530236D002BA4
:1049500045D0204603B0BDE8F04018471A68D2059C
:104960005EBF1A6822F008021A60C2E7500327D51A
:104970001B68190331D4636C0BB120469847636DF3
:104980006BB3636DDA0719D522684FF41653B7FB82
:10499000F3F7052384F83530136823F0010313601F
:1049A000019B0133BB42019302D81368DB07F7D4A4
:1049B000002384F83430012384F83530E36CC6E7F3
:1049C0001A6812F4807208D1196821F01001196078
:1049D000012384F8342084F83530E36BCCE703B04E
:1049E000F0BD00BFCC00002090F8350070470000FB
:1049F0002DE9F04FDFF8C0E16D4E85B000240123B2
:104A000003FA04F80B6808EA030938EA030323D120
:104A10004A68032322F0100A4FEA440C03FA0CF709
:104A20000AF1FF33012B8B6801936FEA070702F04D
:104A3000030317D9D0F80C80019D07EA080805FA8E
:104A40000CF545EA0805C560056803FA0CF33D401E
:104A50002B430360D3003FD40134102CCFD105B0D9
:104A6000BDE8F08FD0F80890CD6809EA070905FA8B
:104A70000CFB4BEA090BC0F808B0D0F80490019D7C
:104A8000120929EA0809A24042EA09024260C26802
:104A900005FA0CF53A401543BAF1020FC56006D08D
:104AA000026803FA0CF33A4013430360D4E7E508C5
:104AB00000EB850504F007082A6A4FEA88084FF0E2
:104AC0000F0909FA08F922EA09090A6902FA08F243
:104AD00042EA09022A62E3E74FF0000ACDF80CA08F
:104AE000DEF8445045F48045CEF84450DEF844509A
:104AF00005F480450395039D24F0030505F18045E9
:104B000004F003070F2305F59C35BF0003FA07FCEB
:104B1000284BD5F80880984228EA0C0C3CD003F5C5
:104B2000806398423AD003F58063984238D003F509
:104B30008063984236D003F58063984234D003F501
:104B40008063984232D003F58063984214BF0723F4
:104B50000623BB4043EA0C03AB6033686FEA0905E8
:104B6000D70354BF2B4049EA0303336073689703AC
:104B700054BF2B4049EA03037360B368D70254BFA4
:104B80002B4049EA0303B360F368920254BF2B4001
:104B900049EA0303F3605FE75346DAE70123D8E706
:104BA0000223D6E70323D4E70423D2E70523D0E783
:104BB000003C0140000002400038024003691942F5
:104BC00014BF0120002070470AB1816170470904B9
:104BD000FBE7436931EA030308BF090481617047B9
:104BE000044A5169014208B502D05061FEF752F9FA
:104BF00008BD00BF003C014001684B6913F48063AD
:104C00004FF0000210D06FF480634B6120230263E9
:104C100080F83D3080F83E20036C80F83C2043F063
:104C20000403036401207047184670472DE9F846D5
:104C300006460F4691461D464FEA114A3368BAF1BF
:104C4000010F0CBF5C699C6927EA0404A4B2B4FAA2
:104C500084F46409A14501D0002017E06A1CEED05D
:104C6000FFF742FC089BC01AA84201D8002DE5D1ED
:104C700000232022336386F83D2086F83E30326CD4
:104C800086F83C3042F0200232640120BDE8F8860C
:104C90002DE9F04104460F46164698462568686996
:104CA00027EA000080B2C0B16B695A0517D52B689E
:104CB00043F400732B606FF480636B612022002348
:104CC000236384F83D2084F83E30236C43F00403D2
:104CD0002364002384F83C300120BDE8F081731C7C
:104CE000DDD0FFF701FCA0EB0800B04201D8002E98
:104CF000D4D100232022236384F83D2084F83E3061
:104D0000236C1343E4E770B504460D46164623684A
:104D10005B691B0601D500201AE02046FFF76CFFF7
:104D2000A8B96A1CF3D0FFF7DFFB801BA84201D8AB
:104D3000002DECD100232022236384F83D2084F849
:104D40003E30226C84F83C3042F020022264012084
:104D500070BD00002DE9F0431546026885B0DDE91D
:104D60000C789946136843F4807313600E463B46F3
:104D7000CDF8008000224FF001110446FFF756FFE6
:104D8000236838B11B68DB0502D54FF40073236438
:104D9000032620E006F0FE061E611A4943463A4605
:104DA0002046FFF775FFA8B9236803905A6903925C
:104DB0009B690393424639462046039BFFF7A3FFB6
:104DC000064660B1236C042B01BF2268136843F4CC
:104DD000007313600126304605B0BDE8F083B9F1D9
:104DE000010F236802D1EDB21D61F4E72A0A1A61AE
:104DF000394642462046FFF786FF0028E2D1236865
:104E0000F1E700BF020001002DE9FF479A46036861
:104E100015461A6842F480621A601A68DDE90C7857
:104E200042F480721A600E463B46CDF800800022A4
:104E30004FF001110446FFF7F9FE236838B11B68F3
:104E4000DB0544BF4FF400732364032021E05FFAC5
:104E500086F906F0FE061E612B4943463A46204677
:104E6000FFF716FFA0B9236803905A6903929B6964
:104E70000393424639462046039BFFF744FF58B14F
:104E8000236C042B01BF2268136843F40073136082
:104E9000012004B0BDE8F087BAF1010F23681AD1F0
:104EA000EDB242461D6139462046FFF72CFF02460F
:104EB0000028E5D121680B6843F480730B6020461D
:104EC000CDF800803B464FF00111FFF7AFFE22689E
:104ED00060B11368B4E72A0A1A613946424620468F
:104EE000FFF711FF0028CBD12368D9E749F0010370
:104EF0001361054943463A462046FFF7C9FE00388C
:104F000018BF0120C5E700BF0200010070B50446CC
:104F10000D46164623685B695B0701D500201AE041
:104F20002046FFF769FEA8B96A1CF3D0FFF7DCFA48
:104F3000801BA84201D8002DECD10023202223633E
:104F400084F83D2084F83E30226C84F83C3042F0F6
:104F500020022264012070BD70B504460D4616463D
:104F600021684B6913F0400301D0002011E04A6929
:104F7000D2060FD56FF010024A612022236384F815
:104F80003D2084F83E30236C2364002384F83C30B9
:104F9000012070BDFFF7A8FA801BA84201D8002DA0
:104FA000DED100232022236384F83D2084F83E30A4
:104FB000236C1343E8E7704770B5044608B9012035
:104FC00070BD90F83D3003F0FF021BB980F83C2023
:104FD000FFF7F1FF242384F83D3023681A6822F09C
:104FE00001021A601A6842F400421A601A6822F438
:104FF00000421A6001F0E6FC3E4B65689D4294BF9A
:105000003D4B3E4B9842DAD921683D4A4B68B0FB94
:10501000F2F223F03F0313434B60431E35480E6A00
:10502000854226F03F0639D8013232430A62C86908
:105030006A00B3FBF2F2531C40F6FC7220F44F40BE
:10504000134220F0FF0045D104230343CB610A68DB
:10505000206AE36922F0C002034313430B608A68AD
:10506000E068236922F40342034322F0FF02134362
:105070008B60CA68A069636922F0FF02034313438F
:10508000CB600B6843F001030B60002020232064F9
:1050900084F83D30206384F83E0091E74FF4967029
:1050A00042434FF47A70B2FBF0F2013232430A62AB
:1050B000C869A26820F44F4020F0FF006AB11922AD
:1050C0006A43B3FBF2F30133C3F30B036BB143F455
:1050D0004043BAE7C3F30B03B7E705EB4502B3FB65
:1050E000F2F20132C2F30B030BB90123ADE743F433
:1050F0000043AAE7A08601007F841E00FF083D0050
:1051000040420F00704710B5044698B1026824234E
:1051100080F83D30136823F001031360FFF7F2FFBE
:105120000020206484F83C0084F83D00206384F86B
:105130003E0010BD0120FCE72DE9F74304469946E7
:105140000C9E0F469046FFF7CFF994F83D30202B88
:10515000054603D0022003B0BDE8F08300903C492F
:10516000192301222046FFF761FD0028F2D194F8AF
:105170003C30012BEED02068012384F83C300368DA
:10518000D9075EBF036843F001030360036823F49B
:1051900000630360212384F83D30402384F83E30CF
:1051A000002323640A9B6362BDF82C306385638D02
:1051B0002385284BE3624246019500964B463946CB
:1051C0002046FFF7C7FD00282AD00120C3E7FFF7DC
:1051D0009AFD40B1236C042B01BF2268136843F48D
:1051E00000731360F1E7636A27681A4612F8011B1F
:1051F00039616262628D218D013A92B262857A696B
:10520000481E80B2520720850AD548B15A783A61C3
:1052100002336362638D013B02399BB22185638552
:10522000238D2A4631462046002BD0D1FFF76EFE53
:105230000028CFD12268136843F400731360202341
:1052400084F83D3084F83C0084F83E0083E700BFDA
:10525000020010000000FFFF2DE9F043044687B074
:105260009946109F0D469046FFF73EF994F83D3061
:10527000202B064604D00225284607B0BDE8F0835F
:1052800000907649192301222046FFF7CFFC002821
:10529000F1D194F83C30012BEDD02068012384F843
:1052A0003C300368DB075EBF036843F00103036023
:1052B000036823F400630360222384F83D30402315
:1052C00084F83E30002323640E9B6362BDF83C30BB
:1052D0006385638D2385624BE362294601960097BF
:1052E0004B4642462046FFF78FFD054608B1012593
:1052F000C2E7228D2368B2B902905A6902929A6974
:105300000292029A1A6842F400721A60DFF854811D
:10531000238D002B2CD1202284F83D2084F83C30B2
:1053200084F83E30A8E7012A0AD11A6822F4806284
:105330001A6003905A6903929A690392039AE1E70B
:10534000022A0ED11A6822F480621A601A6842F4A6
:1053500000621A6004905A6904929B690493049B4A
:10536000D4E705905A6905929B690593059BCDE7A3
:10537000032B56D8012B15D1324639462046FFF76C
:10538000EBFD0028B3D123681A69636A1A70636A57
:1053900001336362238D013B2385638D013B9BB207
:1053A0006385B5E7022B00963B464FF0000241466D
:1053B000204619D1FFF73AFC002898D123681A68D3
:1053C00042F400721A601A69636A1A70626A531CA6
:1053D0006362238D013B2385638D013B9BB2638513
:1053E00023681B695370D2E7FFF720FC02460028B0
:1053F0007FF47DAF2368196821F480611960196911
:10540000636A1970636A01336362238D013B2385EC
:10541000638D013B9BB26385414600963B46204627
:10542000C8E7324639462046FFF796FD00287FF44C
:105430005EAF23681A69636A1A70626A531C6362FA
:10544000238D013B2385638D013B9BB263852368DC
:10545000596949077FF55CAFC3E700BF0200100040
:105460000000FFFF0400010070477047704770475D
:1054700070477047704790F83D10026D10B50346B5
:10548000C9B282B9C26C0168012A826C05D1D2B25C
:105490000A61026D02321A6510BDC2F307220A6169
:1054A0001A6D0132F7E7026D012A03D1826C01689F
:1054B000D2B2F4E7026D022AEED1222905D10268A8
:1054C000136843F480731360E6E7428D92B272B1C1
:1054D00021290AD1426A016812F8010B08615A6257
:1054E0005A8D013A92B25A85D6E75B8DD4E7428D48
:1054F00092B2002AD0D12129CED101684C6824F47F
:10550000E0644C600C6844F400740C602021026379
:1055100080F83D1080F83E20FFF7ACFFBCE77047F5
:105520007047704773B50023806B019390F83D205E
:10553000344BD4B21B6846F2A812B3FBF2F3232219
:10554000534301930368019A02BB026C42F02002AC
:105550000264416B826B01BB002A32D1196821F4CD
:105560008061196042851A6822F001021A6090F881
:105570003D20602A2CD1202380F83D30002380F884
:105580003E300364FFF7CDFF02B070BD019A013ACF
:1055900001921A689205D6D4DBE70025CD6332B9B3
:1055A0001D6825F480651D6042850A65DBE71E687D
:1055B000D56326F480661E6045850D650021116562
:1055C000D1E71D68D16325F480651D604185F5E74D
:1055D00004F02802282A0ED1196841F0010119604F
:1055E000196841F4806119600023036380F83D204D
:1055F000FFF796FFC8E7202380F83D30002380F8AE
:105600003E30F5E7CC00002090F83D2090F83E3089
:10561000102B10B5D9B204460368D2B201D040298C
:105620000CD1222A0AD11A6822F400621A60226878
:105630005268120549D50022226307E002F02801D2
:1056400028293DD10022226384F83D105A6812F4C3
:1056500000625BD05A68606B22F400625A6090F876
:105660003530012B3D4B37D00365FFF7EDF850B1D6
:105670002268606B136823F001031360202384F811
:105680003D30036D9847236C19071FBF226853688C
:1056900023F4E063536094F83D30226C5207DBB290
:1056A0000DD5282B0BD12E4BE36220220023236340
:1056B000204684F83D2084F83E30FFF7DAFE10BD26
:1056C00059680805B7D4602AB5D0202284F83D2057
:1056D000002284F83E20AEE7A06B0365FFF7B4F824
:1056E0000028D0D023685A69510605D51A69636A23
:1056F0001A70636A013363622268A06B136823F037
:1057000001031360202384F83D30BAE794F83D107C
:10571000602915D1202184F83D1022645A6952066F
:1057200005D51A69636A1A70636A01336362226875
:10573000136823F0010313602046FFF7F2FEA2E78F
:105740005A69500605D51A69636A1A70636A01338B
:1057500063622046FFF7E4FE95E700BF2555000889
:105760000000FFFF70B503685A68C66A90F83E10E3
:10577000044690F83D0010298CB0CDB2C0B202D0E2
:10578000402D40F0EC829869596911F0010F07D162
:10579000B6F52A0F02D0B6F12A4F52D10CB070BD27
:1057A00096054ED5E26AB2F52A0F0CD10122E262CB
:1057B00094F83E20402A11D1226D52B9626C02F059
:1057C000FE021A61EAE7E26AB2F12A4FF0D108223A
:1057D000EDE7626C42F00102D2B2F2E72269B2F563
:1057E000804F19D194F83D20212A626C16BF42F0F7
:1057F000010202F0FE02D2B21A61626B0AB1D26BF0
:105800002AB9A26B002AC9D0D26B002AC6D05A6826
:1058100042F400625A60C1E7226D3AB9626CC2F389
:10582000C81202F0060242F0F002CAE7226D012A15
:10583000B4D1626CC2F3C81202F0060242F0F10267
:10584000BFE70E070ED596050CD5626CD2B21A6171
:10585000626B12B9A16B0029A0D0D26B002AD6D1FD
:10586000A26BD1E78E0740F1ED80960540F1EA800A
:1058700094F83E10E26A256B94F83D002228C9B2E4
:1058800040F0D880206D40B9402906D100905A6977
:1058900000929B690093009B80E7216D19B92069F4
:1058A000B0F5404F1FD0618D89B2002929D0618D9C
:1058B00089B2012962D112F5803F34D11A6822F4ED
:1058C00080621A605A6812F4006225D01A6822F4C5
:1058D00080621A60002203925A6903929B690393C3
:1058E000039B00230BE001915A6901929A6901928E
:1058F000019A1A6842F480721A60236D013323659D
:105900004CE702915A6902929A690292029A1A68C5
:1059100042F400721A60E4E704925A6904929A69A8
:105920000492049AF3E7082A1CD0202A1AD0122DD8
:105930000DD1012A16D11A6822F480621A60002261
:1059400005925A6905929B690593059BC9E7102A40
:10595000F1D88B4941FA02F2D607ECD41A6842F426
:105960008062EBE71A6822F480621A6000220692D5
:105970005A6906929A690692069AC8E7618D89B2B9
:10598000022934D1102A03D87E49D140CD0712D440
:10599000196821F480611960196841F40061196087
:1059A0005968080513D4002207925A6907929B6927
:1059B0000793079B95E7196841F48061196059685E
:1059C0000905F0D5072A07D8012AECD10AE0202AD8
:1059D000F8D912F5803FF8E7A2F108016A4ACA40F7
:1059E000D207E0D55A6842F480525A60DBE7196862
:1059F00041F48061196059680E0505D5202A16D832
:105A0000072A09D8012A0DD0002208925A69089263
:105A10009B690893089B64E7A2F108015A4ACA40AF
:105A2000D507F1D55A6842F480525A60ECE712F576
:105A3000803FE8E7002209925A6909929B6909931D
:105A4000099BABE610F0040F586800F09F8000053A
:105A50003FF5A4AE0E06C1F3800055D5510553D5D0
:105A6000002854D194F83D20258D94F83E10E06A2A
:105A7000D2B2C9B27DBB212A2FD1082814D0202848
:105A800012D010F5803F0FD05A6822F4E0625A60BD
:105A900011232363002384F83E30202384F83D3013
:105AA0002046FFF7E1FC79E65A6822F4E0625A608A
:105AB0001A6842F400721A6000232022236384F8DB
:105AC0003D2094F83E2084F83E30402A2046E8D11C
:105AD000FFF7D0FC62E6212A05D040297FF45EAEB4
:105AE000222A7FF45BAE628D92B21AB95A6822F410
:105AF00080628FE694F83E20402A16D120460CB0F2
:105B0000BDE87040FFF7B7BC00283FF447AE9205F0
:105B10007FF544AE102DF1D1E16A94F83D20212AA1
:105B20007FF43CAE628D92B24AB1626A12F8011BF8
:105B300019616262638D013B9BB263852EE6082981
:105B40000DD020290BD011F5803F08D0596821F4E1
:105B5000E06159601123236384F83E209DE75A6871
:105B600022F4E0625A601A6842F400721A6000235C
:105B70002022236384F83D2084F83E3090E700BF64
:105B8000EBFFFEFF140001000101000106053FF5D7
:105B900005AE4D06C1F3800076D5510574D50028B9
:105BA00075D194F83D20222A7FF4F8AD628D92B22F
:105BB000032A14D91A69636A1A70636A013363622B
:105BC000638D013B9BB26385638D9BB2032B7FF496
:105BD000E5AD2268536823F480635360DEE5E16A33
:105BE00002293FF4DBAD012A3FF6D8AD734A0A9093
:105BF000126846F2A811B2FBF1F202EB82020A929D
:105C00000A9A013A0A920A99D1B9226C42F020020A
:105C100022645A6822F4E0625A601A69636A1A7050
:105C2000636A01336362638D013B9BB2638520230A
:105C300084F83D30204684F83E10FFF771FCADE556
:105C40001A6812F40072DBD1196821F480611960BE
:105C5000596821F4E06159601969636A1970636ACF
:105C600001336362638D013B9BB26385202384F81B
:105C70003D3094F83E3084F83E20402B69D12263B9
:105C80002046FFF74CFC89E500283FF487AD9205DC
:105C90007FF584ADE26A608D616A80B2042809D123
:105CA0005A6822F480625A601B690B70636A013380
:105CB00063623FE7608D80B203280CD15868042AE4
:105CC00020F480605860EFD0022AEDD01A6822F4E8
:105CD00080621A60E8E7608D80B20228E4D1042A6D
:105CE00033D007D8012A07D0022A2ED01A6842F4EE
:105CF000007204E0102AF9D11A6822F480621A6056
:105D00001B690B70626A531C6362638D013B9BB21B
:105D1000638523681B695370636A22680133636279
:105D2000638D013B9BB26385536823F440735360DA
:105D3000202384F83D3094F83E30402B4FF0000390
:105D400084F83E3005D123639AE71A6842F48062F2
:105D5000D5E7122323632046FFF787FB1EE5216C5E
:105D600011B3596900258E072AD5960528D5226CCE
:105D700002B19D6994F83D2002F02802282A16D12C
:105D80005A6822F480625A606FEA95012B064FF040
:105D9000000354BFA289228B84F83C3001F001013A
:105DA0002046FFF765FBF9E49D695969DBE76FF071
:105DB00002025A61002384F83C30EFE4CC0000205A
:105DC000CE0640F1C280950540F1BF8094F83D5069
:105DD0005A6822F4E0625A6000220B925A690B92D0
:105DE0001A6842F001021A600B9A1A6822F4806263
:105DF0001A605A681205EDB220D505F0F702222A82
:105E00003DD1A06B0268526892B26285628D92B2F7
:105E10001AB1226C42F0040222645A6822F4006231
:105E20005A60FEF7E1FD012808D0A06B824B0365A4
:105E3000FEF70AFD10B1A06B036D9847638D9BB20E
:105E4000002B3CD1236C002B56D12A2D74D1236317
:105E5000282384F83D302046FFF709FB94F83D30B5
:105E6000282B5AD1754BE36220220023236320465E
:105E700084F83D2084F83E30FFF7FBFA8EE4606B37
:105E80000268526892B26285628D92B21AB1226C37
:105E900042F0040222645A6822F400625A60FEF75B
:105EA000A3FD012808D0606B634B0365FEF7CCFCB3
:105EB00010B1606B036D9847638D9BB2D3B12368BB
:105EC0005A6956071ED423685A69500609D51A69BB
:105ED000636A1A70636A01336362638D013B9BB22C
:105EE0006385638D9BB2002BACD0236C43F004031D
:105EF0002364A7E7236CFBB120460CB0BDE87040DB
:105F0000FFF782BB1A69636A1A70636A01336362BE
:105F1000638D013B9BB26385D5E7236B222B7FF416
:105F20003DAC00232022236384F83D2084F83E30DA
:105F30002046FFF79CFA31E494F83D30282B91D0AD
:105F4000236B222BEDD0222DE9E700F0F70021286A
:105F5000C1F3800536D1090628D5560526D545BB9F
:105F600094F83D10628D92B2C9B2002A3FF416AC8B
:105F7000626A12F8015B1D616262628D013A92B23F
:105F80006285628D92B2002A7FF408AC29297FF4E1
:105F900005AC5A6822F480625A602823206384F892
:105FA0003D302046FFF762FAFFF7F8BB002D3FF4C3
:105FB000F5AB95057FF5F2AB628D92B2002A3FF406
:105FC000EDABB2E5480627D5510525D53DBB94F884
:105FD0003D20618D89B2D2B200293FF4DFAB19694F
:105FE000636A1970636A01336362638D013B9BB21C
:105FF0006385638D9BB2002B7FF4D0AB2A2A7FF49C
:10600000CDAB2268536823F480635360222323635B
:10601000282384F83D308BE7002D3FF4BFAB920579
:106020007FF5BCAB628D92B2002A3FF4B7AB1A6920
:10603000636A1A703AE600BF255500080000FFFFAA
:10604000F8B50368044658695A6894F83E10C705C5
:10605000C9B2C0F3002507D5D60548BF6FF48076D6
:10606000C2F3002548BF5E61870506D5D60542BF4D
:106070006FF4007645F002055E61C0F3C02640056E
:1060800073D5D20544D5678D94F83D00D4F830C05F
:106090002029BFB2C0B26FF480625AD167B15A6191
:1060A00045F00405002E64D1236C2B432364204665
:1060B000BDE8F840FFF7A8BA00F0F701212904D0A5
:1060C0002828ECD1BCF1210FE9D194F83D20E16AF8
:1060D0000829D2B201D020291DD1282A1BD1284A53
:1060E000E2625A6822F4E0625A606FF480625A6198
:1060F0001A6822F480621A6000232022236320465B
:1061000084F83D2084F83E30FFF7B3F9002E30D1FB
:10611000002DC9D1F8BD212A17D11949E1622263A6
:10612000202284F83D20002284F83E205A6822F480
:10613000E0625A606FF480625A611A6822F48062E9
:106140001A602046FFF792F9E0E76FF480625A6127
:10615000DCE710295A6145F0040501D04029A1D19E
:106160001A6842F400721A609CE7002ED0D0D30562
:10617000CED523686FF4006245F008055A6193E7B5
:106180000000FFFF90F83D00704700000B4A1368C5
:1061900023F0030303431360094B1A69012942F0FA
:1061A00004021A6105D130BF1A6922F004021A6193
:1061B000704740BF20BF20BFF6E700BF007000401F
:1061C00000ED00E02DE9F0474E6A3EB1B2F1406FBC
:1061D0001FBF8B6A046803F1FF332361D1F818A055
:1061E000D1F820E0CF69BAF1000F4DD04C690568B5
:1061F0000B68C86AD1F83090D1F834804FEA844CEB
:106200004AEA060444EA020ABEF1000F24D08E686E
:10621000EE614AEA0E040E699FB13B43034343EA31
:106220000903C86843EA08033343034343EA0C0302
:106230002343B2F1406F6B6101D04B68AB61BDE8A5
:10624000F087034343EA090343EA0803334343EA7D
:106250000C0323436B61F2E767B13B43034343EA1B
:106260000903C86843EA0803034343EA0C0343EA0B
:106270000A03DEE7034343EA090343EA080444EA66
:106280000C0343EA0A03E5E7BEF1000F2BD046EA10
:106290000E0504684E698B68E361D1F82C800B69A8
:1062A000D1F830E0D1F834C01543B6048FB13B4388
:1062B00043EA0803C86843EA0E0343EA0C030343B6
:1062C00033432B43B2F1406F6361B8D04B68A36195
:1062D000B5E743EA080343EA0E0343EA0C033343FA
:1062E0002B436361ABE7AFB1CC6A006846EA0703B2
:1062F000134323430C6B23434C6B2343CC6823434E
:106300004C69B2F1406F43EA8443436197D04B68D4
:10631000836194E7002E92D0CB6A00683343134325
:106320000A6B13434A6B13434A6943EA824343614E
:1063300085E72DE9F041DDF8188004460E46154644
:106340001F4622689368334214BF01230023AB42E7
:1063500001D1002012E0B8F1FF3FF3D0FEF7C4F8FE
:10636000C01B404502D8B8F1000FEAD1042384F8DD
:106370004130636C43F0010363640120BDE8F081A8
:106380007047000037B50446FEF7AEF80546002C0E
:1063900046D094F8413003F0FF023BB984F8402026
:1063A0002046FFF7EDFF41F28833A3642168A3681C
:1063B0000A68013B22F4F85242EA0322A36C0A6005
:1063C0002046009300222B462021FFF7B2FF10BB8E
:1063D000E569E36822682B43256A11682B436568E9
:1063E00021F07F4143EA056321F0D0010B431360A4
:1063F000A169636955680B43216943EA014309496F
:1064000029400B435360136843F0010313600123D9
:10641000606484F84130002384F8403003B030BD1C
:106420000120FBE7FEF8E0FF704710B5044668B1B5
:106430000268136823F001031360FFF7F5FF0020E3
:10644000606484F8410084F8400010BD0120FCE73E
:106450002DE9F34704468A469046FEF745F894F83E
:106460004030012B074637D0012384F8403094F8A0
:106470004130012B5FFA83F94FF0020628D1002248
:106480006264034684F841602021CDF800802046F4
:10649000FFF74FFF0546A0B9024651462046FFF7D9
:1064A00091FEDAF8243053B9CDF800803B464A46D5
:1064B00031462046FFF73DFF60B92368DE6084F86F
:1064C0004190002384F84030284602B0BDE8F087B0
:1064D0003546F6E70546F4E70225F5E72DE9F743EB
:1064E00004461F4689461546FDF7FEFF94F84030E6
:1064F000012B064641D0012384F8403094F8413006
:10650000012B5FFA83F836D14223002262642021F6
:1065100084F84130034600972046FFF70AFF20BB6E
:1065200022682B6893626B685362AB68D36213680E
:10653000296923F440030B4343F480031360EB68A1
:10654000C9F828304FF0006249462046FFF73AFE6E
:1065500000973346424608212046FFF7EAFE20B95D
:1065600023680822DA6084F84180002384F84030F0
:1065700003B0BDE8F0830220F7E70220F8E737B563
:106580000446FDF7B1FF94F841309907054634D52C
:10659000002384F8403023681A6852070BD51A6824
:1065A000E06B22F004021A60FEF70BF918B1636C7D
:1065B00043F0040363642268136843F0020313602A
:1065C000A36C009301222B4602212046FFF7B1FE67
:1065D000A0B923680222DA60A36C009302462B461E
:1065E00020212046FFF7A5FE40B92268536923F019
:1065F00040635361012384F84130002003B030BD73
:106600002DE9F341044688461746FDF76DFF94F8DF
:1066100040302568012B06464FD0012384F84030D6
:1066200094F84130012BD8B245D100236364B8F10E
:10663000000F3BD0122384F841302B690133E36211
:106640002B69C4F824800133A3626B6923F0406393
:106650006B61E36AB3B900973346012202212046F9
:10666000FFF767FE28B923680222DA602046FFF7A9
:1066700086FF012384F84130002384F8403002B0C3
:10668000BDE8F08100973346012204212046FFF740
:1066900050FE0028EDD1636A1B7885F82030636ACC
:1066A00001336362E36A013BE362D2E7636C43F068
:1066B00008036364E0E70220DEE70220DFE72DE95C
:1066C000F341044616468846FDF70EFF2568AA6981
:1066D00094F84030012B074652D0012384F8403013
:1066E00094F84130012BD8B248D100236364B8F14B
:1066F000000F3ED0222384F841302B690133A3637D
:106700002B69C4F8308001336363696921F040610B
:1067100041F080616961AA61A36BB3B900963B4601
:10672000012202212046FFF704FE28B92368022235
:10673000DA602046FFF723FF012384F8413000236D
:1067400084F8403002B0BDE8F08100963B4601225B
:1067500006212046FFF7EDFD0028EDD1236B95F8CB
:1067600020201A70236B01332363A36B013BA363C7
:10677000D2E7636C43F008036364E0E70220DEE7DE
:106780000220DFE770B5224C88B00E461546F8B9F6
:106790000190236B43F001032363236B059003F007
:1067A00001030193019B07904FF48073039302232D
:1067B000049303A9032317480693FEF719F9A36866
:1067C00023F0EC6343EA06012943A16008B070BDE1
:1067D00000230293226B104842F004022263226BD2
:1067E000059302F004020292029A07934FF400729A
:1067F00003920222049203A903220692FEF7F8F8FC
:10680000A36823F0784343EA060141EAC501DCE7C7
:10681000003802400000024000080240014B012203
:10682000DA64704700004742134908B58B6803F0EB
:106830000C03042B1CD0082B1CD14A684B684968F8
:1068400013F4800314BF0D480D48C1F3881118BF1D
:10685000002302F03F02A1FB00010FF091FE064B66
:106860005B68C3F3014301335B00B0FBF3F008BD89
:106870000248FCE70248FAE70038024000127A00BA
:106880000024F4002DE9F0410D46044610B9012022
:10689000BDE8F081434B1A6802F00F028A4228D308
:1068A00021688F072DD4C80740D43E4B1A6802F0E8
:1068B0000F02AA4265D8226851076BD4130707D587
:1068C000394A2169936823F4604343EAC103936022
:1068D000FFF7AAFF344B354A9B68C3F30313D35C1D
:1068E000D840334B1860334B1868FDF7CDFD0020BE
:1068F000CEE7CAB21A701B6803F00F038B42C6D1F1
:10690000CEE7294B11F0040F1EBF9A6842F4E05203
:106910009A600E0742BF9A6842F460429A609A6891
:10692000A06822F0F00202439A60BCE762681E4B46
:10693000012A1CD11B6813F4003FA8D01A4EB3687B
:1069400023F003031343B360FDF7CEFD41F2883813
:106950000746B368626803F00C03B3EB820FA4D060
:10696000FDF7C2FDC01B4045F3D9032090E7911EFF
:1069700001291B6802D813F0007FDEE713F0020F35
:10698000DBE7EAB21A701B6803F00F03AB427FF437
:106990007EAF90E70449E0688B6823F4E05303433B
:1069A0008B608BE7003C02400038024040BB01088E
:1069B000CC000020C8000020014B1868704700BFC1
:1069C000CC000020044B054A9B68C3F38223D35CB0
:1069D000034A1068D84070470038024038BB0108AD
:1069E000CC000020044B054A9B68C3F34233D35CC0
:1069F000034A1068D84070470038024038BB01088D
:106A0000CC0000200F2303600B4B9A6802F00302B6
:106A100042609A6802F0F00282609A6802F4E052E2
:106A2000C2609B68DB0803F4E0530361034B1B68FF
:106A300003F00F030B60704700380240003C024037
:106A400002682DE9F34112F0010504460BD09A4982
:106A50004569D1F88C3023F0C0632B43B5FA85F536
:106A6000C1F88C306D0997070BD59348A169D0F810
:106A70008C3023F0C0530B430029C0F88C3008BF82
:106A80000125160734D5002301938B4B8B4E1A6CCE
:106A900042F080521A641B6C03F080530193019BF7
:106AA000336843F480733360FDF71EFD0746336897
:106AB000D80540F19E80804EE269336F13F4407335
:106AC00040F0A180E36903F44072B2F5407F7A4A56
:106AD00040F0BC80916823F0704021F4F81120F45C
:106AE000407001439160116FC3F30B030B431367B5
:106AF00023685B0742BF724B94F83820C3F8E0214B
:106B00002268D70608D56C49606AD1F8943023F41E
:106B100040030343C1F89430960602F0400040F170
:106B200099806549A66AD1F8943023F00063334315
:106B3000B6F1006FC1F8943040F08C8038B1D1F8D4
:106B40009430226A23F080531343C1F894305D4B94
:106B5000594E00229A66FDF7C7FC054633681B01B3
:106B600000F18F80564B626BC3F8D8202268D7079C
:106B700001D563698BB1960701D5A3696BB1950601
:106B800003D5A36AB3F1006F07D0500612D5236A6C
:106B900083B9A36AB3F1006F0CD1E368A1681B0647
:106BA00043EA811361680B43216943EA0173424957
:106BB000C1F8843011060CD5E368A2681B0643EACD
:106BC000821362681343226943EA02733A4AC2F8A5
:106BD00084303C4B384E01229A66FDF785FC054611
:106BE00033681A0146D4FDF77FFC401B0228F7D911
:106BF00005E0FDF779FCC01B02287FF658AF0320A3
:106C000002B0BDE8F08102F4407293423FF45AAF03
:106C1000336F2C4A0121C2F8401E23F44073002137
:106C2000C2F8401E3367336FD9077FF54BAFFDF7CE
:106C30005BFC41F288380746336F9A073FF542AF55
:106C4000FDF752FCC01B4045F6D9D8E7916821F406
:106C5000F81147E740B11849206AD1F8943023F081
:106C600080530343C1F89430012D3FF470AF802A64
:106C70003FF46DAF2268D1050AD4930512D40020E9
:106C8000BEE7FDF731FC401B02287FF667AFB6E791
:106C90000949E06AD1F88C3023F000430343C1F87E
:106CA0008C30EAE7044A216BD2F88C3023F400439D
:106CB0000B43C2F88C30E2E700380240007000401D
:106CC000001047420000474203682DE9F341DD0709
:106CD000044610D4236898075BD423681A0700F190
:106CE0009C8023685B0700F1BC80A269002A40F009
:106CF000238100202CE08D4B9A6802F00C02042ABC
:106D00001ED09A6802F00C02082A02D15B68590270
:106D100016D46368854DB3F5803F1CD12B6843F4CE
:106D200080332B60FDF7E0FB804E054633689B0304
:106D3000D0D4FDF7D9FB401B6428F7D9032007E026
:106D40007A4B1B689A03C5D56368002BC2D101201A
:106D500002B0BDE8F081B3F5A02F04D12B6843F455
:106D600080232B60DAE72A6822F480322A602A68BE
:106D700022F480222A60002BD4D1FDF7B5FB064611
:106D80002B689F03A6D5FDF7AFFB801B6428F7D9BE
:106D9000D4E7664B9A6812F00C0F18D09A6802F08C
:106DA0000C02082A02D15B685E0210D5E268604BD3
:106DB000E2B91A60FDF798FB5C4E05463368990707
:106DC0008BD5FDF791FB401B0228F7D9B6E7574A50
:106DD00013689D0702D5E368012BB8D113682169B8
:106DE00023F0F80343EAC103136076E701221A6037
:106DF000FDF77AFB4D4D06462B68980707D52B68A3
:106E0000226923F0F80343EAC2032B6065E7FDF72C
:106E10006BFB801B0228EFD990E76269444B82B17B
:106E20000122C3F8802EFDF75FFB404E0546736FCD
:106E30009F073FF556AFFDF757FB401B0228F6D9D9
:106E40007CE7C3F8802EFDF74FFB384E0546736F85
:106E500098077FF546AFFDF747FB401B0228F6D9A0
:106E60006CE7324B1A6C12F0805228D101921A6CE6
:106E700042F080521A641B6C03F080530193019B13
:106E800001272C4D2B68D9051BD5A368274D012B55
:106E900027D12B6F43F001032B67FDF725FB234E12
:106EA000054641F28838336F9B0739D5002F3FF4F0
:106EB0001CAF1E4A136C23F08053136415E70027A0
:106EC000DFE72B6843F480732B60FDF70DFB06466C
:106ED0002B68DA05D9D4FDF707FB801B0228F7D908
:106EE0002CE7052B04D12B6F43F004032B67D0E76D
:106EF0002A6F22F001022A672A6F22F004022A6711
:106F0000002BCAD1FDF7F0FA41F2883806462B6F04
:106F10009807CBD5FDF7E8FA801B4045F7D90DE778
:106F2000FDF7E2FA401B4045BDD907E700380240B3
:106F30000000474200700040244DAB6803F00C0392
:106F4000082B3FF404AF224B022A4FF000021A66CE
:106F50002ED1FDF7C9FA06462B68990122D4226A80
:106F6000E3691343626A43EA8213E26A43EA026313
:106F7000226B43EA0273A26A5208013A43EA0243CF
:106F80006B60134B114D01221A66FDF7ADFA0446F2
:106F90002B689A013FF5ADAEFDF7A6FA001B02285B
:106FA000F6D9CBE6FDF7A0FA801B0228D4D9C5E6B6
:106FB000FDF79AFA04462B689B017FF59AAEFDF720
:106FC00093FA001B0228F6D9B8E600BF0038024049
:106FD00000004742704710B5044690B1437903F072
:106FE000FF0213B90271FFF7F5FF226802236371F4
:106FF000136843F004031360002001236371A06051
:1070000010BD0120FCE77047026838B5D36823F053
:10701000A003D3600446FDF767FA05462368DB68E2
:107020009B0601D5002038BDFDF75EFA401BB0F588
:107030007A7FF3D90320F6E738B50368DA68520699
:10704000044601D5002038BD4FF0FF32DA60FDF76D
:107050004BFA05462368DB685B06F3D4FDF744FA78
:10706000401BB0F57A7FF5D90320ECE738B504462C
:10707000B8B1437F03F0FF0213B90277FFF7C3FFF4
:10708000022363772368CA225A6253225A62204637
:10709000FFF7D2FF2368054630B1FF225A6204236E
:1070A00063770125284638BD9A68206922F4E002FA
:1070B00022F040029A606268996802436069024364
:1070C0000A439A60E2681A611A69A16842EA0142B9
:1070D0001A61DA6822F08002DA609B689B0605D4A8
:1070E0002046FFF791FF08B12368D6E72368A1691E
:1070F0001A6C22F480221A641A6C0A431A64FF2262
:107100005A6201236377CDE70368503343F82120A7
:1071100070470368503353F8210070472DE9F04160
:10712000069F0446884616461D462268936838EA3C
:1071300003030CBF01230023B34201D100202DE043
:107140006B1CF3D0FDF7D0F9C01BA842EDD3236828
:107150005A6822F0E0025A606268B2F5827F0AD172
:10716000A268B2F5004F02D0B2F5806F03D11A6861
:1071700022F040021A60A26AB2F5005F07D11A68D5
:1071800022F400521A601A6842F400521A60012375
:1071900084F85130002384F850300320BDE8F0819A
:1071A00030B50B4613490D681349B5FBF1F54FF4A3
:1071B0007A714D43416885B0B1F5827F04460395ED
:1071C0000CD1009280210022FFF7A8FF78B1636DF7
:1071D00043F020036365032005B030BD039B33B14A
:1071E000039B013B039323689B681B06F6D4002096
:1071F000F2E700BFCC00002000366E0137B50B4629
:107200004168B1F5827F044608D000920121002236
:10721000FFF784FFC8B9002003B030BD8168B1F525
:10722000004F08D0B1F5806F0AD10568296821F0B8
:1072300040012960E9E70068016821F04001016030
:107240000092802100222046E2E7636D43F0200394
:1072500063650320E0E7704738B5044600283BD05B
:1072600090F8513003F0FF021BB980F85020FFF76F
:10727000F2FF2168A568A06AA269022384F8513050
:107280000B6823F040030B6063682B43E5682B43D6
:1072900025692B4365692B43E5692B43256A2B43FD
:1072A000034302F400752B430B60120C636AB0F5C4
:1072B000005F02F0040242EA030208BFE36A4A6088
:1072C00008BF0B61CB6923F40063CB61002001236D
:1072D000606584F8513038BD0120FCE738B590F87E
:1072E0005030012B04465CD0012380F8503090F8D8
:1072F0005130012BDDB252D1002939D0002A37D0CC
:10730000032380F85130002343658363C2864364BE
:10731000C387036483878368828602680163B3F549
:10732000004F02BF136843F480431360836AB3F5D0
:10733000005F07D1136823F400531360136843F40C
:1073400000531360A06C184B0364184BC363184BB5
:10735000C36400230365E38E0C329BB2FDF7F8F99A
:1073600058B1636D43F010036365012384F8513015
:10737000002384F85030284638BD23681A68520626
:107380005EBF1A6842F040021A605A6842F020025A
:107390005A605A6842F002025A600025E8E7022566
:1073A000E6E70225E7E700BFDD7400082375000863
:1073B0000175000870B5044690F8500001287ED091
:1073C000012084F8500094F8510066680128C5B285
:1073D00007D0B6F5827F70D1A06800286DD1042D4A
:1073E0006BD1002941D0002A3FD0002B3DD094F82A
:1073F0005100A38604281CBF052084F851000020FA
:107400006065A387E386E387A36A2163B3F5005F22
:107410002168A2632064606407D10B6823F40053E1
:107420000B600B6843F400530B6094F85130254E09
:10743000E06C254D042B254B18BF1D46244B0564DD
:1074400018BF3346C363234BC36400230365E38F34
:107450000C319BB2FDF77CF9034658B1636D43F0E4
:1074600010036365012384F851300120002384F860
:10747000503070BD2268A06C516841F0010151602C
:107480000364C363C3640365E38E216B9BB20C3258
:10749000FDF75EF90028E1D123681A6852065EBF45
:1074A0001A6842F040021A605A6842F020025A609C
:1074B0005A6842F002025A60D8E70220D6E702205A
:1074C000D7E700BF33760008E9740008F5740008B8
:1074D0008D750008017500087047704708B5806B0E
:1074E000FFF7FBFF08BD704708B5806BFFF7FBFF98
:1074F00008BD704708B5806BFFF7FBFF08BD7047FC
:10750000806B026808B5536823F003035360436D32
:1075100043F010034365012380F85130FFF7EFFF7C
:1075200008BD37B50546846BFCF7DEFF2B681B688A
:10753000DB05024626D42368596821F020015960F2
:10754000596821F00201596020466421FFF728FEA6
:1075500018B1636D43F020036365A36833B90193E9
:107560002368DA6801929B680193019B0023E386FC
:10757000012384F85130636D23B12046FFF7BFFF2C
:1075800003B030BD2046FAF7BDFAF9E773B50646F9
:10759000846BFCF7A9FF33681B68DA05054644D401
:1075A0002268536823F020035360A36AB3F5005F99
:1075B0000DD101220090642311462046FFF7AEFD55
:1075C00018B1636D43F0020363652368DB68A2684A
:1075D000236832BB6268B2F5827F22D15A6822F0FA
:1075E00003025A6064212A462046FFF707FE08B1CD
:1075F000202363650023E3872268012384F8513048
:107600009368DB0606D5636D43F0020363654FF6AE
:10761000EF739360636D43B12046FFF770FF02B0D4
:1076200070BD5A6822F00102DBE72046FFF754FFE5
:10763000F5E773B50646846BFCF756FF33681B68A5
:10764000D90505463CD42268536823F020035360D3
:10765000A36AB3F5005F0DD10122009064231146A7
:107660002046FFF75BFD18B1636D43F002036365CD
:107670002368DB682A4664212046FFF791FD18B194
:10768000636D43F02003636523685A6822F00302A8
:107690005A600022E286E287012284F851209A682B
:1076A000D20606D5626D42F0020262654FF6EF72B5
:1076B0009A60636D23B12046FFF721FF02B070BDD1
:1076C0002046FAF739FAF9E77FB5036859689A68EE
:1076D00056060446C2F3801508D4D60706D54E06D2
:1076E00004D5036C04B0BDE870401847900704D57A
:1076F0000E0602D5636C2046F4E79006C2F34016EE
:107700003AD41DB188063AD404B070BDD605FBD575
:107710008D06F9D5626D42F008026265002203927F
:107720009A680392039A626D002AEDD05A6822F09B
:10773000E0025A60012284F851208A0747D05A6833
:10774000E06C22F003025A6040B1234B0365FDF761
:107750007BF818B1636D43F040036365A06C0028AB
:10776000D2D01D4B0365FDF76FF80028CCD0636DB8
:1077700043F040036365C7E78806C5D585B194F833
:10778000510003284FF000051AD0606D40F004004E
:1077900060650095D868009098680090009866B180
:1077A000606D40F0010060650020029098680290D2
:1077B000186820F0400018600298D005AAD4B2E7FB
:1077C0000195DA6801929B680193019B9CE7204632
:1077D000FFF795FE98E700BFDD77000808B5806BDE
:1077E0000023C387C386FFF78AFE08BD704770B5C4
:1077F0000E461546044610B390F8493003F0FF02D8
:107800001BB980F84820FFF7F1FF04F10801206858
:1078100000F004FBA2682068314600F03DFB236BBA
:10782000A2686068294600F061FB2268A16852F8EE
:10783000213043F0010342F82130002070BD0120C7
:10784000FCE770470368DA6842F00102DA609A6880
:1078500002F00702062A1EBF1A6842F001021A60EF
:10786000002070470368DA6822F00102DA60196AC2
:1078700041F21112114208D1196A40F244421142F8
:1078800002BF1A6822F001021A6000207047704798
:10789000704770477047704703681A69910710B5C1
:1078A00004460ED5DA6892070BD56FF002021A6112
:1078B0009B6901229B07027777D0FFF7EAFF00233D
:1078C000237723681A69500710D5DA6851070DD558
:1078D0006FF004021A619B69022213F4407F227741
:1078E000204668D0FFF7D5FF0023237723681A6965
:1078F00012070FD5DA6810070CD56FF008021A616D
:10790000DB6904229907227720465AD0FFF7C1FF8E
:107910000023237723681A69D20610D5DA68D006C7
:107920000DD56FF010021A61DB69082213F4407F55
:10793000227720464BD0FFF7ACFF00232377236844
:107940001A69D10708D5DA68D20705D56FF00102A8
:107950001A612046FFF79BFF23681A69100608D5B5
:10796000DA68110605D56FF080021A61204600F032
:10797000A2F823681A69520608D5DA68500605D5B8
:107980006FF040021A612046FFF785FF23681A69ED
:10799000910622D5DA6892061FD56FF020022046A4
:1079A0001A61BDE8104000F085B8FFF771FF20466E
:1079B000FFF770FF83E7FFF76BFF2046FFF76AFFD3
:1079C00092E7FFF765FF2046FFF764FFA0E7FFF7A8
:1079D0005FFF2046FFF75EFFAFE710BD264A036852
:1079E00090421BD0B0F1804F18D0A2F57C4290425B
:1079F00014D002F58062904210D002F5806290426D
:107A00000CD002F57842904208D002F570529042B4
:107A100009D1CA6823F44073134317E04A6823F07E
:107A200070031343F5E7154A9042F2D002F58062E5
:107A30009042EED0A2F598329042EAD002F58062F0
:107A40009042E6D002F580629042E2D04A6923F08B
:107A50008003134303608B68C3620B688362064B29
:107A6000984203D003F58063984201D10B69036308
:107A700001234361704700BF000001400044014002
:107A800010B50446A0B190F83D3003F0FF021BB9D9
:107A900080F83C20FFF7D5FE0223206884F83D30B3
:107AA000211DFFF79BFF012384F83D30002010BD0E
:107AB0000120FCE7704770470368DA6822F490728F
:107AC000DA605A6922F001025A61202380F83A30C4
:107AD0007047000038B50368C1681A69044622F48B
:107AE00040520A431A612569A268D968C0692A43CD
:107AF000656921F416412A4321F00C0102430A432F
:107B0000DA605A69A16922F440720A43B0F5004F65
:107B10005A61254A28D1934203D002F580629342EC
:107B20001FD1FEF75FFF6268192192184FF0000322
:107B30005B41A0FB01010EF023FD6422B0FBF2F1DA
:107B400002FB1103DB003233B3FBF2F303F0070255
:107B50005B00206802EB011203F4F87313448360A6
:107B600038BDFEF72FFFDEE7934202D00F4A934263
:107B700017D1FEF737FF636819219A00A0FB0101B6
:107B80009B0F0EF0FDFC6422B0FBF2F102FB11032F
:107B900024681B013233B3FBF2F303EB0113A36040
:107BA000DEE7FEF70FFFE6E700100140001401409A
:107BB000704710B5044640B390F8393003F0FF0227
:107BC0001BB980F83820FFF7F3FF2268242384F8DC
:107BD0003930D36823F40053D3602046FFF77AFF8F
:107BE00023681A6922F490421A615A6922F02A0223
:107BF0005A61DA6842F40052DA6000202023E06320
:107C000084F8393084F83A3010BD0120FCE7704721
:107C1000704790F83A30222B10B524D1816804695E
:107C20000268836AB1F5805F22D15268E4B9C2F379
:107C3000080223F8022B8362C38D013B9BB2C385EC
:107C40008BB90368DA6822F02002DA60DA6822F47D
:107C50008072DA605A6922F001025A61202380F8AA
:107C60003A30FFF7D5FF10BDD2B223F8012BE2E77F
:107C7000591C526881620CB91A70DDE702F07F026C
:107C8000FAE7704702681368D16870B51E07556936
:107C9000044607D19E067CD58D067AD5BDE8704096
:107CA000FFF7B7BF15F001052ED013F0010F03F059
:107CB000040246D11AB1E26B42F00202E2639E076F
:107CC0002CD5E26B42F00402E26313F0080F03D0FC
:107CD000E26B42F00802E263E26BA2B1980604D5BF
:107CE0008A0602D52046FFF794FF21684B69E26BB4
:107CF00003F0400302F0080253EA020520462ED1A9
:107D0000FFF7BFFFE56370BD11F4907F41D013F022
:107D1000010F03F0040207D19A070DD41E07DBD52B
:107D200001F020022A43D2E7C8050FD4002AF3D17C
:107D30009807F3D5002DC4D11A07CDD511F0200F27
:107D4000C5E7CE0502D4002AB5D1F1E7E26B5807AA
:107D500042F00102E263EBD5002DDDD0ABE7FFF787
:107D6000ABFE4B695B0610D54B69606B23F040039B
:107D70004B6150B1244B0365FCF766FD0028C2D06F
:107D8000606BBDE87040036D18472046FFF779FF30
:107D9000B9E71E0628D50D0626D594F83930212BD3
:107DA000B1D1A168236AB1F5805F18D11988C1F3F8
:107DB00008015160216981B902332362E38C013BE0
:107DC0009BB2E384002B9ED1D36823F08003D36061
:107DD000D36843F04003D36095E70133EDE7591CC6
:107DE00021621B785360E9E758068CD54B068AD58B
:107DF000D36823F04003D360202384F83930204631
:107E0000FFF705FF7FE700BF0D7E000808B5806B18
:107E10000023C385C384FFF734FF08BDF0B50C68A9
:107E20001C4D50F824308F68CA684E6BD1F838C0AA
:107E30001D404B683B4313430A6913434A6913438C
:107E4000CA6913430A6A13434A6A13438A6A13438B
:107E5000CA6A13430A6BC96B134333430B4343EAA8
:107E60000C032B43082F08BF43F04003B6F5801FD7
:107E700040F8243009D154B1036843F480130360FF
:107E800003684CEA0302026001E0002CF8D10020F4
:107E9000F0BD00BF8004C0FFF0B50B688F690C69AE
:107EA0003B434F6843EA07138F6800EB820243EAC3
:107EB0000723CF6849695668013C43EA074343EA10
:107EC0000453023906F0404643EA016333435360EA
:107ED0000368DB0248BF43684FEA045542BF23F4FE
:107EE00070032B4343600020F0BD0000B3F5804FCA
:107EF00030B514D150F822300A4C8D691C400B6803
:107F00002B434D6843EA05138D68C96843EA05238E
:107F100043EA0143234340F82230002030BD6FF094
:107F20007043F8E70000F0CF054BD3F8882042F407
:107F30007002C3F888204FF000629A60704700BF5B
:107F400000ED00E0DFF834D0002103E00C4B5B587B
:107F5000435004310B480C4B42189A42F6D30B4A5B
:107F600002E0002342F8043B094B9A42F9D3FFF7A1
:107F7000DBFF0FF0F9FCF8F739F970470000042037
:107F8000E00B020800000020080200200802002088
:107F900088180220FEE737B50D4600F108010246B9
:107FA000C36A03C91C688DE803001046694601F0E6
:107FB0008AF8B5F90020BDF9003022449A4217DC56
:107FC000B5F90420BDF90430121B9A4210DBB5F953
:107FD0000220BDF9023022449A4209DCB5F90600BC
:107FE000BDF90630041B9C42ACBF0020012000E01C
:107FF000012003B030BDB0F9003070B5B0F90460B5
:108000001588D088948852884D80F31A9BB2181A2C
:108010009B1A08808B80CC8070BD438E1B0713B5E4
:108020000C460FD5684601F061FBBDF80230238095
:10803000BDF80630A380BDF800306380BDF8043081
:10804000E38002E0084601F051FB02B010BD38B5F4
:1080500004460D4601F0F9FFE36A284629461A68EE
:10806000BDE8384005F0DCBA37B50C46054607F0E8
:108070003FFB428E0190944203D04486284602F092
:108080002CF801A807F042FB03B030BD37B50C4611
:10809000054678B107F02CFB428E019004EA0201FC
:1080A0008C4204D014434486284602F016F801A8F6
:1080B00007F02CFB03B030BD37B50D46044670B158
:1080C00007F016FB428E019022EA05018A4203D096
:1080D0004186204602F001F801A807F017FB03B023
:1080E00030BD0000024B42861B68C36201867047A8
:1080F000D0000020F0B50D4685B00646002800F0FF
:10810000938007F0F5FA2B680290162B52D00CDC06
:10811000112B33D002DC0D2B3ED07EE0142B77D018
:10812000152B7AD1B0F9303070E01F2B6BD002DC08
:108130001E2B42D071E0312B1ED0B3F5407F6CD1A5
:10814000C36A1968EB68C3621B6802A8CD1A07F0FE
:10815000DDFA304607F0CCFA04AC694244F8040D6D
:108160000A462B46009500F034FF204607F0CEFA71
:10817000304601F0B2FF4EE000243FE0438ED906C6
:108180004BD5EB681B7A002B47D002A807F0BEFA4C
:10819000304601F017F840E0EB68DB68002B3CD07C
:1081A0001B7A002B39D002A807F0B0FA304601F054
:1081B000BDFA30E0EB6803862DE0EB68418E012BC1
:1081C00008D1CA060DD5304641F00101FFF74CFF3A
:1081D000082708E021F001013046FFF745FF092795
:1081E00001E04FF0FF3702A807F090FA7B1C4FF038
:1081F000000405D03046394601F0B7F8EC600DE0D8
:108200000123EB600AE0438EC3F30013EB6002E04E
:10821000E968FFF71CFF002400E00124029B23B162
:1082200002A807F073FA00E00124204605B0F0BD73
:1082300070B50D46FE211646044601F035FA294672
:1082400000F0B3FF2046FF2101F02EFA3146BDE8D1
:10825000704000F0AABFF8B51C46438E069F1B076E
:108260000D4616460AD5002C07DB2846311BA219FD
:1082700006F018FB013C3D44F5E7F8BD002C07DB98
:108280002846311BA21906F095F8013C3D44F5E75C
:10829000F8BD37B505460C4619B9684601F026FA0F
:1082A0006C466B8E1B0705D5224628466946FFF7AC
:1082B000A2FE6C4628462146FFF76DFE18B1EB6A18
:1082C00020461B69984703B030BD2DE9F04F2DEDD6
:1082D000028B85B00D4607F00BFA0090006905F09F
:1082E0001BFF009BD86805F045FF022005F0F8FE53
:1082F000009CA68CE36916F001061AD0002B77D0FB
:10830000A06807F0F5F90190C26A636917681F4415
:1083100001F01EF9A369384433B1012B70D1B5F9CE
:10832000003083426CDD1CE0B5F90430834218DB79
:1083300066E0002B5CD0A06807F0DAF90190C36A10
:10834000D3F8008006F010F863690746C8EB03090C
:1083500001F006F9B5F90210EA88484407448F4253
:1083600003DA01A807F0D2F942E012B29042F8DC39
:10837000A06802A901F0FCF8019BBDF90CB0DA6D10
:10838000D3F854A0BDF90870256AC2EB0B0BB3F803
:108390007820D207574458BFD3F88C603D44354409
:1083A000BD4222DDE369ED1AFAE7BD421BDDA0699B
:1083B00005F0A0FE236AD4ED0A7AEB1ACAEB030398
:1083C000C8EB03039B1B08EE103AB8EEC88A284698
:1083D00028EE278A494605F0ABFFB0EE480A94F82C
:1083E0002C0005F0A5FCE3691D445D45DDDDB8E723
:1083F000684607F08BF905B0BDEC028BBDE8F08F45
:10840000A06802A901F0B4F8019B1D6ED3F8588052
:1084100005F0AAFFBDF90E60019BBDF80AA0D3F8D4
:108420008030761B256A751B1D44B54201DAE3696D
:10843000FAE74FF0020990FBF9F908FA8AF39D4236
:108440008FDBB5421CDCA06905F054FE236AD4ED35
:108450000A7A711BC91A019BD3F880208A1808EE8A
:10846000102AB8EEC88A384628EE278AC9EB0501DB
:1084700005F05EFFB0EE480A94F82C0005F058FCB9
:10848000E369ED1AD9E700002DE9F3478146302072
:10849000884617461E4607F0FDFB8246D0B107F01E
:1084A00027F902AD0D4A45F8040D4FF07E53836263
:1084B000C0F81490C0F818808784C66100F10C03DE
:1084C000044692E8030083E80300054B2360284636
:1084D00007F01CF9504602B0BDE8F087D400002038
:1084E000CB82000800B52DED028BF0EE408A83B000
:1084F00090B107F0FDF890ED0A8A0190B4EE688A19
:10850000F1EE10FA04D0C0ED0A8A806801F0E5FDB2
:1085100001A807F0FBF801E09FED048AB0EE480ADD
:1085200003B0BDEC028B5DF804FB00BF000000004F
:1085300013B5044607F0DCF80190406A20B107F05B
:1085400011F9019B00225A6201A807F0DFF82046CA
:1085500007F008F902B010BD2DE9F0438BB007F029
:10856000C7F80790406A002860D007F0C1F8079B61
:1085700005900646986807F0BBF8079BD0F8548032
:10858000056E876DC46D069008A9986800F0F0FF2D
:10859000BDF82230079A0698BDF82010D2F8209036
:1085A0001F44ADF82270BDF82430BDF826701C1BA6
:1085B0007F1B1369D0F88C505D1B92F82830414422
:1085C00089B2A4B2BFB2012BADF82010ADF824409F
:1085D000ADF82670D0F8808009B208D024B2641BB0
:1085E0000134A14204DD0C1B06EB44062D1B0C4696
:1085F000002D15DD906905F0BDFD4FF0FF32012320
:108600008DE80C00079A3FB292F829300293C9EB2B
:10861000070930462946224609EB080306F066F9A9
:1086200006A807F073F805A807F070F807A807F088
:108630006DF80BB0BDE8F0831FB590F82830012B22
:108640000446806827D102A900F092FFA06807F0D5
:108650004FF8BDF80A20836D01901344ADF80A303D
:10866000BDF80E20036ED31AADF80E30426DBDF882
:1086700008301344226913449BB29A1E01A8013B9F
:10868000ADF80820ADF80C3007F040F8A06802A95A
:1086900001F0E7FC01E000F05FFB04B010BD00005A
:1086A0002DE9F74380462C200E4617461D4607F05D
:1086B000F1FA044618B3700007F0ECFA814658B19D
:1086C00057B14DB107F014F839466A0001900FF028
:1086D000CFF901A807F01AF8204607F009F80A4B6D
:1086E0000190C360094B0360094BC0F82490C0F8A7
:1086F000188046610561436001A807F007F820462D
:1087000003B0BDE8F08300BF398600085985000832
:10871000318500081FB5ADF8061006F0E9FF02909C
:1087200068B1406A06F0E4FF0DF1060201460390CD
:108730000223029800F03FFB03A806F0E7FF02A81F
:1087400006F0E4FF05B05DF804FB13B50C4660B11C
:1087500006F0CEFF036A0190A34203D00462806852
:1087600001F0BBFC01A806F0D1FF02B010BDF0B5CE
:108770008BB002A9044600F0FBFE204606F0B8FFCD
:10878000BDF90A20BDF90E600190B61A826D456DE3
:10879000C76DB61A026EB61AB0F87820510707D422
:1087A000416FB1422046D4BF0021012100F0FBFC03
:1087B000019BBDF90C105A6FDA67BDF90820C3F8A8
:1087C00084608A1A551BB3F878209207C7EB050519
:1087D00007D4196FA9422046D4BF0021012100F01F
:1087E000E0FC0198036FC0F88830C0F890507C30EE
:1087F00000F08AFF0198883000F086FF019B03F1AA
:108800007C0207CA883307AE86E8070093E80700B2
:1088100004AD85E8070001A806F078FF2046314640
:108820002A46FFF705FD0BB0F0BD73B50C460646B2
:1088300006F05EFF0190204607F066FB05462046E5
:1088400000F0F6FE019BFE280CBFC3F88050C3F871
:108850008C50304601F041FC01A806F057FF02B0F1
:1088600070BD2DE9F04F44680668054697B0204674
:108870002946FFF73FFCB6F5407F074602D1204668
:10888000FFF775FF002F00F064822B680B2B00F0C0
:10889000008206DC052B40F059822046FFF767FF77
:1088A00054E20F2B03D0262B00F03D824EE2ED6800
:1088B0000295204606F01CFFC36AC16D1B68D0F804
:1088C0005490D0F858B0D0F860A00D900EAD284666
:1088D0000393019100F00AFF0D982946FFF7D9FC98
:1088E00095E8030012AB83E803000398BDF84A1033
:1088F00082B25944BDF84E001144ADF84A1002EB63
:108900000A01411AADF84E10BDF84810114449440F
:10891000ADF8481001990A44BDF84C108A1AADF818
:108920004C2093E8030010AA82E80300104600F0F0
:10893000FBFB0D9B586B05F01BFC06F0A9FA0D9B89
:10894000D3F8943013B12046002198470D9D95F837
:108950006C30002B00F08D80204614A900F008FE3A
:10896000EB6ABDF856001B68BDF85420BDF85210E4
:1089700004930790BDF85030286C05920693089137
:108980006E6CAF6C05F0F6FB05F0E8FC099016B9CB
:10899000002F4BD146E0EB6C06EB030CB5F87830BA
:1089A000DB0754BFD5F88C3000230CEB0308B0452F
:1089B00002DBC6EB0808FAE795F87A0005F0A4FB9D
:1089C0000598019A03B206984A4401B2C2F1010225
:1089D0005B1A13449845DBDA0498BDF95210BDF9CF
:1089E000563095F87A20484440445944CAEB030372
:1089F0001AB1024605F038FF02E01A4605F0DAFC2B
:108A0000B044DDE795F87B0005F07EFB07990898F8
:108A10000BB20BEB0A0201B2C2F101025B1A134462
:108A20009E420CDB099805F06FFB22E02E6DD5F815
:108A300080303E44F61ABE42E4DBF61BFBE70198A9
:108A4000BDF95420BDF95610BDF95030121A95F8F1
:108A50007B00CAEB0101891B4B4420B118460B4631
:108A600005F002FF03E00846194605F01BFF3E44EF
:108A7000CCE7039A12A80EA904F0D2FD12A800F0C8
:108A800053FB0D9B93F83B20FF2A00F0A380B9F124
:108A9000000F08D1BBF1000F05D1019919B9BAF146
:108AA000000F00F09780DA6A14A920461568009339
:108AB00000F05EFD00F04CFD049000F051FDBDF9AA
:108AC0005220009BBDF9546005905A440392019ACC
:108AD000986BBDF95070BDF95680B61A05F048FB89
:108AE000009BD86B4F44CAEB080805F043FBB9F173
:108AF000000F1BD002980499B0F9003009F1FF3241
:108B00002A445B1A934211DCBDF95630BDF950007E
:108B1000CAEB030305EB0B01013306F087F9039A57
:108B2000781E511E08F1010205F044FCBBF1000F54
:108B300017D002980599B0F902200BF1FF332B44AE
:108B4000521A9A420DDCBDF95000BDF95210BDF920
:108B5000542006F06BF9039A791E501E721C05F022
:108B6000A1FE019BD3B10299BDF95420D01AB1F9ED
:108B70000430049901305B1A83420FDBBDF9563093
:108B8000CAEB030305EB0B01013306F04FF9039A1F
:108B9000701C511E08F1010205F00CFCBAF1000F27
:108BA00018D00298BDF95630B0F906200598CAEBE6
:108BB00003010131C0EB020A8A450BDBBDF950000D
:108BC000BDF9542006F032F908F10100791E721C3B
:108BD00005F068FE0D9BD3F8943013B120460121B7
:108BE000984710A800F0A0FA0D9B586E07F098FC6B
:108BF00000250746BD421AD00D9B2946586E07F046
:108C000011FD06F075FD149078B10668304606F047
:108C10006FFD0C9030B103680299304698470CA85C
:108C200006F074FD14A806F071FD0135E2E712A804
:108C300000F07AFA0D9B986E07F072FC002507464B
:108C4000BD421AD00D9B2946986E07F0EBFC06F04A
:108C50004FFD149078B10668304606F049FD0B9040
:108C600030B103680299304698470BA806F04EFDD4
:108C700014A806F04BFD0135E2E7002000F054FA9D
:108C80000D9BD3F8943013B12046022198470DA8CC
:108C900046E0204606F02CFD1290406E07F040FCA6
:108CA00000240646B442129B18DA586E214607F09B
:108CB000B9FC06F01DFD149070B10568284606F059
:108CC00017FD109028B1476810A806F01FFD284630
:108CD000B84714A806F01AFD0134E3E7986E07F0D0
:108CE0001FFC00240546AC42129B0FDA986E214609
:108CF00007F098FC06F0FCFC149028B1006806F020
:108D000031FD14A806F002FD0134ECE716AC586EF4
:108D100007F05FFC54F8103D986E07F05AFC2046AF
:108D200006F0F4FC15E0EB68052B0FD12046AE6889
:108D300000F0F0FB864205D02046AE6800F0E5FB6F
:108D4000864203D16868A968FFF76FFD284601F0E5
:108D5000EFFD17B0BDE8F08F2DE9FF41044606F0A6
:108D6000C7FC034604A8D3F8548040F80C3D9F6D1F
:108D7000DE6D1D6E06F0CAFC204602A900F0F8FB6D
:108D8000BDF808309844BDF80A30ADF808801F449B
:108D9000BDF80C30ADF80A709E1BBDF80E30ADF872
:108DA0000C605D1B204602A9ADF80E5001F059F988
:108DB00004B0BDE8F081F8B51D46836804460E4650
:108DC000174623B30069636998420ED1421E6A4375
:108DD000084629440EF096FD2069013800FB056025
:108DE00039462A460EF08EFD0CE0431C236100FB41
:108DF000051011462A460EF085FDE36813B12046A2
:108E00009847F8BDA068BDE8F840FFF7A5BFF8BDDA
:108E1000F0B587B00C9C00940D9C0194174C029403
:108E2000109C6C34039401F099F9064618B307F0CE
:108E30000CFC054607F009FC0446304606F058FCD9
:108E400045660F4D84660F9905900022FFF74AF999
:108E500006AF0FCD57F804ED0EF134040FC40FCD5B
:108E60000FC495E80F0084E80F000E9BAEF8783031
:108E7000384606F04BFC304607B0F0BD638800086A
:108E8000DC00002010B586B0089C0094099C019479
:108E90000A9C02940B9C039400240494FFF7B8FFEF
:108EA00006B010BD30B585B004460191D0B106F0D2
:108EB0001FFC04AB456E43F8040D184606F026FC73
:108EC000019806F015FC024604A8946040F8082DAD
:108ED00006F01CFC284601A9042207F030FB2046BE
:108EE00001F0FBF805B030BD30B585B00446019106
:108EF000D0B106F0FDFB04AB856E43F8040D1846B7
:108F000006F004FC019806F0F3FB024604A8946006
:108F100040F8082D06F0FAFB284601A9042207F0C4
:108F20000EFB204601F0D9F805B030BD73B50D46F3
:108F30001446064698B106F0DBFB032C019009D8D5
:108F400000EB8400446BAC4205D04563304601F031
:108F5000C4F800E0002401A806F0D8FB00E00446B5
:108F6000204602B070BD73B50E46054678B106F0D6
:108F7000BFFB90F86C400190B44204D080F86C6064
:108F8000284601F0AAF801A806F0C0FB00E004465C
:108F9000204602B070BD2DE9F3410F4690461D46B4
:108FA000064698B106F0A4FB044602A8089B236677
:108FB00040F8044D6765C4F85880E56506F0A6FBE7
:108FC0003046FFF7D4FB304601F087F802B0BDE829
:108FD000F0812DE9F04F87B0C46903938A46934628
:108FE000002C6DD0204606F083FB816A059001F4C9
:108FF0002073802BB0F8008042888688C58808D00E
:10900000B3F5207F08D108EB0A091FFA89F9039B01
:1090100008E0039883B201E01FFA8AF303EB080922
:109020001FFA89F901F4A0613344B1F5807F9BB246
:1090300008D0B1F5A06F08D102EB0B0C1FFA8CFC25
:10904000109F08E010998FB201E01FFA8BF707EB31
:10905000020C1FFA8CFC0FFA89F90FFA88F812B289
:109060002F440FFA8CFCB9EB08010292BFB2C2EB9D
:109070000C0200D142B120460193CDF800C000F0AF
:1090800008FADDF800C0019B1BB2C9EB030936B238
:10909000029BC6EB08083FB22DB2CCEB070C5D1B60
:1090A00019EB08010CEB050200D112B1204600F0CB
:1090B000E1F806A850F8043D1C6A06F027FB8FE78C
:1090C00007B0BDE8F08FB0F90030B0F902200846D3
:1090D0005242594205F0E0B810B5044670B100F0B4
:1090E000FCFF204600F0BBFA04463CB12046FFF7E7
:1090F000F3FF204606F0F2FA046AF6E710BD13B556
:10910000044670B106F0F4FA826A0190930705D420
:1091100042F0020282622046FFF7DEFF01A806F05D
:10912000F5FA02B010BD0000044B10B51B685C6C72
:10913000586400F02BFE204610BD00BF2401002023
:10914000F7B50D46114606461F4600F0ADFA044637
:10915000A5B120B93046394606F0E5FE14E006F028
:10916000C7FA02AB826A43F8040D22F4004242F0CF
:1091700002028262184606F0C9FA05E020B100F04A
:109180008CF9204601F006FB201C18BF012003B01B
:10919000F0BDFE220823FFF7D3BFFF220023FFF715
:1091A000CFBFFFF7FABFFFF7F4BF1FB530B129B14A
:1091B000242303916946009300F038FF05B05DF861
:1091C00004FB0000F0B587B00446002102A810227D
:1091D0000EF0B2FB002C3AD01F4B204A196852F80F
:1091E0002100844216461F4631D01E238DE811000F
:1091F000029310B102A907F03FFA0123204602A909
:10920000059307F039FA059D15BB3B6846F82340E6
:10921000204600F084F9044638B12023029302A9C5
:1092200000AB059307F028FAF2E7009C204600F017
:1092300032F968B1204600F072F9044640B12023AB
:10924000029302A900AB059307F016FAF2E7012595
:10925000284607B0F0BD00BF2817022018170220CB
:10926000024B1A6818601046704700BF3017022082
:1092700007F0EEB92DE9F04151EA02038AB08046C9
:109280000E4617466ED000286CD006F031FA034621
:10929000039003C804AD06AC85E8030084E803002E
:1092A0007EB19A6A02F42072802A05D1BDF8182096
:1092B000961BADF8186004E0BDF81C201644ADF80C
:1092C0001C6087B19A6A02F4A062B2F5807F05D172
:1092D000BDF81A20D71BADF81A7004E0BDF81E20A7
:1092E0001744ADF81E709B6ADA0302D5404600F0C1
:1092F00081FD94E80300039B83E803009B6A9B07BE
:109300000AD508A82946224604F0D6FF039B08A8E0
:1093100099691A6A00F072FEBDF91C40BDF914305B
:10932000BDF91E70BDF91600BDF91860BDF9101029
:10933000BDF91A50BDF91220E31A381A0AACAA1A5C
:109340000090711A0398FFF744FE54F81C1D01F1B8
:10935000080004F021FA4046052100F06BFE20468B
:1093600006F0D4F90AB0BDE8F0811FB526230391B9
:109370006946009307F0A6FA05B05DF804FB2DE9F5
:10938000F04188B006460C46154604A8002110227C
:109390000EF0D2FA36B3304606F0AAF921462A4634
:1093A000019004F079FF0198214608302A4604F024
:1093B00073FF08A850F81C2DD2F81C80176A06F01D
:1093C000A5F9404621462A46FFF7D9FF0323049317
:1093D000304602AB04A90793029403953E4607F07A
:1093E0004BF9D7E708B0BDE8F0812DE9F0438BB029
:1093F00006460D46144606A8002110220EF09CFADF
:10940000002E43D00DB9002C40D0304606F070F944
:109410000346019003C80DF1080888E803002246BE
:109420001846294604F038FF01980AAF294622461B
:10943000083004F031FF57F8243DD3F81C9038462B
:1094400006F064F9224648462946FFF798FF304661
:1094500006F04EF9826A019092070AD5816941B1FE
:10946000026A00F0B6FD019B404699691A6A00F055
:10947000B0FD384606F04AF903230693304604ABA4
:1094800006A909930495059407F0F6F80BB0BDE81A
:10949000F083FFF7AABF00F09DBC13B588B106F0BA
:1094A00027F9826A02AC910744F8040D06D522F030
:1094B000020282628169026A00F0A0FD204606F085
:1094C00025F902B010BD70B506460D4606F006F946
:1094D000C4694CB1204600F0ABF8A842204613D036
:1094E00006F0FCF8046AF4E7304606F0F7F8C469C1
:1094F000204644B12946FFF7E6FF28B9204606F08A
:10950000EDF8046AF4E770BD70BD10B1FF21FFF7FC
:10951000DABF704710B1FE21FFF7D5BF704708B51D
:10952000034610B106F0DAF88369184608BD08B59D
:1095300020B106F0D3F8B0F9000008BD08BD08B5A9
:1095400020B106F0CBF8B0F9020008BD08BD00005C
:10955000024B1B68986CFFF7EABF00BF2401002094
:10956000024B1B68986CFFF7EABF00BF2401002084
:10957000F0B50C4687B0064600284BD0002949D0EC
:10958000FF2100F091F8FE210546304600F08CF8EE
:1095900069460746304607F0BDF9304602A900F09B
:1095A0003BF8C7B1384604A907F0B4F9BDF900107B
:1095B000BDF9022004A84942524204F06DFE38462B
:1095C00000F046F800F08200822804D1BDF8103087
:1095D000013BADF80C30CDB1284604A907F09AF94B
:1095E000BDF90010BDF9022004A84942524204F01E
:1095F00053FE284600F02CF800F48170B0F5817F0E
:1096000004D1BDF81230013BADF80E3002AB03CBF4
:109610002060616007B0F0BD1FB5039104A9142359
:1096200041F8103D694600F001FD05B05DF804FB0E
:109630001FB504461022684600210EF07DF915235F
:1096400020466946009300F0F1FC039804B010BD79
:1096500008B518B106F042F8008D08BD08BD08B580
:10966000034610B106F03AF8C369184608BD37B58D
:109670000D4606F03DF802ABC46943F8040D1846E8
:1096800006F044F820466CB1FFF7D2FFA84220460E
:1096900008D02946FFF7EBFF20B9204606F01EF858
:1096A000046AEFE703B030BD08B1FFF7E0BF7047D1
:1096B000034B1B685A7C034B53F82200704700BFD2
:1096C000240100200817022037B50D4658B151B1CA
:1096D00006F00EF802AC294644F8040D00F0B5FC83
:1096E000204606F013F803B030BD0000044B0146DD
:1096F000186810B9034B1B68986CFFF7E5BF00BFF3
:10970000041702202401002002688368D31A4268EB
:10971000002ABCBF00224260426823EAE3739A42F7
:10972000C8BF4360704700F0D8BC000073B5054661
:10973000002832D005F0DCFF02AC034644F8080DE7
:10974000006A08B968460EE09B6A1A0711D405F052
:10975000CFFF836A02AE1B0746F8040D06D56846A4
:1097600005F0D4FF304605F0D1FF16E0304605F095
:10977000CDFF009B68469E6905F0C8FF284600F0B3
:10978000B7FA3146284600F061FA284600F0A5FCF9
:1097900028460349002207F0DCF802B070BD00BF84
:1097A000279700080A4A0B49002313700A4A0B60E6
:1097B00013600A4A4B601360094A13605360094AF8
:1097C0001360094A1360094A1360094A136070471D
:1097D000D8D7012018170220B0D701203C1702204B
:1097E00044170220501702200417022030170220CD
:1097F0004017022010B5044605F070FF836A044A42
:1098000013F4803F034B204608BF1346984710BD12
:1098100059A6000845AC0008F0B5054685B00C46D1
:109820001646002D4CD0284605F062FF876A01904D
:10983000BB0701463DD502AD26B12846324603F0AE
:1098400079FF02E003C885E803002046294604F0BA
:10985000D9FC70B317F0010F019B1ED13EB1B3F9D3
:109860000220B6F902309A42A8BF134601E0B3F9CC
:109870000230B4F902209342B4F9062006DDBDF8A7
:109880000A3019B28A4214DB013B04E0BDF80E3005
:1098900019B28A420DDDE3800BE0DF694FB1384633
:1098A00021462A46FFF7B8FF384605F017FF076A3A
:1098B000F4E704A850F80C3D1D6A05F027FFB0E757
:1098C00005B0F0BD2DE9FF4104460F469046002546
:1098D000002C37D0204605F00BFF866A0190B207B6
:1098E000014628D502ACB8F1000F04D0204642460C
:1098F00003F020FF02E003C884E803003846214655
:1099000004F080FCB8B1F30705D4BDF80C30013386
:109910003B8001250FE0019BDE6966B13046394688
:109920002246FFF7CFFF0028304618BF012505F07B
:10993000D5FE066AF1E704A850F80C3D1C6A05F054
:10994000E5FEC5E7284604B0BDE8F081F0B5044661
:1099500085B00E461746002C31D0204605F0C8FED3
:10996000856A0190AA07014622D502AC27B120469C
:109970003A4603F0DFFE02E003C884E80300304605
:10998000214604F03FFC98B1EB0704D4BDF8083041
:10999000013BB3800CE0019BDD694DB128463146A7
:1099A0002246FFF7D3FF284605F098FE056AF4E744
:1099B00004A850F80C3D1C6A05F0A8FECBE705B0E2
:1099C000F0BD00002DE9F341214D2B680646986C4F
:1099D00005F08EFE0090304605F08AFE02AC01468E
:1099E000019054F8080D083004F00CFC074628B329
:1099F0000199009A2B68174C1F6DD3F84C8001F128
:109A00000800083203F096FE684605F07FFE019AD2
:109A10002B68B2F90010B2F90220D9641A6501A8C6
:109A2000266005F073FE3046FFF7E4FE0023236056
:109A30002B681F65C3F84C80012705E0684605F0D8
:109A400065FE01A805F062FE384602B0BDE8F0816F
:109A500024010020041702202DE9F347064605F0F3
:109A600047FE836A01909B0705D401A805F04EFECE
:109A700002B0BDE8F087C469002CF6D0204605F09E
:109A800037FE836A02AD03F00303032B45F8080D8C
:109A900037D10199083104F0B5FB002831D002A874
:109AA00050F8043DB3F80890B3F80A809F89B3F8E2
:109AB0000EA005F02BFE684605F028FE2046FFF7B5
:109AC00081FF70B1204605F009FE00902046FFF7A7
:109AD000C3FF204605F002FE0090304605F0FEFD73
:109AE0000190304605F004FE0190204605F000FE8E
:109AF000019B0090A3F80890A3F80A809F81A3F827
:109B00000EA0009B68461C6A05F000FEB4E700004A
:109B100037B5044605F0ECFD826A019040F601037A
:109B20001340012B05D001A805F0F0FD2046FFF7FA
:109B300061FE144B1B6813B32046FFF78DFF2046D0
:109B400005F0CCFD8569046ACDB194B1204605F0DD
:109B5000C5FD836A03F00303032B02D12046FFF700
:109B600031FF2046FFF778FF204605F0B7FD046A75
:109B7000EBE7284605F0B2FD046A8569E4E703B027
:109B800030BD00BF501702202DE9F347174D2B6859
:109B90000646986C05F0ACFD2A68B0F808A0B0F84D
:109BA0000A90B0F80C80C78902AC083244F8040D62
:109BB00000F1080392E8030083E80300204605F063
:109BC000A5FD3068FFF7A4FF2B68986C05F090FDA9
:109BD0000190A0F808A0A0F80A90A0F80C80C78116
:109BE000204605F093FD02B0BDE8F0872401002077
:109BF000F7B507460D46284605F07AFD836A02ACA4
:109C000013F00206014644F8040D04D1204605F085
:109C10007DFD304616E0384603F0BEFD019B9E698F
:109C2000204656B905F072FD074B1A68954208D0D8
:109C300058682B1A5842584104E005F067FD354634
:109C4000D9E7012003B0F0BD08170220F0B50446A3
:109C500085B00D46002949D005F04AFD0023036276
:109C600085610190284605F043FD019BC56902907E
:109C70009F6A2DB9C46101A805F048FD02A833E030
:109C8000284605F035FD04AE07F0080746F8040D38
:109C900077B9836A1A070BD5019B1D62029B01A845
:109CA000DC6105F033FD02A805F030FD30461BE015
:109CB00002A805F02BFD304605F028FD284605F0EA
:109CC0000DFD0390039B1D6A0DB91C620BE0284635
:109CD00005F004FD002FF4D1836A1B07F1D5039B27
:109CE0001C62019B1D6201A805F010FD05B0F0BDCE
:109CF00070B5044605F0F2FC05468069A8B105F090
:109D0000EDFCC369A342064605D1184605F0E6FC02
:109D1000036AF36170BD43B1184605F0DFFC036AC6
:109D2000A342F8D12B6A036270BD70BD034608469A
:109D3000B3F90220B3F9001004F0AEBA114B30B5FC
:109D40001C68626C85B00546BAB11068516802ABF8
:109D500003C30D4B186800B9A06C05F0C9FC04AC36
:109D600002A944F80C0DFFF7E1FF204605F0CEFCF8
:109D700002A8294603F010FD02A802F033FF05B047
:109D800030BD00BF24010020041702201FB50E4B78
:109D90001B6893F854200AB10C4811E0986C05F048
:109DA000A7FC019003C802AC84E8030001A805F0F9
:109DB000ADFC074B196811B12046FFF719FF20468B
:109DC000FFF7BCFF04B010BD24010020BCD7012068
:109DD00004170220064B10B50446186828B1A042AB
:109DE00004D005F07BFC4069F8E710BD012010BDF0
:109DF0002417022013B5044600B305F079FC826AEB
:109E00000190930717D5406A40B10D4B1B68A342E0
:109E100004D001F0DFFD019B00225A622046FFF7CB
:109E20001EFC04463CB12046FFF7E4FF204605F047
:109E300055FC046AF6E701A805F068FC02B010BD05
:109E40004C170220B0F90020B0F904309A4208DC27
:109E5000B0F90220B0F906309A42CCBF00200120B0
:109E60007047002070470000F0B585B006460D46EB
:109E7000174605F033FC846A0190A30734D52846C1
:109E8000FFF7E0FF00282FD040F601032340012B0D
:109E90002AD0304605F02CFC02AC0246019029463F
:109EA000204603F047FC2046FFF7CCFFC8B1019BDA
:109EB0009E6A44F22001314003F1080529B1284689
:109EC0002946224604F0F8F90BE094E803003E43EB
:109ED00085E803009E62054B1A8801321A8003F060
:109EE00021FE01A805F012FC05B0F0BD20170220EC
:109EF0002022FFF7B9BFF0B50F4685B015460646DC
:109F000048B305F0F5FB836A04AC9B07024644F8AE
:109F10000C0D03D4204605F0F9FB1CE002A83946DD
:109F200003F008FC0028F5D0204605F0EFFB304692
:109F300002A92A46FFF798FF3046FFF790FB044638
:109F40004CB1204602A92A46FFF7D5FF204605F06E
:109F5000C5FB046AF4E705B0F0BD2DE9FF4180467A
:109F600017461D460C46002930D0084605F0C0FBB8
:109F7000866A0190B307024625D502A8414603F040
:109F8000D9FB00B340F601033340012B07D1019BFD
:109F900002A899691A6A2B46FFF7DFFF04E0204602
:109FA00002A92A46FFF760FF019BDC695CB1BC4255
:109FB00009D0204602A92A46FFF79DFF204605F05A
:109FC0008DFB046AF2E701A805F0A0FB04B0BDE830
:109FD000F08170B5054608460C46164605F07EFB36
:109FE000836A13F4803F2846214632460CBF202363
:109FF0004FF48043BDE87040FFF7AFBF2023FFF769
:10A00000ACBF13B5044605F073FB8169019041B103
:10A01000026AFFF7F3FF2046FFF76AFE019B00226A
:10A020009A6101A805F072FB02B010BD08B106F0FC
:10A0300023BB70471FB504AB019043F8101D694660
:10A0400006F01AFB05B05DF804FB00230B80828844
:10A050004B800388D31A8B80C2884388D31ACB8065
:10A060007047F0B50F4687B00546002833D005F09D
:10A070003FFB866A0190B2072AD503C804ACF303FC
:10A0800084E8030002D52846FFF7B4FE5FB13868C4
:10A09000796802AB03C3019802A9FFF747FE204687
:10A0A00002A903F079FB20462946FFF7A1FD78B10C
:10A0B00040F601033340012B06D1019B20469969EC
:10A0C0001A6AFFF79BFF03E028462146FFF710FFBF
:10A0D00001A805F01BFB07B0F0BD0021FFF7C1BFD1
:10A0E00010B5044605F0FAFA80690028F9D1054B4D
:10A0F0001A68944205D05868844214BF4FF0FF306C
:10A10000012010BD0817022008B5FFF7E9FF00285D
:10A1100003DBBDE8084004F041B808BD0D4A1368F0
:10A1200070B59D6C0446164608B90B4A14689C64C9
:10A130002046FFF7E9FF03F059F9204605F0CEFA73
:10A140003368B0F90010B0F90220D9641A652846C6
:10A1500070BD00BF24010020241702202DE9F74F15
:10A160000C9D9B464B4B0746884692461E6865BB36
:10A17000494B1B8863B3494B1B685A7C484B53F8C7
:10A1800022305A1C24D01BB31D46284605F0B0FAD5
:10A19000B0F90020B0F90230019017449844BAF1A8
:10A1A000000F05D1B0F904A0C2EB0A0A0AF1010AB6
:10A1B000BBF1000F05D1B0F906B0C3EB0B0B0BF1EF
:10A1C000010B01A805F0A2FA02E06B1CDDD100250D
:10A1D0000F982C3005F05EFD0446002856D00D9BEC
:10A1E0001E432D4B1A8801321A8005F081FA0E9B0E
:10A1F00003610DF108092B4B826A49F8080D3340C1
:10A200000780A0F802805744D8441343013F08F167
:10A21000FF3883628780A0F80680684605F076FAEA
:10A22000214B186848B105F059FA0746204605F059
:10A2300055FA7B6943617C6100E01C602946204639
:10A24000FFF704FDB50602D52046FFF767FFF007CC
:10A2500003D5164B1A6801321A60710602D52046E2
:10A2600006F082FBB2070DD5204605F041FA836A5D
:10A27000009043F002038362684605F047FA2046E7
:10A28000FFF72BFF20460121FFF7D4FE204603B045
:10A29000BDE8F08F301702200017022024010020B3
:10A2A000081702209F3F3F0024170220501702206A
:10A2B00073B5044600286ED0FFF78CFD00286AD0E5
:10A2C0002046FFF70DFF0B2105462046FFF7B2FEA3
:10A2D000204606F034FA204605F00AFA0190406A5A
:10A2E00008B101F077FB2D4B2D4A002119602D4B51
:10A2F0001B6852F82300A04208BF42F823102A4AE4
:10A3000052F82310A14204BF002142F82310274B2A
:10A310001B682BB15A68A24204BF00225A60F7E7BB
:10A3200020460721FFF721F8019EF069FFF7C0FFE3
:10A33000F369002BF9D12046FFF763FE1C4B186828
:10A3400050B105F0CBF906464069A042F8D120464D
:10A3500005F0C4F943697361019B9B6ADA0703D571
:10A36000144A1168013911609B0603D5124B1A88F3
:10A37000013A1A8001A805F0C9F9104B1A88204645
:10A38000013A1A8005F0EEF9002D04DB0C4B53F86E
:10A390002500FFF7C3FE02B070BD00BFCCD701207F
:10A3A0001817022028170220441702203C17022009
:10A3B0002417022050170220201702200017022025
:10A3C000081702202DE9FF415D4F3B6893F85400C8
:10A3D000002800F0B2805B4B5A69012A1C4603DD5D
:10A3E000013A5A610020A8E004F108061B6996E8CA
:10A3F0000300013302AD236185E8030023B92388FC
:10A40000ADF80830638811E0A3896289ADF80A20AD
:10A4100001339BB2B4F90420ADF808301BB29A4264
:10A4200006DA2388ADF80830E3890133ADF80A3045
:10A43000BDF90A20B4F90630DFF808819A4204DD3C
:10A440006369013B0020636177E03B68986C05F02D
:10A450004FF9BDF90820B8F9003001909A421CD19B
:10A46000B8F80630ADF80E30B8F80430ADF80C305E
:10A47000334B1B689A6C5AB1104605F02FF9804691
:10A480000022006A2946FFF7C7F9D8F81820F2E73A
:10A49000019B2946D869FFF7BFF9BDF80830ADF830
:10A4A0000C303B689A6C6AB1104605F017F92946E2
:10A4B00080460022006AFFF705FA0028EDD1D8F89F
:10A4C0001820F0E7019B2946D869FFF7FBF900281F
:10A4D000E3D1A388BDF90820ADF80C301BB29A4235
:10A4E00007DD95E8030086E8030001A805F00EF9F2
:10A4F00097E73B689A6C52B1104605F0EFF80746B3
:10A500000022006A2946FFF721FABA69F3E704AF8F
:10A51000294657F80C3DD869FFF718FA384605F078
:10A52000F5F8236944F62062934289DC95E803003C
:10A5300086E80300FFF72AFC012004B0BDE8F081A3
:10A5400024010020B4D701202DE9F041394F3B68A8
:10A5500093F8542086B0064612B9FFF717FC64E062
:10A56000354D6A690132012A6A612C465DDC986CBE
:10A5700005F0BEF84FF0FF322A61304A00901278A1
:10A580002AB100F1080302AA93E8030005E0826AF9
:10A5900012F002080AD003C802AA82E8030002AD42
:10A5A00066B12846314603F0F7F807E06B69684664
:10A5B000013B6B6105F0AAF8404637E03B68204E4E
:10A5C0005A6CC2B1009B10685168019304AB03C37D
:10A5D000336833B101A805F099F8306805F088F8C0
:10A5E0000190019804A9FFF7A1FB284604A903F0F4
:10A5F000D3F801A800E0684605F088F8316819B181
:10A600002846FFF7F5FA28B13B682846996CFFF712
:10A61000EFFA18B96369013B636107E095E803004D
:10A6200084E80300FFF7CEFE00E0012006B0BDE89D
:10A63000F08100BF24010020B4D701202D17022093
:10A640000417022008B503F073FD024B1B680022BB
:10A650005A6408BD24010020F0B589B0044605F015
:10A6600047F80769866A0190083003C802AD85E89B
:10A67000030001A805F04AF8002F31D0B3072FD509
:10A6800020462E21FEF7F4FD164B1A7816F4805F53
:10A6900002F101021A701E460AD00F23059404939A
:10A6A0000795FFF7CFFF204604A905F0E5FF10E06E
:10A6B0002846FFF749FF60B10F23049305940795DF
:10A6C000FFF7C0FF204604A905F0D6FFFFF77AFE8A
:10A6D000F1E733782046013B2F213370FEF7C8FDA8
:10A6E00009B0F0BD2D170220F0B589B006AC03907B
:10A6F00004F0FEFF00F108020346059092E8030013
:10A700009D6A9E691F6984E8030005A804F0FEFFA6
:10A7100044F220032B40002B34D0BFB120460399D4
:10A72000FFF766FA90B10398FFF7F8FC69070FD5B9
:10A7300026B105F0010585F0010500E00125009531
:10A740002046124903AA002300F0DAFA002403E0AD
:10A750000398FFF7DDF90124039804F0C9FF826A2A
:10A76000059022F4804323F02003920448BF43F075
:10A770000403836205A804F0C9FF054B1A88013A57
:10A780001A8000E01C46204609B0F0BD899B0008F5
:10A790002017022008B504F0A1FF836A43F40043A8
:10A7A0008362024B01221A6008BD00BFB0D70120AE
:10A7B0002DE9F04F4C4B1B689FB003B19847002622
:10A7C0004A4D2B68DBB14A4B1C68BCB1204604F0F3
:10A7D0008FFF826A47691EAB12F4004F43F8700D79
:10A7E00007D0184604F092FF2046FFF761FD3C4673
:10A7F000EBE718463C4604F089FFE6E72C603D4B4A
:10A800001B6803B198473C4B1B682BB93B4F3B6817
:10A8100093F8543043B103E098470028F6D058E04D
:10A8200003F01EFD002854D13B6893F854504DB1FD
:10A83000334B1D8835B1334B1B68002B4BD01B6845
:10A84000984701253B6893F8543013B9002D37D150
:10A8500045E0DFF8AC80B8F80030002BF6D0DFF828
:10A86000A890D9F800400CB9214B1C6802A803F04D
:10A87000B5FC3B68D3F830B0D3F834A014B9002449
:10A880000DE063B92046FFF72FFF034620460193F2
:10A8900004F024FF4469019B002CF2D1EFE75846F5
:10A8A000C9F8004003F066FC504603F061FC02A8C2
:10A8B00003F09EFCB8F80030002BC7D00126C1E79A
:10A8C000104B186810B14368984708E002F02AFF5F
:10A8D00005E0012674E7012002F024FFB1E73046CD
:10A8E0001FB0BDE8F08F00BF14170220B0D70120C1
:10A8F00024170220101702209017022024010020A4
:10A900002017022040170220CCD70120024B1B68E1
:10A91000012283F85420704724010020034B1B6858
:10A92000002283F8542002F061BD00BF2401002002
:10A9300010B5044640682368E168172B0FD006DC89
:10A940000E2B0ED0142B14D1FEF7BEFE11E0222BDD
:10A950000CD0282B0DD1BDE81040FFF7BEBBE06046
:10A9600010BD2146BDE8104005F0ACBF6FF070434C
:10A9700000E00023E36010BD03680E2B10B5044611
:10A9800002D00F2B09D020E0C3685A68012A21D1D8
:10A990001868BDE8104003F05BBC0F4A43681168BB
:10A9A0008B4206D05268934214BF4FF0FF3301230D
:10A9B00000E00023094A52F823006FF070439842E8
:10A9C00003D003F0D5FB04F063FA2046BDE8104045
:10A9D000FFF7AEBF10BD00BF0817022034170220DA
:10A9E00030B52B4B187885B01D4600284DD1294B2A
:10A9F0001860294B1860294B1B685864284B188035
:10AA0000284B04461880204604F01EF9C0B14FF0D0
:10AA1000FF3202238DE80C00002043F6FF72224B28
:10AA20000293039013460146FFF798FB1F4B43F830
:10AA300024001F4B6FF0704243F82420FFF74DFBBA
:10AA40000134022CDFD11B4805F086FF1A4805F0BF
:10AA500083FF1A4805F080FF194805F07DFF19486B
:10AA600005F07AFF184805F077FF104B1868FFF7DC
:10AA700055FBFFF74BFF01232B701448144B036069
:10AA800005B0BDE8304004F013BA05B030BD00BFDA
:10AA9000D8D7012024170220CCD701202401002080
:10AAA000201702200017022079A9000808170220A9
:10AAB000341702207418022064180220541802204F
:10AAC0007C1802206C1802205C180220D0D70120CC
:10AAD000A59700082DE9F04F87B0044604F008FE62
:10AAE00006AFB0F800808688B0F80290B0F806B0E3
:10AAF00047F8040D0FFA88F836B2C8EB0606D0F80E
:10AB000024A0013638460FFA89F90FFA8BF504F0C4
:10AB1000FDFDC9EB0505002E05F101054DDD002DFC
:10AB20004BDDBAF1000F4AD0504604F0E1FD06AB10
:10AB3000868843F8080DC58836B2184604F0E6FD4D
:10AB4000464502D12DB24D4532D0504641464A4687
:10AB500000F086F82CE0836A43F480338362384641
:10AB600004F0D4FD404600F093FF0746504603F042
:10AB700003FB404600F0B4F82D4B05FB06F21978B4
:10AB80002C4D2D4E920002F021FD2046D5F800807C
:10AB90003460FEF7CCFC28602046FFF75DFD002006
:10ABA000C5F80080306003F0E7FA384600F070FF27
:10ABB000204604F093FD406A37E0002035E0FEF7C0
:10ABC00077FD844212D102F0A3F8824602F0A8F881
:10ABD000564502DC854209DD00E056468542A8BFA5
:10ABE0000546314620462A4605F014FE134B0193D4
:10ABF0004FF0010A124B02934046494632462B461B
:10AC0000CDF800A000F04EFE8046204604F070FD16
:10AC10000590C0F82480B8F1000F9CD1384604F0AC
:10AC200075FD2046FFF718FD404607B0BDE8F08FE0
:10AC30000C0100205C1702204C17022090BB010879
:10AC400068E6010838B5054605242846FFF742FFA7
:10AC500010B9013CF9D138BDBDE8384006F092BBCF
:10AC600037B50D46144618B9114B1B68186EE8B17C
:10AC700004F03EFDA4B2ADB2C4808580009002F025
:10AC8000B5FB009B586970B104F032FD009B019048
:10AC90001A895B898280C38012B10BB10580448020
:10ACA00001A804F033FD684604F030FD03B030BD68
:10ACB0002401002013B520B9084B1B68186E044608
:10ACC00048B104F015FD02ABB0F90A4043F8040D99
:10ACD000184604F01BFD204602B010BD24010020E0
:10ACE00013B550B104F004FD044602A840F8044D29
:10ACF00004F00CFD04F11800FFE702B010BD0000E5
:10AD00002DE9F04F1E4689B04E4B04921A6803910C
:10AD1000547C4D4A1257012A05469B46204606DDC3
:10AD200001F0E0FF0746204601F0DFFF05E001F0FB
:10AD3000DFFF0746204601F0DEFF044625B306A8E4
:10AD400007A903F0FDFA069BB5F900A0B5F90420A8
:10AD5000B5F902801F44079B2AEAEA7A013F97422D
:10AD6000D4BFCAEB0707CAEB02071C44B5F906209B
:10AD700028EAE878013C9442D4BFC8EB0404C8EB4D
:10AD800002040137013401E0A846AA4606B966422A
:10AD9000002F52DD002C50DD129B0093504641469F
:10ADA0003A46334600F038FE054620B90498039B26
:10ADB0009847012042E0FFF77DFFA042064606D0FB
:10ADC000DBF80030986C10B1322105F041FC2846C8
:10ADD00000F05EFE73420593A1460027B14503DAF9
:10ADE0002846494606F0CEFB47B12846514607EBB8
:10ADF0000802FFF735FF284606F0DAFB039B0498AC
:10AE00009847124B1B680BB100209847284600F06A
:10AE1000B7FE3744059BA7429944DFDB284600F084
:10AE2000D9FD002000F034FEA64206D0DBF8003049
:10AE3000986C10B1332105F00BFC002009B0BDE87F
:10AE4000F08F00BF2401002054170220DCD701201E
:10AE50000248012918BF0020704700BF90BB0108BD
:10AE60000248162918BF0020704700BF951101083D
:10AE700008290CBF20200020704708B50068C3686F
:10AE80001B6A984708BD37B580680C4604F030FC53
:10AE9000034602A89988DA881D8940F8043D5B8939
:10AEA0002180628029441A440139013AA180E2805C
:10AEB00004F02CFC03B030BD0E4B1B6873B5054687
:10AEC000186E0E4604F014FC034602A8B3F90640BF
:10AED00040F8043D03F11801361BDC68B3F9043077
:10AEE00004FB0614ED1A04F011FC04EB8504204663
:10AEF00002B070BD2401002008B508461146FFF7D6
:10AF0000DBFF006808BD0000154B1B6873B5186EA9
:10AF100015460E4604F0ECFB294600903046FFF73C
:10AF2000CBFF009B1B681B6904469B6898472368FE
:10AF30005840009B2060586960B104F0D9FB02AC16
:10AF4000836844F8040D1B6831462A46984720461A
:10AF500004F0DCFB684604F0D9FB02B070BD00BF12
:10AF60002401002073B51C46104B1B68186E0E465A
:10AF7000154604F0BDFB294600903046FFF79CFFC4
:10AF8000009B0460586960B104F0B2FB02AC8368B6
:10AF900044F8040D1B6831462A469847204604F0C1
:10AFA000B5FB684604F0B2FB02B070BD240100207E
:10AFB0002DE9F7432C4D1E462B68186E0F4614469C
:10AFC00004F096FB00904069A94608B104F090FB9C
:10AFD000019021463846FFF76FFFD9F80020009B0B
:10AFE000D16B127CD3F80C80D1F80090D2070546C3
:10AFF0001FD51B681B699B6898478046019828B13C
:10B0000082683946D2F800C02246E0472B6883EABE
:10B0100008032B60009B0134DB68B4421D44EDDD66
:10B02000684604F073FB019BD3B101A804F06EFBEA
:10B0300016E0019B63B10198836822461B6839467C
:10B0400001349847B442C5F800904544F3DDE7E782
:10B05000341B0134013CC5F800904544FAD1DFE7C8
:10B0600003B0BDE8F08300BF240100202DE9F04FBC
:10B07000DFF8ACB01446DBF8002085B0106E0F4648
:10B080001D4604F035FB214602903846FFF714FFB9
:10B09000029ADBF80030D2F80C90DB6B0646506960
:10B0A000D3F800A0ED1B013538B304F021FB0E9A54
:10B0B0000DF11008131B48F8040D013300933946B5
:10B0C00022462B4606F048FA404604F01FFB14E0E7
:10B0D000DBF800301B7CDB0713D5029B1B681B6968
:10B0E0009B68984732462B461168013B81EA000174
:10B0F00042F8041BF8D14E4401340E9B9C42E7DD1C
:10B1000008E0002DF7DD2B463246013B42F804AB48
:10B11000FBD1F0E702A804F0F9FA05B0BDE8F08F22
:10B120002401002007B50092FFF7A0FF03B05DF8EF
:10B1300004FB00002DE9F04F9D4C9A46236891B026
:10B140008046186E07920E46DDF874B01F9D0028E9
:10B1500000F0878304F0CCFA0E90406908B104F047
:10B16000C7FA0F9010A850F8083DDB680A9304F066
:10B17000CDFA1E9F0F983744049750B123681B7C6B
:10B180009C0706D41A9F00970499079A534606F025
:10B19000E3F904980799FFF78FFE1B9F172F0646C8
:10B1A00064DD4FEA8A0706974FF000091A9F0F984F
:10B1B000B94557DA30B18368079A5C6804994A4404
:10B1C0005346A047D8F81030D86828B130465946C1
:10B1D000069A0CF04DFC3EE05B689847000E059027
:10B1E000354657465C463B4622464FF0000C52F827
:10B1F000041B0598090E8142059808BF0CF1010C4B
:10B20000814203F1FF3314D0BCF1000F14D04FEA98
:10B210008C03284621461A460393CDF808C00CF04B
:10B2200027FC039BDDF808C01D441C44CCEB07073A
:10B230000FE0002BDBD1E7E72068020EFF2A05D0E4
:10B24000D2432968D2B202F0C5FA2860043504342A
:10B25000013F002FC7D11C9FBB440A9F09F1010980
:10B260003E44A3E7002840F0F982FAE21B9F102F2A
:10B2700037D1061F00251A9F0F9CBD4280F2A08087
:10B28000079F2F443CB1A3680499D3F804C020461B
:10B290003A465346E047ABF1020306930596D14682
:10B2A0000499D8F81030069A5B6832F8020F0692BB
:10B2B0005144C9EB010103919847059B039943F859
:10B2C000040F059324B1A36820461B683A469847AB
:10B2D000B9F10109E4D11C9FBB440A9F01353E44EA
:10B2E000C9E71B9F082F00F104066DD1079F07993E
:10B2F0001A9A0F9C7B1A9342A6F1040060DA2C4B39
:10B300001B681B7C6DB313F0030305D0022B51D1D6
:10B31000B146DDF810801CE01BF8032055F8222010
:10B3200040F8232001335345F6D143E055F823304C
:10B3300049F8043C2CB1A36820461B6841463A46B4
:10B340009847049B08F101085344434509F1040957
:10B3500030D00498C0EB0B0313F80830002BF0D06A
:10B36000E4E713F0030305D0022B23D1B146DDF847
:10B37000108015E0594652460CF07AFB1AE049F865
:10B38000043C2CB1A36820461B6841463A469847C6
:10B39000049B08F101085344434509F1040909D00D
:10B3A0000499C1EB0B0313F80830002BF0D0E6E74B
:10B3B000240100201C9A0A9B934401371E4496E7FF
:10B3C000002C40F04B824CE21E9FB24B09967F004E
:10B3D0000C971E9FBF000D97079F0597002D08BF74
:10B3E0001D46099F07983C1F059F3B1A1A9FBB42A9
:10B3F00080F232821B9F022F00F0AD80042F00F0FC
:10B400004F81012F40F01E82DFF89092D9F8003072
:10B41000186E04F06DF99BF800309F4A1E99D65CB7
:10B42000D9F800300E901B7CDDF83CC003F003031C
:10B43000022B5746C1F1080846FA01F620D0032B2B
:10B4400061D0012B5FD05A46474538BFB846C8EB9C
:10B4500007074346214606F00100013B55F820004E
:10B4600041F8040B4FEA5606F5D104EB8804002F8F
:10B470006DD012F8013F88494FF00808CE5CE3E731
:10B480006B68DDF810900B93CDF820B0474538BFBE
:10B49000B846C8EB0707BCF1000F26D01EB904EB75
:10B4A0008804C14425E0F0070CD5DCF80830059A83
:10B4B0001B68CDF808C06046494698470B9BDDF8ED
:10B4C00008C02360B8F1010809F1010904F104047E
:10B4D0000FD07608E2E7F10744BF0B9B2360B8F179
:10B4E000010804F1040404D07608002EF3D104EB23
:10B4F000880467B30898684A10F8013F0890D65C42
:10B500004FF00808C2E703681B699B6898475946D3
:10B51000474538BFB846C8EB0707231DC646F207A4
:10B5200004D553F8042C424043F8042CBEF1010E1C
:10B530004FEA560603F10403F1D104EB880437B156
:10B5400011F8013F544A4FF00808D65CE0E70EA816
:10B5500004F0DCF876E11E9F0C9BDDF83CC0C7F1DF
:10B5600004069BF800709F404C4B1B681B7C03F04B
:10B570000303012BF6B2FFB266D008D3022B40F0D2
:10B5800061810498CDF820B0D04606903EE05A463E
:10B5900053469E42C8BFDEB29B1B314620464FEA4F
:10B5A000971C013955F82CC040F804CBBF0011F0AE
:10B5B000FF01FFB2F3D1013EF6B2013604EB86047F
:10B5C000002B00F03F8112F8017F0426E1E7069985
:10B5D00017F0C00F494422D109F101095FFA89F23D
:10B5E000BF009642FFB2F2D1069F013EF6B27B1C2D
:10B5F000721C9E1904EB82040696B8F1000F00F04D
:10B600002181089B13F8017F089304264645C8BF93
:10B610005FFA88F6C6EB08084FF00009D7E7BA09C9
:10B6200055F8222044F82920BCF1000FD4D0DCF8D2
:10B63000082012680B926046CDF808C0059A0B9B53
:10B640009847DDF808C0C7E7584653469E42C8BF32
:10B65000DEB29B1B221DB44617F0C00F05D052F876
:10B66000041C81F0FF0142F8041C0CF1FF3CBF00F8
:10B670001CF0FF0CFFB202F10402EDD1013EF6B264
:10B68000013604EB8604002B00F0DC8010F8017F0B
:10B690000426DBE750BB0108D0E4010824010020A8
:10B6A000714A9BF8003012680D98127C0F9F02F0CF
:10B6B00003028340012ADEB200F09C8002D3022AFA
:10B6C00035D0BFE01E9F5FB136090BF1010255F87E
:10B6D000263023609BF80160099C0AF1FF3301E0EA
:10B6E00053465A46012B1ADD581004F1080103F0A5
:10B6F000010302EB00084FEA161C06F00F0655F88E
:10B700002C7041F8087C55F8266041F8046C12F85A
:10B71000016F424501F10801EDD104EBC004002B9B
:10B7200000F09080360955F8263023608AE01E9894
:10B73000C0B113F0F00F0AD0360955F82630236057
:10B740002FB1BB6804991B68059A3846984704993D
:10B75000099C9BF8016001F101080AF1FF3C0BF123
:10B76000010911E0D446D946DDF810800CE016F04E
:10B77000F00F0DD116F00F061BD119F8016F083428
:10B7800008F10208ACF1020CBCF1010FEFDC21E082
:10B79000330955F823302360002FEBD0BB68059A9E
:10B7A0001B68CDF808C0384641469847DDF808C008
:10B7B000E0E755F826306360002FDED0BB68059ABD
:10B7C0001B68CDF808C0384608F101019847DDF83C
:10B7D00008C0D2E7BCF1000F34D0360932D055F89A
:10B7E0002630236077B3BB68059A1B68384641460C
:10B7F000984727E01E9FC7F10203DBB25F4652461F
:10B800009342C8BFD3B2D21A201D9C4616F0C00F77
:10B8100005D050F8041C81F0FF0140F8041C0CF125
:10B82000FF3C36011CF0FF0CF6B200F10400EDD134
:10B83000013BDBB2013304EB83041AB117F8016F4B
:10B840000223DDE7059B1C9F0133BB4405930A9F40
:10B85000099B3B440993C4E50F9B13B10FA803F068
:10B8600055FF11B0BDE8F08F240100202DE9F34110
:10B870000E469046074603F03BFF036802ACDB68C8
:10B8800044F8040D5B6A00201621984705462046BF
:10B8900003F03CFF1DB1384631464246A84702B08E
:10B8A000BDE8F0812DE9F04F3E4E87B01D4633686C
:10B8B000109F5B7C83468A4690461198129900221D
:10B8C00003F0D4F90446002833D003699B689847F5
:10B8D00001F0CBFA08FB00F60390073604F0D0F82D
:10B8E00017F001094FEAD60604D1042390FBF3F0C8
:10B8F00000EB4000002D09DC1EB11838B0FBF6F05B
:10B9000000E030466D42A842B8BF0546B9F1000FCD
:10B9100009D1CDF800905846514642462B4605F0D5
:10B92000DBFD074600E00027002D04DC204603F085
:10B930009BF9002032E006FB05F01830B9F1000F4A
:10B9400002D004F029F901E004F0A4F9814640B9DD
:10B95000204603F089F9002FEBD0384603F002FFB0
:10B960001BE003F0C5FE034606A8039A40F8043D19
:10B970001A611C60A3F804B0A3F806A0A3F808801D
:10B980005D81DE605F6103F0C1FE064A129B2361A8
:10B990001368C4F808905B7CA361484607B0BDE813
:10B9A000F08F00BF2401002037B5054670B103F0C9
:10B9B0009FFE036802AC1B6944F8040D9B6898471E
:10B9C00001F053FA0546204603F0A0FE284603B0D6
:10B9D00030BD000037B50446D0B10E4B1B681B6E5E
:10B9E000834201D102F0F0FB204603F081FE01907A
:10B9F000406908B105F09CFD02AD55F8043D18689A
:10BA000003F032F9284603F081FE204603F0AAFE37
:10BA100003B030BD240100202DE9FF479A46194BA1
:10BA20000C9D1B680746587C174B53F820408846EE
:10BA30009146E3681B68042B06D02468002CF8D1DB
:10BA400003F002F9044630B1E3682046DB6A0121C5
:10BA50009847064608B9002010E02469A368984773
:10BA6000013004BF45F00105084C02948DE86000E8
:10BA7000384641464A465346FFF714FF04B0BDE836
:10BA8000F08700BF240100208417022068E6010827
:10BA9000114BF7B51A680446166E1F4610B902F02E
:10BAA00093FB16E00EB102F08FFBFEF737FF204646
:10BAB00003F01EFE02AD3B6845F8040D1C660068ED
:10BAC00003F010F9284603F021FE01F079F801F0A7
:10BAD0008DFC304603B0F0BD240100202DE9F04379
:10BAE0000C4685B015460646002841D0002002F0DD
:10BAF0001DFB214B1B6807463046D3F8608003F0DE
:10BB0000F7FD03680190986902F048FB1B4B9C42CB
:10BB1000019B04BFB3F90440B3F906501A895B894D
:10BB2000ADF80840013A013B22442B448146ADF870
:10BB30000C20ADF80E30ADF80A50FEF7E7FE01A874
:10BB400003F0E4FD02A8FEF7FFFC48B9484602F006
:10BB500025FB4046FFF79CFF384602F0E7FA07E076
:10BB6000304621462A4604F083FFFEF72BFCECE723
:10BB700005B0BDE8F08300BF2401002001F0FFFF05
:10BB800001490A46FFF7AABF01F0FFFFF8B50446D6
:10BB90000E46D0F88C302A2115469847E16AD4F831
:10BBA000903031442046C1F30F219847E16AD4F820
:10BBB0009030B7B239442046C9B29847E16AD4F808
:10BBC000903031442046C1F30F219847E16AD4F800
:10BBD000903039442046C9B29847D4F88C3020467A
:10BBE0002B219847216BD4F8903029442046C1F38B
:10BBF0000F219847216BD4F89030AEB231442046E3
:10BC0000C9B29847216BD4F8903029442046C1F33B
:10BC10000F219847216BD4F8903031442046C9B2A7
:10BC20009847D4F88C3020462C219847F8BD2DE950
:10BC3000F041044688461F462A21D0F88C30069DE4
:10BC400016469847E16AD4F8903041442046C1F343
:10BC50000F219847E16AD4F8903041442046C9B298
:10BC60009847E16AD4F8903039442046C1F30F2157
:10BC70009847E16AD4F8903039442046C9B29847D1
:10BC8000D4F88C3020462B219847216BD4F8903083
:10BC900031442046C1F30F219847216BD4F89030EE
:10BCA00031442046C9B29847216BD4F890302944DA
:10BCB0002046C1F30F219847216BD4F890302944D6
:10BCC0002046C9B29847D4F88C3020462C2198479A
:10BCD000BDE8F08113B50D4A0446516810686B4603
:10BCE00003C3D4F88C30204636219847636BA18C6F
:10BCF00002AA134421F0E00113F8083C194320463E
:10BD0000D4F8903089B2984702B010BD54E40108CD
:10BD100013B50446D0F80C312E209847216AD4F888
:10BD20002831684603319847226A00AB13441DF856
:10BD3000022059789878D2088908D20242EA411242
:10BD400042EAD00002B010BD1FB50446D0F82C3135
:10BD50002E209847216AD4F8483168460231984726
:10BD6000236A00A901EB43023DF81300528802F454
:10BD70007C41C2F3C40242EA511200F0F80042EAE8
:10BD8000002004B010BD38B504460D46D0F80C3183
:10BD9000080A9847D4F80C31E8B2984738BD08B57E
:10BDA000D0F82C310846984708BD08B5D0F81031B6
:10BDB000C8B2984708BD08B5D0F830310846984752
:10BDC00008BD0000082902D0102905D07047064B95
:10BDD000C0F88C30054B03E0054BC0F88C30054BA8
:10BDE000C0F89030704700BF87BD0008ABBD0008A9
:10BDF0009FBD0008B7BD0008F0B585B084680A9FF4
:10BE00000097BD1A581A013500FB0555D4F8A870E3
:10BE10000B9E2046B847D4F80C312E209847D4F812
:10BE20002831216A02A89847D4F8283102A80321B2
:10BE300098479DF808309DF80920DB089208DB023E
:10BE400043EA42139DF80A20013D43EAD20326F853
:10BE5000023BE9D105B0F0BDF0B587B084680C9F16
:10BE60000097BD1A581A013500FB0555D4F8A87083
:10BE70000D9E2046B847D4F82C312E209847D4F890
:10BE80004831216A02A89847D4F8483102A8022113
:10BE90009847BDF80A3003F47C42C3F3C40343EA75
:10BEA0005213BDF8082002F0F80243EA0223013DD4
:10BEB00026F8023BE8D107B0F0BD000010B50446FB
:10BEC00000F0A6FDA368124AC3F8AC20114AC3F8DB
:10BED000A820114AC3F8B020104AC3F8B8200022A5
:10BEE000C3F8BC20C3F8CC200D4A0E491268C3F831
:10BEF000C420DA8C0968C3F8B41022F003020A499E
:10BF0000DA840A4AC3F8C810C3F8942010BD00BFF1
:10BF10008DBB00082FBC0008D5BC000811BD00086F
:10BF20001401002010010020F9BD0008C5BD000863
:10BF300008B5D0F8B430984708BD08B5D0F830310E
:10BF400088B2984708BD00002DE9F04F3D4F846846
:10BF500082463868007C10F0010F85B00E46154609
:10BF60009846C1EB030945D04FEA490B0E9885422C
:10BF700065DCD4F8C4C0E76EBCF1000F01D1B44653
:10BF800007E08DE8A000504631462A464346E04788
:10BF900011E0C4450EDCD4F8EC30CDF80CC061469D
:10BFA00050462A469847DDF80CC027F8020B0CF1E2
:10BFB000010CEEE7E76EBB1E09F1010C5F44BB42CA
:10BFC00005D0A26A59884A4023F8022FF7E7009566
:10BFD0002A46D4F8A870CDF80CC020463146434616
:10BFE000B847DDF80CC0D4F83831E06E61469847A8
:10BFF0000135BBE70E980090851AD4F8A86020465A
:10C00000B0473B68A76EDB6B09F10109D3F80080EC
:10C0100005FB0995012395B1FA2D34BF2E46FA266A
:10C020002BB138461FFA88F1324601F0A1FAD4F854
:10C030003831384631469847AD1B0023EBE705B051
:10C04000BDE8F08F240100202DE9F04F8DB0856808
:10C05000179F05937B1E012B099008910A920B955F
:10C0600003D9042F01D0082F06D18F4B1B681B7CEE
:10C0700003F00303022B10D00A9A169F1A9D089909
:10C08000059B3A442944013A0B9D00920B44D5F894
:10C09000A8400A9A2846013BA047DDF828B00A9F2D
:10C0A000169DC7EB0B03AB4280F25182179F7B1E9C
:10C0B0000F2B00F24582DFE813F01000B7004302B7
:10C0C0004001430243024302D701430243024302B9
:10C0D00043024302430243023D02734B099D1B6826
:10C0E000AC681B9D1B7C2F686D680795DDF820A050
:10C0F0001A9D03F00303022BAA441BD0032B6ED01E
:10C10000012B6CD0059EDDF8648098F80010D4F8FF
:10C11000303180222A41114216BF0799B8B288B245
:10C1200001359847082D04BF08F101080025013E9C
:10C13000EBD105E2199D0695D4F86C90DDF8688086
:10C14000CDF80CA0002556462B46069F4FF0800CDC
:10C150003A784CFA08FC12EA0C0C0BD013B9D4F85C
:10C160006C900396079FA9F80070013509F1020948
:10C17000012317E0012B14D1CDF800B0CDF810C089
:10C1800020460399D4F8A8705A46731EB847D4F8CD
:10C190003831E06E29469847DDF810C065466346A1
:10C1A00000E0634608F10108B8F1080F06F1010646
:10C1B00004D1069F013706974FF00008059A5244B4
:10C1C000B242C2D1059F7B1E5344002D00F0B881BE
:10C1D000CDF800B0D4F8A860039920463DE1DDF821
:10C1E00014801A9E199DDDF814902A78802333411B
:10C1F000D1441A42C8EB09090DD0D4F8EC300998A3
:10C2000049465A469847A36AD4F8F07043404946D5
:10C2100009985A46B8470136082E04BF0135002652
:10C22000B8F10108DFD18BE1099D1B9FAC68002F9D
:10C2300000F086811C4B199D1B6895F800A01B7CA3
:10C2400013F0030311D0022B40F07A811A9DDDF820
:10C250002090E76E0397A944A846199D07950025ED
:10C26000CDF818904E462B4640E01A9D059E199F2A
:10C27000C5F103035B00C3F10602C02141FA02F2DB
:10C2800002EA0A02DA401B99D4F8303131F8220070
:10C2900001359847042D03D197F801A000250137F7
:10C2A000013EE5D14CE100BF2401002013B9E76E47
:10C2B000039706961B9F57F82C30039F3B8002374D
:10C2C00001350397012308F10108B8F1040F06F1C5
:10C2D000010606D1079F97F801A0013707974FF095
:10C2E0000008059A4A44B24200F0AC80C8F103024B
:10C2F0005200C2F106014FF0C00C4CFA01FC0CEAEE
:10C300000A0C3CFA02FCD1D1012B14D1CDF800B0BB
:10C31000CDF810C020460699D4F8A8705A46731E6E
:10C32000B847D4F83831E06E29469847DDF810C098
:10C3300065466346C7E76346C5E7099D1B9FAC6832
:10C34000002F00F0FD80834B199D1B6895F800A01D
:10C350001B7C13F0030311D0022B40F0F1801A9DD7
:10C36000DDF82090E76E0397A944A846199D07952C
:10C370000025CDF818904E462B463CE01A9D059EB0
:10C38000199FC5F101039B00C3F10402F02141FA9A
:10C3900002F202EA0A02DA401B99D4F8303131F88D
:10C3A000220001359847022D03D197F801A00025FE
:10C3B0000137013EE5D1C3E013B9E76E0397069656
:10C3C0001B9F57F82C30039F3B80023701350397A2
:10C3D000012308F10108B8F1020F06F1010606D1A8
:10C3E000079F97F801A0013707974FF00008059ABB
:10C3F0004A44B24226D0C8F101029200C2F10401BF
:10C400004FF0F00C4CFA01FC0CEA0A0C3CFA02FC6E
:10C41000D2D1012B14D1CDF800B0CDF810C02046F8
:10C420000699D4F8A8705A46731EB847D4F8383124
:10C43000E06E29469847DDF810C065466346C8E7B8
:10C440006346C6E7059F7B1E4B44002D78D0CDF890
:10C4500000B0D4F8A860069920465A46B047D4F8F0
:10C460003831E06E29466AE0099D1B9FAC68002FB9
:10C4700066D0384B1B681B7C13F0030309D0022BDA
:10C480005ED1DDF82090D4F86C8000264F4633460C
:10C4900022E0199D199B059F3B445B1B002B4FDD40
:10C4A00015F8012B1B9FD4F8303137F8220098473C
:10C4B000F0E713B9D4F86C80B9461B9D55F82A30C3
:10C4C000A8F80030013608F102080123089A059DFA
:10C4D00001372A44BA421CD0199D08982A1A12F82A
:10C4E00007A0BAF1000FE4D1012B10D1CDF800B0B4
:10C4F000204649465A467B1ED4F8A850A847D4F88F
:10C500003831E06E3146984756465346DEE753468B
:10C51000DCE7089F6B1E3B4496B1CDF800B0204687
:10C520004946D4F8A8505A46A847D4F83831E06EA6
:10C53000314604E00B9D1998D5F838310599984794
:10C54000199F189D2F4419970BF1010BA7E50DB00A
:10C55000BDE8F08F2401002010B5044600F058FA21
:10C56000A468104BC4F8E4300F4BC4F8E8300F4B0C
:10C57000C4F8EC300E4BC4F8F0300E4BC4F8A030C9
:10C580000D4BC4F8A430D4F8C430C4F8FC302046B5
:10C59000D4F89430102198471023A363074B6364A9
:10C5A00010BD00BF49C0000849BF00085FC90008AE
:10C5B000CFC8000831BF00083BBF0008F4E60108FF
:10C5C000084670470068401A0138704708467047AF
:10C5D0000068401A01387047104670474068801A5A
:10C5E00001387047104670474068801A013870471C
:10C5F00010467047104670474068801A01387047EF
:10C600004068801A013870470846704708467047EE
:10C610000068401A013870470068401A01387047B6
:10C6200010B58468D4F8F040A04710BD08B5836801
:10C63000D3F8EC30984708BDF7B504460F461646C8
:10C640008568FFF7F3FF0190DDF804E0AB6A204650
:10C65000394632468EEA0303FFF7E2FF03B0F0BD2E
:10C6600013B584680092D4F8E840A04702B010BD2A
:10C6700013B584680093D4F8E8400B46A04702B095
:10C6800010BD37B5069C85680094D5F8E840A047F2
:10C6900003B030BD30B587B085680A9C00940B9C10
:10C6A00001940C9C02940D9C03940E9C04940F9C8A
:10C6B0000594D5F8E440A04707B030BD70470000AE
:10C6C00073B5079E84680C4D76B1286888B90698C2
:10C6D0000090D4F8A8602046B047D4F8A8302B606A
:10C6E000064BC4F8A83004E02B6813B1C4F8A83096
:10C6F0002E6002B070BD00BFE0D70120BDC60008AB
:10C7000008B5026CD0F8D4309069984708BD08B5D8
:10C71000026CD0F8D8309069984708BD2DE9F743EE
:10C720000A9D8468009517462046D4F8A86099466B
:10C730008846ED1BB047216CD4F8DC3088690B9932
:10C74000C8EB09086A1C08FB0222984703B0BDE841
:10C75000F0832DE9F7430A9D84680095174620462B
:10C76000D4F8A86099468846ED1BB047216CD4F8F0
:10C77000E03088690B99C8EB09086A1C08FB0222A3
:10C78000984703B0BDE8F0830139172924D8DFE8C2
:10C7900001F01023232323232323230C250E152309
:10C7A000232323232323231F1A210D4870470D48D9
:10C7B000704703689B68D3F8FC00704703689B6868
:10C7C000D3F8F400704703689B68D3F8F80070470B
:10C7D0000548704705487047002070470448704777
:10C7E0003FCB0008E1CA000845CA0008C1C60008DE
:10C7F0002BCB0008013980680D2923D8DFE801F030
:10C80000090B0D0F2222221107252513181D0020C8
:10C810007047006870474068704780687047C0681C
:10C820007047806B704788B1406B00F00100704723
:10C8300060B1406BC0F34000704738B1406BC0F34B
:10C84000800070474FF0FF307047012070478368C9
:10C8500001290CBF586C00207047836800220A80B1
:10C860004A801A685B68013A013B8A80CB80704736
:10C87000F0B5104D2E4607460FCE91B06C460FC452
:10C8800096E80F00203584E80F000FCD08AC0FC4E8
:10C8900095E80F0084E80F007B6B10AA02EB83037E
:10C8A00053F8402CC7F8002153F8203CC7F8043156
:10C8B00011B0F0BD5CE4010807B580698DE80600A1
:10C8C00003216A46F3F720FF03B05DF804FB2DE96E
:10C8D000F74384689846E38C9B078946174632D510
:10C8E000D4F8003120469847D4F8045106463A4619
:10C8F00020464946A8472369A2699E42ACBF00234F
:10C9000001239642D4BF1A4643F00102636998425C
:10C91000ACBF134642F00103054613B9E3699842E0
:10C920000ADD62682368013A00920021D4F8A870F9
:10C9300020460A46013BB847D4F8AC702046314641
:10C940002A46B84703E0D4F8AC502046A847D4F8AC
:10C95000A43020464146984703B0BDE8F083F7B5C0
:10C960008468E38C9B070F46164645D5D4F8003102
:10C9700020469847D4F804313246054639462046C9
:10C980009847D4F8983006461BB120460121002272
:10C9900098472369A2699D42ACBF002301239542B9
:10C9A000D4BF1A4643F0010263699E42ACBF1346EE
:10C9B00042F0010313B9E3699E420ADD626823680D
:10C9C000013A00920021D4F8A87020460A46013BA3
:10C9D000B8472946D4F8AC30204632469847D4F8B8
:10C9E000A03020469847D4F8983005466BB12046D1
:10C9F00000210122984708E0D4F8AC30204698473F
:10CA0000D4F8A030204698470546284603B0F0BD2C
:10CA100038B58568044695B94FF4BA7002F0C0FF86
:10CA20004FF4BA72A060294600F0D0FDA36802223C
:10CA3000DA8401221A62024A1C64C3F8082138BD54
:10CA400071C8000870B506460D461446FFF7E0FFB2
:10CA5000B368002B3BD0262D02D0272D16D070BDF9
:10CA60009A6B102A02D0122A08D070BD184AC3F857
:10CA7000D440C3F8B820C3F8B42070BD154AC3F839
:10CA8000D840C3F8BC20C3F8C02070BD9A6B102AF0
:10CA900002D0122A0ED070BD3CB10F4AC3F8DC4060
:10CAA000C3F8C820C3F8C42070BDC3F8C840C3F899
:10CAB000C44070BD3CB1094AC3F8E040C3F8CC2083
:10CAC000C3F8D02070BDC3F8CC40C3F8D04070BDCF
:10CAD00001C700080FC700081DC7000853C700089A
:10CAE00038B50546FFF794FFAC684FF4FA7002F0D2
:10CAF00057FFA36BA0660733D8102368584302F092
:10CB00004FFF01210022E066A869F3F7FDFDD4F88C
:10CB100008310546204698472046D4F8B03098475B
:10CB2000002DD4BF0020012038BD70B504460D464D
:10CB30001646FFF76DFFA36883E8600070BD70B50F
:10CB400004460D461646FFF763FFA3689D60DE604E
:10CB500070BD38B505460C46FFF75AFFAB68226832
:10CB6000DA6262681A63A2685A63520707D593E8CB
:10CB700006001A605960DA689968D9609A60A289DB
:10CB80009A84226912B122EAE2721A6238BD2DE952
:10CB9000F04104461F4616468846FFF739FFA56850
:10CBA0004146682205F586700AF062FF2046B047CC
:10CBB0002046B84723699B689847A862BDE8F08182
:10CBC00010B5074C2368186B00F06AFC00F088FC75
:10CBD0002368586B00F064FCBDE8104000F09CBC7A
:10CBE0002401002037B5094C23685A7C084B0546C0
:10CBF00053F82200C2686946126B904720682946A4
:10CC00006A46083000F096FD03B030BD24010020D4
:10CC10008417022037B50D46144602F015F801902E
:10CC200008B901200CE0C3680A215B6A01A8984793
:10CC300003460028F5D0019829462246984700204F
:10CC400003B030BD37B50D46144601F0FDFF01902D
:10CC500008B901200CE0C3680B215B6A01A8984762
:10CC600003460028F5D0019829462246984700201F
:10CC700003B030BD37B50D46144601F0E5FF019015
:10CC800008B901200CE0C36810215B6A01A898472D
:10CC900003460028F5D001982946224698470020EF
:10CCA00003B030BD012810B50C4608DC01F0CCFF04
:10CCB00020B1C36821469B6A984710BD10BD002073
:10CCC00010BD38B5044621460120FFF7EBFF214691
:10CCD00005460020FFF7E6FFA842B8BF284620EA35
:10CCE000E07038BD0121FFF7DDBF0221FFF7DABF99
:10CCF0000321FFF7D7BF0421FFF7D4BF0821FFF7B7
:10CD0000D1BF0921FFF7CEBF0E21FFF7CBBF000037
:10CD1000024B1B68587CFFF7E5BF00BF24010020D1
:10CD2000024B1B68587CFFF7E0BF00BF24010020C6
:10CD3000024B1B68587CFFF7E4BF00BF24010020B2
:10CD4000024B1B68587CFFF7DFBF00BF24010020A7
:10CD500008B5044B53F82000C36808219B6A984724
:10CD600008BD00BF8417022008B501F06DFF20B197
:10CD7000C3680221DB6A984708BD08BD024B1B68E7
:10CD8000587CFFF7F1BF00BF24010020024B53F88D
:10CD900020301B695868704784170220024B53F8F3
:10CDA00020301B6918687047841702200120FFF7A4
:10CDB00088BF0220FFF785BF0320FFF782BF000076
:10CDC000024B1860024B1960704700BFE8D7012082
:10CDD000E4D70120014B1868704700BFE8D7012055
:10CDE000014B1868704700BFE4D7012000283BD0F2
:10CDF00030F0010329D030F0030328D030F00703CE
:10CE000027D030F00F0326D030F01F0325D030F0AC
:10CE1000FF0324D020F4FF7323F001030BB320F4AD
:10CE20007F6323F00F03E3B120F4FF4323F07F037C
:10CE3000BBB1030C1B04A3B1830C9B049BB110F08A
:10CE40007F4F0CBF18202020704701207047022020
:10CE50007047032070470420704705207047082062
:10CE60007047102070471220704708B5FFF7BEFFCB
:10CE700001280FD0831E062B09D9A0F10903072B27
:10CE800007D91138102834BF2020002008BD082001
:10CE900008BD102008BD000070B5084B1B681A7C47
:10CEA00080EA0201490705D59C6BD96B26680D689D
:10CEB00025600E601874104670BD00BF240100206C
:10CEC00008B5024B1B689B68984708BD18010020F5
:10CED00038B5144B1B680A46B3F90A108A42044657
:10CEE0001EDBB3F90E108A421ADCB3F9081088422F
:10CEF00016DBB3F90C10884212DC197C587C11F057
:10CF0000010F094951F8200004D0C3682146DB69AC
:10CF1000984738BDC168DB6B8D691B682146A847FF
:10CF200038BD00BF240100208417022038B5104B03
:10CF30001C68B4F90A3099420D4617DBB4F90E307B
:10CF4000994213DCB4F90810B4F90C308842A8BF38
:10CF500001469A42B8BF13468B4207DB607C054A04
:10CF600052F82000C26894682A46A04738BD00BF26
:10CF7000240100208417022038B5104B1C68B4F936
:10CF8000083005469D42104617DBB4F90C309D422F
:10CF900013DCB4F90A20B4F90E309142A8BF0A4656
:10CFA0009842B8BF0346934207DB607C044951F8BE
:10CFB0002000C168CC682946A04738BD2401002064
:10CFC0008417022073B50E4612490C68B4F9081094
:10CFD000B4F90C508842A8BF0146AA42B8BF154612
:10CFE0008D4214DBB4F90A20B4F90E009642A8BFB2
:10CFF00032468342A8BF0346934208DB647C06485E
:10D0000050F82400C468009324692B46A04702B05E
:10D0100070BD00BF24010020841702202DE9F04FCD
:10D02000DFF8ACC18FB0DCF800C009900E461546A1
:10D030009B461C9CDDF87880BCF1000F0DD0189D3C
:10D04000199E009501961A9F1B9D1D9E02970395A0
:10D0500004940596DCF8004053E0189F199847EABD
:10D060000003012B4FD1584B1868B0F90A20511A10
:10D07000002908DDC1EB0B03002B40F3A2801B9FAE
:10D0800007FB014401E05B4632465E44B0F90E10F6
:10D09000013E761A002E03DD9B1B002B40F391808E
:10D0A0000999B0F90C6029440139891B099E0029AE
:10D0B000C8BFC1EB0505C8EB0601B0F90860B14275
:10D0C0000CDAC1EB060C08EB0C078E1B2CF0070CDE
:10D0D000354404EBE704614407F00708002D70DDD8
:10D0E000467C3A481A9F50F82600C6680197039478
:10D0F0001B9F1D9C00930297CDF8108005947468C7
:10D100002B46A0475DE01A9FC7F108070C976746BA
:10D11000DC4556DA2C4B19981B683044B3F90A20C9
:10D120000A90411E91420B9145DBB3F90E309E42AD
:10D1300041DC4FF00008DDF824900894C246AA456F
:10D1400039DAB8F1000F05D1089A17780132089240
:10D150004FF008080C981A991B4A47FA00F3C1EBE4
:10D1600008088F4013F0FF01FFB203D11068007C64
:10D1700080071BD41268D26B10680D901D9810B1F7
:10D1800050F8213000E0DBB2189913604A1E4A447F
:10D190000B9BCDF81CC048463146FFF713FF0A4BE6
:10D1A0000D9A1B68DDF81CC0DB6B1A60189B0AF136
:10D1B000010A9944C3E71B9E0CF1010C34440A9EFA
:10D1C000A6E70FB0BDE8F08F2401002084170220ED
:10D1D000581702202DE9F04FDFF80CC291B0DCF8AF
:10D1E00000900792054688469B461C9E1E9CB9F1FE
:10D1F000000F0CD01A9D1B9F009501971D9D1F9F2E
:10D200000296039504940597D9F8004081E01A9F8F
:10D210001B9847EA0003012B7DD1714B1868B0F9C8
:10D220000A20531A002B08DDC3EB0B01002940F341
:10D23000D4801D9F07FB034401E059464246D84471
:10D24000B0F90E3008F1FF38C3EB0808B8F1000F51
:10D2500004DDC8EB0101002940F3BF80079BB0F952
:10D260000CC02B44013BCCEB0303002B02DD079FDA
:10D27000FF1A0797B0F908C0654533DA079FC5EB79
:10D280000C03FF1A082E079727D00DDC022E14D0AE
:10D29000042E1AD0012E26D123F0070C04EBE30450
:10D2A000654403F007031EE0182E18D0202E16D078
:10D2B000102E18D104EB430413E023F0030C04EB0D
:10D2C000A304654403F003030DE023F0010C04EB19
:10D2D0006304654403F0010305E01C4401E004EB32
:10D2E000830465460023079F002F76DD90F811E048
:10D2F0003C481D9F50F82E00D0F80CE003948DE8B8
:10D3000042001F9C049302970594DEF80440079B9B
:10D310002946A04761E0C6F108070E97CDF828908E
:10D320000A9F5F4559DA2E4B1B9F1B684744B3F990
:10D330000A200C97013F97420D9746DBB3F90E3058
:10D34000984542DC4FF0000A0B94AC4657460798CC
:10D3500087423ADABAF1000F06D10B9890F80090A4
:10D3600001300B904FF0080A0E991D4A49FA01F35B
:10D3700013F0FF0109FA06F95FFA89F9C6EB0A0A08
:10D3800003D11068007C80071BD41268D26B106830
:10D390000F901F9810B150F8213000E0DBB21A99BD
:10D3A00013604A1E624460460D9BCDF820C0414682
:10D3B000FFF708FE0A4B0F9A1B68DDF820C0DB6BF5
:10D3C0001A601A9B01379C44C1E70A9FDDF8308040
:10D3D00001370A971D9F3C44A2E711B0BDE8F08FCA
:10D3E00024010020841702205817022008B5054B9D
:10D3F0001968054B4A7C53F82200C36808311B6B3F
:10D40000984708BD240100208417022037B5FFF794
:10D41000EDFF04F02DFF044600283DD105462846C7
:10D4200001F012FC019048B1C3680C215B6A01A8AD
:10D430009847034670B30198984704430135022D7D
:10D44000EDD14CBB04F030FF0124204601F0FCFB81
:10D450000190D0B1204600F0A1FE0420FFF730FD7E
:10D4600043F6FF72002001461346FFF7ABFD002094
:10D47000FFF726FD02A80E2150F8043DDB685B6A29
:10D480009847034608B10198984714F1FF34DCD25D
:10D49000002002E0012000E0204603B030BD000083
:10D4A00008B5054B1B685A7C044B53F822301B69A6
:10D4B0001B68984708BD00BF240100208417022084
:10D4C00008B5054B1B685A7C044B53F822301B6986
:10D4D0005B68984708BD00BF240100208417022024
:10D4E000044B1B681A7C52074CBF9B6BDB6B1860AC
:10D4F000704700BF2401002008B5064B1B68196B5C
:10D50000814206D01863FFF7CBFFBDE80840FFF764
:10D51000E7BF08BD24010020044B1B681A7C52079A
:10D520004CBFDB6B9B6B1860704700BF2401002071
:10D5300008B5064B1B68596B814206D05863FFF74C
:10D54000AFFFBDE80840FFF7E7BF08BD240100209A
:10D5500008B5024B1B685B68984708BD180100209E
:10D5600008B5024B1B681B68984708BD18010020CE
:10D5700070B5840702D50180013A023055082B4668
:10D5800005B3032D01EB014402DC06461D4612E003
:10D5900003462E46043E032E1C605C609C60DC60EB
:10D5A00003F11003F6DC043DAB085E1C00EB061033
:10D5B000A5EB8303E9E71DB146F8044B013DFAE70B
:10D5C00000EB8300D30748BF018070BD70B52AB15E
:10D5D000830703D000F8011B013AF8E7930801D153
:10D5E000024417E04FF0013402F003024C43032BD6
:10D5F000054606DD046044608460C460043B10306E
:10D60000F5E71E461BB145F8044B013BFAE700EB7A
:10D610008600E5E7904202D000F8011BFAE770BDF2
:10D620000B8892B2134403808B889B1A83804B88AB
:10D6300013444380CB889A1AC28070470128F7B5FB
:10D6400004460D4665DC344B1B6803B19847012D39
:10D6500004D0022D21D0002D5BD135E02F4E56F89D
:10D660002470B7B9204601F0EFFA0190002850D09D
:10D67000C3680D215B6A01A898470346002848D07B
:10D6800001982946984756F82430013346F824304B
:10D6900018E0013746F824703BE0204601F0D4FA48
:10D6A0000190002835D0C3680D215B6A01A8984716
:10D6B000044600282DD01A4B1B6803B198470198E7
:10D6C0000221A047002025E0144D55F82430012BFD
:10D6D00001D0012015E0204601F0B6FA01900028A3
:10D6E000F7D0C3680D215B6A01A898470646002859
:10D6F000EFD00B4B1B6803B1984701980021B0474E
:10D70000002055F82430002B18BF013B45F8243089
:10D7100000E0012003B0F0BDF8D70120F0D70120D0
:10D72000ECD70120024B1B680146587CFFF786BFEF
:10D730002401002070B5B2F90030B1F90040B1F910
:10D740000250B1F90460B1F906109C42B8BF1C4602
:10D75000B2F902309D42A8BF2B46B2F90450B2F98B
:10D760000620AE42B8BF3546A4B2ADB29142B8BFB2
:10D770000A460480858024B22DB29BB292B2A542A3
:10D780004380C28006DB10B21BB29842B4BF0020B7
:10D79000012070BD002070BD0B8810B5B0F90040AD
:10D7A0001AB29442B8BF03804B88B0F902401AB253
:10D7B0009442B8BF43808B88B0F904401AB29442B7
:10D7C000C8BF8380CB88B0F906101AB29142C8BF97
:10D7D000C38010BD01F07F43B3F17F4FF0B527D078
:10D7E000D343DBB2CDB2C6B25D4302FB065501F4B2
:10D7F0007F4600F47F445E4302FB046601F47F042D
:10D8000000F47F075C43090E000E02FB07444B4304
:10D81000360A02FB0032240AC5F3072306F47F40D0
:10D820001843120404F47F03184302F07F421043AC
:10D83000F0BD000070B50A4C0A4D20680A4E01F098
:10D8400043FF286801F040FF306801F03DFF074AC0
:10D8500000231360064A33602B602360136070BDA1
:10D8600000D80120FCD7012004D8012008D80120CD
:10D8700018D801202DE9F8431C46284B17461A6892
:10D880000646884632B9012225481A60254B0360B6
:10D8900001F00EFB244D2B6833B9244B1B682B6021
:10D8A00013B9FFF789FA28600CB12B68236096B191
:10D8B0001F4B1A68994600244AB92868800002F074
:10D8C0006FF8D0F10104C9F8000038BF0024D9F87E
:10D8D0000030336000E03446B8F1000F0DD0154E33
:10D8E00033683BB92868800002F05AF8002830609D
:10D8F00008BF01243368C8F8003067B10E4E3368A2
:10D900003BB92868800002F04BF80028306008BF5F
:10D91000012433683B602046BDE8F88318D8012015
:10D9200010D8012035D8000808D801208C17022013
:10D9300000D80120FCD7012004D801202DE9F04FA8
:10D9400093B000241D9E0B900C9190461F463460AE
:10D950000FA810A9224611ABFFF78CFF054600283F
:10D9600040F0C380634C119A2368587C624B53F893
:10D97000203007939742A8BF17461A690D920A975D
:10D98000FFF7E6F923680890587CFFF7FFF95B4B37
:10D990000490984205D05A4BC31A18BF012306932E
:10D9A00000E0069500250A9CAB4643461C9A53F8B6
:10D9B000040B05939047030E8146099300F0858080
:10D9C000BBF1000F3FD14B4B0B9F1B680A9AB3F979
:10D9D0000830DDF82CC00C992F44BB42C8BFC7EB00
:10D9E000030B0BEB050AC8BF1F460F9B4FEA8A0AC1
:10D9F000534494440093079B01930CF1FF32384643
:10DA00000B46CDF80CC004F0F9FB089A0F98DDF82E
:10DA10000CC0172A06DC5044CBEB04010D9B04F02C
:10DA200093FC01E0069B13B94FF0010B0BE0C7EB31
:10DA30000C078244DAF80000049A9047013F4AF844
:10DA4000040BF7D1F0E72F4B0F99D3F800C0109FCC
:10DA50004FEA850ABCF1000F24D007EB0A025144BB
:10DA6000109223460F914046E0470F9D109A0023E5
:10DA700058F8031001F07F40B0F17F4FE85801D112
:10DA8000D05005E000F07F40B0F17F4F08BFD1508B
:10DA9000013C03F10403EBD13368109743F0010319
:10DAA000336020E0099BFF2B04D151F80A3047F87E
:10DAB0000A3011E0099B51F80A10DA434846D2B205
:10DAC000FFF788FE47F80A0002E0109B43F82500A4
:10DAD000336843F001033360013C05F1010502D0D6
:10DAE000DDF8148061E7109800E0204613B0BDE82F
:10DAF000F08F00BF240100208417022047FE000899
:10DB000045FE00080CD801201FB508B103AA00E0AB
:10DB1000024601A802A90023FFF7ACFE05B05DF89C
:10DB200004FB000008B5024B1B6803B1984708BD11
:10DB30001CD80120B5EEC00AF1EE10FADFED0D7A27
:10DB400048BFB1EE400A30EE270A0020B5EE400A89
:10DB5000F1EE10FA0CD0F2EE047A20EE270A013032
:10DB6000FCEEC07AC0B217EE903A002BF3D07047AB
:10DB7000704700BF5F708930B5EEC00AF1EE10FA51
:10DB800008B5F6EE007A0AD570EE677A17EE900ABD
:10DB900008F076FB41EC100B07F00EFB09E070EE8D
:10DBA000277A17EE900A08F06BFB41EC100B07F098
:10DBB00083FB51EC100B08F043FC00EE100A08BD8B
:10DBC0000E4B53F8213007EE903AF8EE677A70B5B5
:10DBD00020EE270A05460C461646FFF7CDFFBDEEA0
:10DBE000C00A294610EE100A22461EB1BDE8704058
:10DBF00000F0AEB8BDE8704000F09DB828E601081E
:10DC000038B5B5EE400AF1EE10FA2DED028B044660
:10DC1000B0EE408A0D4652D0B5EEC00AF1EE10FAD1
:10DC200024DBF7EE008AB4EEE80AF1EE10FA1DD517
:10DC3000FFF780FFA04202DC78EE287A46E0F6EE9D
:10DC4000007AB4EEE78AF1EE10FA09DBDFED367AFE
:10DC5000002C18BFF0EE687A08BFB0EE688A35E095
:10DC600044B3F0EE687A9FED308A2FE0B5EEC08ABB
:10DC7000F1EE10FA28D5FFEE008AB4EEE88AF1EE54
:10DC800010FA21DDB0EE480AFFF754FFA04204DC91
:10DC9000F7EE007A78EE677A18E0FEEE007AB4EEDE
:10DCA000E78AF1EE10FA03D84CB9B0EE688A0BE0BF
:10DCB00044B104E0DFED1C7AB0EE678A06E0F7EECF
:10DCC000007A03E09FED188AF0EE487A174B53F87C
:10DCD000243000EE103AB8EE400A27EE800AFFF733
:10DCE0004BFFBDEEC00A10EE100A01F061FF012DDE
:10DCF000C4EB000020EAE07005D1B5EEC08AF1EE79
:10DD000010FAC8BF0130B0EE480ABDEC028B002CFF
:10DD10000CBF2346631C184421462A46C0B2BDE806
:10DD20003840FFF74DBF00BF0000000028E60108A3
:10DD30000021FFF765BF1FB504AB01AC43F8104DE0
:10DD40006B4601F059FF204600F0FAFE04B010BD0A
:10DD5000F0B585B004AC0D4601AE6946174644F8EF
:10DD6000106D01F03DFF0028C4BF05F1FF35EDB295
:10DD700029463A466B4601F03FFF304600F0E0FE90
:10DD800005B0F0BD034A00231360034A1360034A41
:10DD90001360704720D8012024D8012030D80120FA
:10DDA0002DE9F043194B1F6885B000259846D8F837
:10DDB0000030164C33B300F091F90646206801F0AC
:10DDC00097FC034604A8596940F8103D891B0029B7
:10DDD00013DC21680391019619695E680291684617
:10DDE0002660D3F8009001F091FC01A8C8474EB11D
:10DDF0002368BB4205D00125D9E7684601F086FCBF
:10DE000000E00025284605B0BDE8F08324D80120B5
:10DE1000F0B5254C85B0054601F06AFC23680190F9
:10DE200013B92560436039E0184601F061FC04AB8A
:10DE3000466943F8100D684601F068FC019B5A6979
:10DE4000921B002A03DC22685A60256026E02668BF
:10DE5000304601F04DFC04AC466844F8080DBEB1F4
:10DE6000304601F045FC04AB476943F8040D184601
:10DE700001F04CFC019A5369DB1B002B029B02DC76
:10DE800056605D6007E020465E6801F03FFCDFE71A
:10DE9000019B5E604560204601F038FC01A801F05E
:10DEA00035FC05B0F0BD00BF24D8012037B50546CC
:10DEB000F0B101F01DFC0F4B00901C68AC4204D186
:10DEC00042681A6011E001F021FC74B1204601F0B3
:10DED0000FFC034602A85C6840F8043DAC42F2D156
:10DEE000009A52685A6001F011FC684601F00EFC7D
:10DEF00003B030BD24D80120002337B50360094B9F
:10DF00001C68054654B1204601F0F2FB02AB0269E1
:10DF100043F8040D2A60184601F0F8FB204603B0D0
:10DF200030BD00BF20D80120002373B50B600E4622
:10DF3000044690B101F0DCFB02AD846845F8040DA5
:10DF400044B1284601F0E2FB204601F0D1FB036911
:10DF500001903360284601F0D9FB204602B070BD25
:10DF60002DE9F74381461C200E4690461F4601F0DE
:10DF700091FE0446002831D01A4B1B4A1A6001F06A
:10DF8000B7FB009016B900F0A9F8064602A850F8B1
:10DF9000085D68466E61C5F80090C5F81080AF81D5
:10DFA00001F0B4FB2046FFF733FF104B1A6832B97B
:10DFB00001220F481A600F4B036000F079FF2046E2
:10DFC00001F096FB0C4A0190136813B9146083604A
:10DFD00001E08360146001A801F098FB204603B0C3
:10DFE000BDE8F08368170220A1DD000830D80120C9
:10DFF00028D8012085DD000820D8012073B504460B
:10E0000058B3174D2E6886420BD101F071FB02AB5D
:10E01000826843F8040D2A60184616E0684601F04D
:10E0200075FB304601F064FB866802ADA64245F8F8
:10E03000080DF3D1204601F05BFB009B8268019044
:10E040009A6001A801F062FB684601F05FFB204680
:10E05000FFF72CFF204601F085FB02B070BD00BF2A
:10E0600020D8012013B50C4640B101F041FB02ABB2
:10E07000846143F8040D184601F048FB02B010BD5E
:10E0800013B5044698B101F033FB019000F026F877
:10E0900002AB53F8042D916908445061184601F011
:10E0A00035FB2046FFF702FF2046FFF7B1FE02B026
:10E0B00010BD13B50C4668B101F01AFB02AB8289A2
:10E0C00043F8040D144218460CBF0024012401F04B
:10E0D0001DFB00E00124204602B010BD05F016BB78
:10E0E000034B1B68B3F92A2058851046704700BFC0
:10E0F00024010020034B1B68B3F92C20988510469F
:10E10000704700BF24010020024B1B689A7E98765E
:10E110001046704724010020034B1B68D96900B1E9
:10E12000D8610846704700BF24010020FEF7C8BE32
:10E1300008B5002000F01CF86FF07F4000F01AF8DE
:10E14000012000F07DF80020FFF7D4FF0020FFF74A
:10E15000C7FF0020FFF7EAFF044B1868FFF7DCFF5A
:10E160000020BDE80840FFF7CFBF00BF2801002016
:10E17000FFF7EEB9FFF7F4B910B5074B1C7820B1E3
:10E1800001221A704FF0FF3002E018706FF07F40EC
:10E1900004F0C8F8204610BD7517022070B5084D70
:10E1A0002B68012804465E7C08D800F04DFD28B19C
:10E1B0002B685C7400F008F8024B1C60304670BDA0
:10E1C000240100202817022008B503F003FFFEF702
:10E1D000F7FCBDE80840FCF799BB000008B5034B0D
:10E1E0007022196809F044FC08BD00BF240100201A
:10E1F00008B5034B01467022186809F039FC08BDC8
:10E2000024010020B0F90220B1F906309A4214DC52
:10E21000B1F90220B0F906309A420EDCB0F90020C4
:10E22000B1F904309A4208DCB0F90430B1F90020A9
:10E230009A42CCBF002001207047002070470000A8
:10E24000024B1B681A7E1876104670472401002086
:10E25000024B1A6802B91860FFF764BC34D8012079
:10E260000A4A0B49136809688B4210B50BD0094C58
:10E27000A34293E8030014BF0833503B136002F03D
:10E280002FFB012010BD002010BD00BF2001002089
:10E290001C01002088D8012068B1038889B20B4492
:10E2A0000380838819444388818092B21344438059
:10E2B000C3881A44C280704710B538B309B30AB393
:10E2C000B1F90040B2F900309C42B8BF2346038048
:10E2D000B1F90240B2F902309C42B8BF23464380F4
:10E2E000B1F90440B2F90430B1F906109C42A8BF5C
:10E2F00023468380B2F906309942A8BF0B46C380FB
:10E3000010BD11460B6803604B68436010BD0000F0
:10E31000054B1B68002B18BF0020044B0129B8BF18
:10E3200001211954704700BF90D8012054170220D2
:10E33000024B1B68588499840020704724010020F8
:10E34000044BB3F900300360034BB3F900300B60AA
:10E35000704700BF6C17022060170220014B1B683A
:10E36000987E70472401002003F0E4BF0A4B10B5EB
:10E370001C681CB1A047041C18BF0124FCF718FA44
:10E38000064B1B68002818BF01241BB198470028C2
:10E3900018BF0124204610BD6817022080170220F4
:10E3A00010B50024FFF7E2FF08B10124FAE7204688
:10E3B00010BD00000F4B73B51B68DE6C1C6D06446E
:10E3C0000D19B3B214446846ADF80030ADF804300E
:10E3D000ADF80250ADF80640FCF7B6F838B130465B
:10E3E00029462246FEF7C8FDFBF7ECFFF6E702B030
:10E3F00070BD00BF240100201E4B1B689B7E013BAB
:10E40000032B32D8DFE803F0020D1A221A4B063034
:10E410000340002B03DA013B63F00F0301330B2BA6
:10E4200008E0164B0340002B03DA013B63F00303C3
:10E430000133012BCCBF002001207047142390FB37
:10E44000F3F203FB12000B2809DC10E0182390FB09
:10E45000F3F203FB12000B2809DD20F00400103852
:10E4600001288CBF00200120704700207047012048
:10E47000704700BF240100200F00008003000080CF
:10E48000C0F30B00B0F5006FC6BFA0F5006001211E
:10E490000021B0F5806FC8BFC0F5006000F03F03F9
:10E4A00010B582110B4CC3F140039BB234F812003B
:10E4B000402B00FB03F008D0102A06D00132C3F134
:10E4C000400334F8122003FB02002030800901B120
:10E4D000404210BDDCE5010800F58060FFF7D0BFC9
:10E4E0002DE9F74FDDF83080171A5C1A54EA070C53
:10E4F00005460E46D8F800B004D103B0BDE8F04F91
:10E5000004F000BB87EAE770A0EBE77084EAE471EF
:10E51000A1EBE471884204DB21463C460F46002112
:10E5200006E011461A460B46294635460E4601219D
:10E53000009184EAE471A1EBE4718C4208D01E469C
:10E540002B46644215467F421A464FF0FF3A01E0DF
:10E550004FF0010A002FDFF848913ED1009BD3B164
:10E56000D9F800309B7E8BB93046294603B0BDE810
:10E57000F04FFEF701BDFFF73FFF30B9D9F800308B
:10E580005B6E30465B68791998470137A74207EB05
:10E590000B00F0DD1DE0D9F80030997E11B1DDF8F7
:10E5A00000A012E05B6E28461B683146984774E075
:10E5B000FFF722FF38B9D9F800305B6E0AEB05008F
:10E5C0005B68314698470AF1010AA2450AEB0B0045
:10E5D000EEDD0138C8F800005FE0D9F800104FF018
:10E5E0000202897E94FBF2F2B8BF5242D9B9934637
:10E5F000A846C5EB0803A3424FDC009B9BFBF4F14C
:10E6000031442BB9D9F800305B6E40465B6805E0B9
:10E61000D9F800305B6E5B6808464146984708F1C0
:10E620000108BB44E5E7BAF1FF3F04BF04EB0B016F
:10E63000C8F800100192AB46C5EB0B01A142D8F817
:10E6400000001EDC5044C8F80000FFF7D5FE80B97A
:10E65000DDF804C0D9F80000009B406E9CFBF4F18B
:10E66000314413B94368584602E0436808465946A6
:10E670009847DDF804C0BC440BF1010BCDF804C091
:10E68000DAE7BAF1FF3F04BF2418C8F80040D8F811
:10E690000020CAEB0203C8F8003003B0BDE8F08FD9
:10E6A000240100202DE9F04F674D2C6894F818B034
:10E6B000BBF1010F87B08146884617461E46AA4621
:10E6C00004D1109C0094FFF70BFFBAE0841ACD1A16
:10E6D00054EA050300F0B580002CBABF6442012360
:10E6E0000023002DBCBF6D4243F00203A5420BF195
:10E6F000FF3B04DD224643F004032C46154602226C
:10E7000094FBF2F202EB852595FBF4F4A1114F4A3C
:10E71000C4F38304C4F1100532F91100102D05FB78
:10E7200000F004D0013132F9112004FB0200102264
:10E73000083090FBF2F0590748BFC0F58060DA0757
:10E7400048BFC0F500609B0748BFC0F5805000F58A
:10E7500080652846FFF7C0FE00FB0BF42846FFF754
:10E760008FFE002C00FB0BF004DAC4F500739B1243
:10E770005B4202E004F500739B12002806DAC0F544
:10E78000007B4FEAAB2BCBF1000B03E000F5007BE5
:10E790004FEAAB2B002B03DD581C40105B1005E04B
:10E7A000022293FBF2F0013B93FBF2F3BBF1000F6B
:10E7B00005DD0BF1010252104FEA6B0B06E002215E
:10E7C0009BFBF1F20BF1FF3B9BFBF1FB80B21FFACD
:10E7D00089F4011992B2ADF808101FFA8BFB1FFAE9
:10E7E00088F15518CBEB01019BB2ADF80E10B9B210
:10E7F000E41ACB1AADF81030B3B20144CBEB030BE3
:10E8000013440022ADF81410ADF8163002A81346D8
:10E810000421ADF80A50ADF80C40ADF812B004F088
:10E820008FF8DAF800305B7E1BB94846414604F0A9
:10E8300069F9DAF800305B7E1BB93846314604F0DE
:10E8400061F907B0BDE8F08F24010020FEE5010862
:10E8500030B585B004AC002544F8045D0094FFF7A2
:10E8600021FF05B030BD00002DE9F8431E460C4BDA
:10E870001C6881460020E56C246D88461746FBF72E
:10E8800063FE50B109EB050008EB04017A19331956
:10E89000FFF7DEFFFBF796FDF3E7BDE8F88300BF67
:10E8A00024010020F7B5104F3B681D6DDC6C05445A
:10E8B0000E19ABB214446846ADF80060ADF80440E0
:10E8C000ADF80230ADF80630FBF73EFE48B13B68CC
:10E8D0005B6E30461B68294622469847FBF772FD5F
:10E8E000F4E703B0F0BD00BF240100202DE9F04F94
:10E8F0009846814B8BB08A46196806900020914655
:10E90000149F159ECD6C0C6DFBF71EFE002800F0C9
:10E91000EF800AF100430698013B00EB43030793A5
:10E92000169B002B14BF6FF001030223A94444443B
:10E93000099327B9FBF746FD0028FAD1D8E0002E4D
:10E94000F8D0BAF1000FF5DD7B1C04D1012E14BF05
:10E95000022301230AE0012F04D1012E14BF032357
:10E96000002303E0012E14BF052304230593624B0B
:10E970001B685B69EBB1B3F90080B3F90200B3F92E
:10E980000420B3F906B0049008F1FF38C14509EB43
:10E990000A03B8BFC9EB080803F1FF33B4BF28EA84
:10E9A000E8784FF0000893420ADDC9EB0202013219
:10E9B00007E04FF0FF3B5246CDF810B0984600E01C
:10E9C0005246169B1BB9069B03EB480300E0079BCE
:10E9D00090450393AEDA4A4408920022C8440123CA
:10E9E000029203980999058808442DB247F6FF71F1
:10E9F0008D4203900DD1029800286FD1002B6FD16A
:10EA0000114608F1FF300192FEF762FA0123019AE4
:10EA100067E00598411EDBB1042917D8DFE801F053
:10EA20000305070B0F00621B0EE0651B00E0254489
:10EA3000B5FBF6F208E0254407FB05F204E02544A7
:10EA400007FB05F2B2FBF6F200234AE02A19FBE7C6
:10EA5000042912D8DFE801F00305070B0E00651B3F
:10EA60000CE0651B00E02544B5FBF6F506E0254407
:10EA70007D4303E025447D43F6E7254404998A421B
:10EA800001DA8D4225DB5A4501DD5D4521DC05EBD0
:10EA9000020C0221AA429CFBF1FC08F1FF300BDCC6
:10EAA000114662468DE80810FEF766FADDF804C0EC
:10EAB000404661462A4609E061468DE80810FEF7A7
:10EAC0005BFADDF804C0404629466246FEF754FA78
:10EAD000009B029A013202922A4602E0002302932E
:10EAE0000123089808F1010880457FF47AAF21E7F7
:10EAF0000BB0BDE8F08F00BF24010020F8B50B4B30
:10EB00001B680546B3F92C0040F002000F4616467C
:10EB1000FFF7F0FA394604463246284600F008F876
:10EB20002046BDE8F840FFF7E5BA00BF2401002009
:10EB3000024B1B6859849A8400F002B8240100201B
:10EB40002DE9F74F0446002879D03E4D00F0B4FC83
:10EB50002B688046B3F8229000F096FC2B689A8CC4
:10EB600087B2D21B9A842378002B5DD047F6FF71C1
:10EB7000204600F0D7FB06463146204600F000FC58
:10EB80002B689A8D02F00302012A05D0022A14BFD5
:10EB9000002290FBF2F200E00246598C8A1A92B2EF
:10EBA00091B259841FFA80FA9B8CADF800100AF1DB
:10EBB000FF310A44ADF802301FFA88FB013B5B4489
:10EBC000ADF80420204631466A46ADF8063000F024
:10EBD00007FC2B68BDF802209A842046314603F0DA
:10EBE00029FE235C0A2B04EB000201D00D2B12D16D
:10EBF0002B68998D01F00301013901298ABF198C15
:10EC0000A3F82290598411780A290BD1998C8B444E
:10EC1000A3F824B006E00B4BBDF800001B6882444B
:10EC2000A3F822A0137843B92B689A8C17449A8DC5
:10EC30009F8422F003029A8501E0541C93E703B0FD
:10EC4000BDE8F08F24010020012809DC054B53F8B2
:10EC5000200020B1C3681B681BB10068F9E770474A
:10EC6000002070478417022000F02EBD012BF8B55C
:10EC700006460D4617461C4601DD0020F8BD1C2047
:10EC800000F08EFE0028F8D00DB1056109E0094BB7
:10EC900053F8241029B10B680BB11946FBE70B6937
:10ECA00003610023836084618782C66003604360E0
:10ECB000F8BD00BF84170220094B826953F8221067
:10ECC000814204BF016843F8221043680BB1026817
:10ECD0001A60026802B1536000230360436070470A
:10ECE0008417022070B538B38269012A24DC1949DF
:10ECF00051F822300D4613B941F822001AE0596844
:10ED000009B10B46FBE7C1680E68D9680C68B442CC
:10ED100003DD1B68002BF8D10EE002D1818A0129A6
:10ED200011D0596899B1086041605860984208BF95
:10ED300000230360002070BD012070BDCB681B68FC
:10ED4000A3420B46EDDB19680029F7D1E9E745F846
:10ED50002200EAE78417022038B51D46FFF786FF38
:10ED6000044648B1FFF7BEFFE3681B6823B9034BB5
:10ED700016351B6843F82540204638BD2401002085
:10ED800010B5074B07480024214670221C60FEF78F
:10ED90001DFC214604480822BDE81040FEF716BCC1
:10EDA00010D9012098D801208417022038B5194DB8
:10EDB0002B681A1DDA6303F108029B631B6442612E
:10EDC0005A7C154B044653F82200C36804F108012D
:10EDD0001B6B9847114B6366114B1B68E3612B68F3
:10EDE0000833636101232376FAF762FC032384F876
:10EDF00068306FF0704323636363A0640020FEF704
:10EE0000A7FB6FF07F40FEF7ABFB064B064A1A608C
:10EE100038BD00BF240100208417022020E601082D
:10EE2000280100207C1702200C0702082DE9F34777
:10EE3000074604209A460E469146FEF741F8134BCA
:10EE40001C68E56C246D2F44264480464D44544490
:10EE50006846ADF80070ADF80450ADF80260ADF84A
:10EE60000640FBF771FB28B94046FEF729F802B0CF
:10EE7000BDE8F087384631462A462346FEF7A2F819
:10EE8000FBF7A0FA0028F5D1EEE700BF240100202F
:10EE900010B500200146FFF74BFA044843F6FF7215
:10EEA00001461346BDE81040FFF7C0BF01C0FFFF99
:10EEB00080B483B000AF7860054B1A687B685A60F5
:10EEC000034B7A681A600C37BD465DF8047B7047C7
:10EED00094D8012008B5084B1A6862B901221A605B
:10EEE000F1F7A2FBF1F7C8FB0448054B0360BDE84E
:10EEF0000840FFF7DDBF08BD10D9012008D9012067
:10EF000081ED000890B583B000AF204B1F4A126816
:10EF100022F001021A601E4B01221A601D4B1E4A8C
:10EF20001A601C4B1A681D4B9A4200D0FEE7FFF78F
:10EF3000D1FF1B4B2E221A7004F0EAFB1948FFF791
:10EF400035FFFEF763FA7860FDF744FF0346002BB8
:10EF500004D0FDF745FF0346002B09D1FDF726FF3E
:10EF60000446FDF726FF034620461946FDF728FF15
:10EF70000020002103F070FCFBF732FD0A4B012258
:10EF80001A707B6818460C37BD4690BD002000E023
:10EF90000830024000300240C2A507F4CDB5E8B504
:10EFA0005617022098D801207417022038B1038820
:10EFB0008B4202D843888B4201D28068F6E77047C3
:10EFC0002DE9F04F384C2368B3F92A90DB690546E8
:10EFD00089B0D8692946FFF7E9FF002861D0B0F869
:10EFE00000804768C8EB050807EBC806484696F856
:10EFF00002B0FDF765FF256817F83820D5F81CE04A
:10F00000B5F924109EF81AC09EF81830069382466F
:10F01000B5F92200CDF800C09EF81BE0CDF804E061
:10F020004FF0010ECDF80CB0CDF808E073680493F2
:10F03000AD6B069B0595FEF7CDF82368DA6992F86B
:10F0400019B0117E8B4520D9B9F1020FD57E1CD0A5
:10F05000079103F04DFC814603F043FCFFF78AF86B
:10F06000246817F83870E269B4F92430B4F9220042
:10F07000D27E079907FB020201FB05310BFB05332A
:10F08000FDF7A0FF4846FFF775F85046FDF718FF5B
:10F09000054B1B68DA69598C907E727800FB02126E
:10F0A0005A8409B0BDE8F08F240100200D4B70B5E3
:10F0B0001B68DD6906460C46E8693146FFF776FFB6
:10F0C00070B103884268F61A02EBC6035878AB7E2B
:10F0D00010FB03F024B112F8362012FB03F3236077
:10F0E00070BD00BF2401002001230B80704708B5CC
:10F0F000C069FFF75BFF003018BF012008BD0000AA
:10F10000524B2DE9F04F1B68D9695F8CCC699D8CFF
:10F11000A28990428BB008D3E689864205D3D4F801
:10F120000090821A4FF0FF3B15E0A268D4F80490DB
:10F13000002A00F081801688B0427DD3B2F802C068
:10F14000844579D35268801B80B202EB800632F985
:10F150002020B6F902B0501C6ED091F81880A17C26
:10F16000B3F82AA0267C069218FB01F107910FFA4A
:10F170008AF108460891FDF7A3FE344909900B680F
:10F18000069AD969887E0090C97E01910121029179
:10F19000A17C0391079901FB029204929B6B05935A
:10F1A0003FB22DB23846294632464346FEF712F8A2
:10F1B000BBF1FF3F1BD04AF0020000B2FDF780FE1A
:10F1C000224A1368DA69917E0091D27E0192012170
:10F1D00002910799A27C039201FB0B9204929B6B14
:10F1E00005933846294632464346FDF7F3FFDFF8DC
:10F1F0005C80D8F80030DB695A7E1B7E9A4217D9B2
:10F20000089A022A14D08AF0040000B2FDF758FED2
:10F21000D8F80030DB6993F818E0D97E9A7E5B7EDF
:10F2200038460EFB015106FB02722B44FDF7CAFE65
:10F23000099BD8B2FDF744FE044B617C1B685A8CD5
:10F240000A445A840BB0BDE8F08F00BF24010020AF
:10F25000044B1B68DB69DB6909B11A7C0A60587CC6
:10F26000704700BF2401002002230B807047C36950
:10F270009A898A4202D8DA898A420FD2986880B184
:10F28000038899420CD342888A4209D3C91A42683A
:10F2900032F82100C043C0F3C030704701207047EE
:10F2A000002070477047000037B5154602AB1A4A78
:10F2B00043F8081D01901268184C6946904723686E
:10F2C0000190586958B90120FEF72CFA2368DB69D0
:10F2D0005B69BBB19B6801980099984717E0294684
:10F2E000FEF790FF0028EED114E001A803F08EFA9B
:10F2F0002368DB691B6805469847094B1B680BB1FF
:10F3000028469847009B013B002B0093EDDA002034
:10F31000FEF708FA03B030BD2C01002024010020C4
:10F320007017022037B50D460190044698B10B4B7B
:10F330001B68DB695B690BB15B680BB9002408E0F3
:10F34000984709E001A803F061FA20B10A2802D029
:10F350000134AC42F6DB204603B030BD240100206E
:10F3600013B502A9002441F8044D00F0B7F8019B41
:10F370008342CCBFC0EB0300204602B010BD0000AA
:10F3800037B5154A019002AB126843F8081D69466B
:10F3900090470190F0B1114B1B68DB695B690BB1C1
:10F3A0001B6813B900252C4602E00099984711E02C
:10F3B000009B013B002B009307DB01A803F026FA1A
:10F3C000054600F081F80444F2E72846FFF7C8FF3D
:10F3D0002044FFE703B030BD2C01002024010020B1
:10F3E000274B1B6873B505460C4663B10020FBF73D
:10F3F000ABF8002841D0284621466A46FFF754FF63
:10F40000FAF7E0FFF5E7106851681E4E6B4603C33C
:10F410003368BDF80010B3F84C20B3F850301144F5
:10F42000ADF80010BDF802101944ADF80210BDF897
:10F4300004100A44ADF80420BDF8062068461344C1
:10F44000ADF80630FBF780F8336840B9598CDA6CB8
:10F450008A1A5A84998C1A6D8A1A9A840DE0BDF81A
:10F4600000205A84BDF802209A84284621466A4624
:10F47000FFF71AFFFAF7A6FFE6E702B070BD00BF7C
:10F4800058170220240100200A4B1B689A8D02F0B5
:10F490000C02082A07D00C2A05D0042A07D1DB6900
:10F4A000187E01387047DB69187E400870470020DD
:10F4B000704700BF24010020024B1B68DB69587EA7
:10F4C000704700BF2401002008B5034B1B68DB69AF
:10F4D00000215B68984708BD2401002008B5034B54
:10F4E0001B68DB695B68984708BD00BF24010020EA
:10F4F000074B5A68596A013210B55A605A6B02EBD1
:10F50000C0046160002102F83010586210BD00BFD5
:10F510009417022038B50B4D002405F14000214618
:10F52000802285F82840FEF751F828462146C0225F
:10F53000FEF74CF8214604480C22BDE83840FEF79F
:10F5400045B800BF9417022014D9012010B54268B5
:10F550000F230D4901EBC304246CA24203D213F123
:10F56000FF33F6D210BD0F2B0CD80C68A21A0A601C
:10F570008268C06802B1506008B1026010BD01EB42
:10F58000C3035A6410BD00BF94170220F8B5264E7D
:10F59000F3685A1EB36B05461344081898420C468C
:10F5A00005D84B591BB943681D44FFF7CFFFB36B18
:10F5B0009C420AD954F8047CE71B3B682BB97B6852
:10F5C00038461D44FFF7C2FF3C460F2306EBC3023B
:10F5D000126C954203D213F1FF33F7D222E00F2BC6
:10F5E00020D8083306EBC30261195268A2600020DC
:10F5F00084E82100246141F8045C04F1080102B1AF
:10F60000516006EBC303E0605960336896F8291037
:10F61000054A2B44336029B9D168CB1A91689942C5
:10F6200038BF93602846F8BD94170220254B2DE97A
:10F63000F74FDA689C6B013A824602EB04099B465D
:10F6400094E82800002B33D104EB0508C8452FD2DD
:10F6500054F805C0D8F80460BCF1000F28D0DBF8DE
:10F660003430184F13F83C30012B21D1FB6A20466F
:10F670008DE80810FFF76AFFD8F800107A6B02EBEC
:10F68000C102204654604146324608F03BF99DE8ED
:10F6900008109C4502D17B6B5B1B7B632846A1193C
:10F6A000FFF774FFBAF1000F01D0824505D9354646
:10F6B0002C444C45C4D3012000E0002003B0BDE839
:10F6C000F08F00BF9417022028B1034AD36B036068
:10F6D00003B15860D06370479417022028B1034BE0
:10F6E0005B6B03EBC0004068083070479417022042
:10F6F000054BD9690131D9615B6B13F830100131C9
:10F7000003F83010FFF7EABF9417022030B5026803
:10F71000094B52F8081C5A6B12F83140012C03D9DE
:10F72000DD690DB1013DDD61013C02F8314000238E
:10F730000360184630BD00BF94170220024B21F031
:10F74000030118605960704714D9012030B1044B8F
:10F750005B6B03EBC000436858680C38704700BF10
:10F760009417022010B5044680B1094B5B6B03EB84
:10F77000C00213F83030012B08D151684868FFF7F8
:10F7800005FF2046BDE81040FFF7B2BE10BD00BF28
:10F79000941702202DE9F041224CE36A3BB9224B39
:10F7A0009D685B680835B3FBF5F5023503E0236916
:10F7B0001D1D05EBD305E80000F078F9804660B325
:10F7C000616B2269E76A01EBC003D2005E6808360C
:10F7D000304608F04DF92269666306EBC201C4F8B1
:10F7E0002C8004311346681E834201F1080103D2C4
:10F7F000013341F8083CF6E706EBC30300265E60E0
:10F80000636862629B1A2B446360256138463FB18E
:10F81000FFF7A8FF3046BDE8F0810120BDE8F08188
:10F82000BDE8F0819417022014D90120F8B5584E94
:10F8300096F82810002940F0AA80564D6A680123E6
:10F8400086F82830B2F5205F28BF4FF420522B688D
:10F8500094080020A0420CD047184FF0FF0EB7FBD1
:10F86000FEFECEEB0E2ECEEB070743F820700130E4
:10F87000F0E70020A04216D047184FF0FF0EB7FB6C
:10F88000FEFECEEB0E2ECEEB070E53F82070774522
:10F8900007D0AA683F4B002A55D15A6892089A604F
:10F8A00051E00130E6E701310229D2D154080021AC
:10F8B0000020A0420CD047184FF0FF0EB7FBFEFE11
:10F8C000CEEB0E2ECEEB070723F810700130F0E7D9
:10F8D0000020A0420FD047184FF0FF0EB7FBFEFEEE
:10F8E000CEEB0E2ECEEB070733F810C0BFB2BC45EF
:10F8F000CFD10130EDE701310229D9D1002100201B
:10F90000904207D04418FF27B4FBF7F73C441C543F
:10F910000130F5E7002090420BD04418FF27B4FBDC
:10F92000F7F73C441F5C04F0FF04A742B1D101305B
:10F93000F1E701310229E2D100219142A9D0002052
:10F9400058540131F9E71448144B0360FFF7B0FA3B
:10F950005A2333620023102106EBC302994001337E
:10F96000102B0B4C1164F6D168682968A16302233F
:10F970002361A0F114030B4401256363E0605D6023
:10F9800065626560FFF702FEFFF704FF2563F8BDBF
:10F990009417022014D9012020D9012015F5000860
:10F9A0002DE9F0410546264E0335FFF73FFF25F0D0
:10F9B0000305336CF26B04359D4238BF1D46144677
:10F9C0002CB154F8043CAB422CD02468F8E7F3681F
:10F9D000B26B02EB030858F8047CC7EB08073B68DE
:10F9E00033B12046FFF722FE58F8047CC7EB080726
:10F9F0003B6813BB7B68AB421FDB38461C1DFFF71F
:10FA0000A5FDF36878685B1BF3607369641B2B4486
:10FA1000401B3C44736102D03946FFF7B7FD44F800
:10FA2000045C0AE023680BB161685960616801B148
:10FA30000B60A24201D12368F3632046BDE8F08148
:10FA40009417022008B5FFF7F1FE00220B4B134478
:10FA5000D3F8BC3013B19B6800200BE0083A12F1D8
:10FA6000800FF3D1F8E75A689B68904238BF104680
:10FA700013B19B68002BF6D10C3808BD94170220F7
:10FA800008B5FFF7DFFFB0F5800F4FF06403064ABB
:10FA900004D990FBF3F0136A584308BD126A50432F
:10FAA000B0FBF3F008BD00BF941702202DE9F84326
:10FAB000384D0446FFF7BAFE2F6C2B68BC4224BFBA
:10FAC000E71C27F003070C379F42324C3ED8236BCC
:10FAD00062689A420FD96B686E6A013B6B606B6B10
:10FAE0004FEAC60903EB090252686A62012203F871
:10FAF000362056B92AE0013B2363FFF74BFE236B08
:10FB0000013323630028E6D020E00F2305EBC30276
:10FB1000126C97420CD213F1FF33F7D208E09468CD
:10FB20002CB16268974214D9A268002AF7D1013338
:10FB30000F2B03D805EBC302526CF6E73846FFF7EC
:10FB400075FD0028E1D03046FFF7D2FC0020BDE86B
:10FB5000F883D4F804802B6CC7EB08020C332046E2
:10FB60009A4238BF4746FFF7F1FC6B6B4B44E119F3
:10FB70005C60B8454FF0000384E8C000A3602461D6
:10FB800041F8047C03DDC7EB0800FFF7FFFC3046BB
:10FB9000BDE8F8839417022008B1FFF787BF7047CC
:10FBA00010B504460068FFF7DDFD0023236010BD9B
:10FBB00010B580EAE071A1EBE0710022531C0A2B22
:10FBC00006D0064C54F82340A14201D31A46F5E76B
:10FBD0000028B8BF931C184610BD00BF28E60108D6
:10FBE000002807DD0B685A1C0A602B221A700B686C
:10FBF00000221A7070470000B0F1004FF0B51C6889
:10FC000009D1601C186001392D202070C9B26FF035
:10FC1000004001260CE0002806DA651C1D602D2539
:10FC200025704042012400E00024091BC9B20026CF
:10FC30000AB30139C9B21EE04D1E9142EDB205D1A1
:10FC40001C68671C1F60114F3F782770104C54F8D8
:10FC5000257090FBF7F4E4B20A2C0ED807FB1400D1
:10FC60007DB10A2C18BF29461D6808BF01246F1CEE
:10FC700030341F602C700029DED11B6800221A70FE
:10FC8000F0BD002EEDD00134E4B2EAE756170220B1
:10FC900028E6010873B50546FFF77EFF064658B112
:10FCA000FFF726FD02AC002144F8040D2A46FDF7BB
:10FCB0008DFC2046FFF72AFD304602B070BD0000E3
:10FCC0002DE9F7431E4CD4F800E0DEF84C40DEF896
:10FCD0005060051914449EF81820013A92B28F1909
:10FCE0001E44AB1AADF800301319ADF80430684665
:10FCF000BB1A3244ADF80230ADF80620FAF724FC06
:10FD0000D0B1284639462246FDF710F907F101091E
:10FD100028463146224606F1FF38FDF707F9284606
:10FD200049464246FDF728F9204649464246FDF736
:10FD300023F9FAF747FBE3E703B0BDE8F08300BF20
:10FD400024010020C0F3C421064B00F01F02C0F3C1
:10FD500045109A5C5B5C03EB0243034A105C03EBC7
:10FD600000207047EC040208AC040208C0F307410D
:10FD7000064BC2B2C0F307209A5C5B5C03EBC22364
:10FD8000034A105C03EB4010704700BF0C060208EA
:10FD90000C0502084FF6FF7070470000F8B50F4FD2
:10FDA0003F6806460D4614469C460FB1B847F8BD5D
:10FDB00056F8042B0A49D3B2013CC85CC2F307438E
:10FDC000C2F30722CB5C07498A5C03EBC02303EB39
:10FDD00042132B806544EBD1F8BD00BF2CD9012024
:10FDE0000C0602080C050208F8B5134E3668844666
:10FDF00014461D460EB1B047F8BD501E02F18042B8
:10FE0000013A03FB00C001EB820102880B4B02F0B8
:10FE10001F06D70A9E5DDB5DC2F3451203EB064366
:10FE2000074EB25C013C03EB022341F80439C5EBF9
:10FE30000000EAD1F8BD00BF28D90120EC04020877
:10FE4000AC0402087047704770474FF0FF307047AE
:10FE500010B550F8044B0C60013A1944F9D110BDAB
:10FE600010B5046841F8044B013A1844F9D110BDAB
:10FE700010B59CB004466846FEF7B0F9094B186807
:10FE8000FDF76EFBB4F90000B4F90210B4F90420D8
:10FE9000B4F90630FFF714FF6846FEF7A9F91CB065
:10FEA00010BD00BF30D9012010B59CB00446684693
:10FEB000FEF794F9094B1868FDF752FBB4F90000FE
:10FEC000B4F90210B4F90420B4F90630FFF7F8FED3
:10FED0006846FEF78DF91CB010BD00BF30D9012077
:10FEE00007B56846F9F702FC6846FFF7C1FF03B0A3
:10FEF0005DF804FB07B56846F9F7F8FB6846FFF7BD
:10FF0000D3FF03B05DF804FB13B5044640B1FFF71F
:10FF1000EFFB02AB046D43F8040D1846FFF7F6FB48
:10FF2000204602B010BD1FB501F00803002B40F2BF
:10FF30008A3440F28A5208BF22460CBFFF23FE23B8
:10FF40008DE8050000200291039302460346014616
:10FF500000F0AEF806210446F9F707FA204604B08F
:10FF600010BD07B5FFF7C4FB0190406E00F0D4FB55
:10FF700002A8002250F8043D5A66DA65FFF7C6FB76
:10FF800003B05DF804FB438E1B0710B512D5B0F922
:10FF90000420B0F9003008884C880C80D31A8A8875
:10FFA000CC888C8001339BB2C043D24318441344A5
:10FFB000C8804B8010BD10B5044600F0B6FCFAF7BF
:10FFC0008CF82046F9F7ABFA2521BDE81040F9F787
:10FFD0004FB90000F0B589B00E9E109C119DFAB982
:10FFE000F3B9304606A9F9F717FB14F0080F2C4BAC
:10FFF000BDF91C70BDF91EE009D0BDF91A10B3F9A6
:020000040801F1
:100000000020781CC1EB0E03801A013308E0BDF913
:100010001800B3F900300EF101013A1AC91A013281
:1000200000960F9E01961F4E0296129E3C36039636
:10003000FAF794F8064600282FD0FFF759FB04F092
:100040000802E30648BF42F01002A5F1FE0348BFD4
:1000500092B2012B88BF42F0100229460590F8F7B2
:1000600041F8114B08AF0FCB57F80C4D04F1340594
:1000700085E80F006423E3640C4D0A2363650023C5
:1000800023652B6863643846FFF740FB2B683046D6
:100090005B6898473046FFF78EFF304609B0F0BDE9
:1000A00044010020530101083001002040010020DC
:1000B00010B586B0089C0094099C01940A9C029497
:1000C0000B9C039400240494FFF784FF06B010BD3A
:1000D00037B50C46054600B3FFF70AFB002C01902C
:1000E000C16C426D05DB8A1A22EAE272944202DC9C
:1000F00000E000242246016D91420BD002652846A3
:10010000F9F7EBFF01A8FFF701FB28460521F9F7F6
:100110002CF902E001A8FFF7F9FA03B030BD73B57E
:100120000D46064660B1FFF7E3FA024602A8146DD9
:1001300040F8042DFFF7EAFA30466119FFF7C8FFCF
:1001400002B070BD4FF0FF31FFF7E9BF0121FFF7AB
:10015000E6BF2DE9F04F446880468FB02046414607
:10016000F7F7C8FF002800F0C081D8F80030232B33
:1001700000F082810BDC0E2B00F02A810F2B12D0B5
:100180000B2B40F0AF812046FFF715FFAAE140F2AC
:100190001312934200F07F81B3F5107F12D0242B0D
:1001A00040F0A08143E12046FFF7A2FA0590002825
:1001B00000F09B81436C05A81D68FFF7A7FA204655
:1001C000A84792E1D8F80C70002F00F08B813B7AA1
:1001D0002046002B00F0D680FFF78AFA05A9836C31
:1001E0000390066D20469847039BB3F832A05D6DDF
:1001F000DA6C1AF0080FC5EB020903D097E8060085
:100200003A6079609A6D3F68032A14D12046FFF75F
:10021000A8FE0D9B0C99022093FBF0F3FF1A069B9E
:10022000FB1A581E00FB09F002F049F9039B064631
:10023000186603A87EE0069887420BDC022A39D0B4
:100240005B6E13B12046FFF78CFE039B0222013E3A
:100250009A652FE007998F4202DA761B6D422FE0F4
:1002600008998F4212DC0C9900290BDD0D9B0222AC
:1002700093FBF2F3FF1A3F1A013F07FB09F002F06C
:100280001EF90646039B03229A6516E009998F42E0
:1002900001DA2E4414E00A998F420EDC012A0ED0B6
:1002A0005B6E13B12046FFF75CFE039B0125013610
:1002B0009D6505E04FF0FF3502E0002500E01546A2
:1002C000DDF80CB00C99DBF85C30DDF834E0069A10
:1002D00071B102209EFBF0F0381A801A013800FB41
:1002E00009F0019302F0EBF8019BCBF8600009E004
:1002F000DBF85820012A04BFDBF84C1001F1FF3174
:10030000CBF8601003A80193FFF700FA019BA5B199
:10031000BBB94FF4C87240F2D241204600F034FA23
:1003200007462046FFF7E4F902460EA840F8282DBC
:100330005766D565FFF7EAF903E013B12046FFF7EA
:1003400010FE2046012100F0A3FA20463146FFF7B7
:10035000BFFE1AF4807F40F0C5802046FFF7C8F941
:100360000EAB856A43F8280D1846FFF7CFF94FF416
:1003700080712046F7F78AFEA90740F1B380204636
:10038000012174E0FFF7B4F9458E039003A8FFF74D
:10039000BDF9EA0540F1A68020464FF48071F7F7D9
:1003A0008BFE2046FFF7A4F9C36D059013B12046DC
:1003B000FFF7D7FD0EA8002250F8243D9D6A9A65EC
:1003C000FFF7A4F9AB0740F18D80204602214EE0F3
:1003D0002046FFF78DF90EAB456D43F8240D184606
:1003E000FFF794F9D8F80C2013685268002A79DDD9
:1003F000103B122B76D8DFE803F016161212757533
:1004000075757575757575757575750A0D00204668
:10041000294601E020466942FFF781FE62E020465E
:10042000FFF794FE5EE02046FFF78CFE5AE0204680
:10043000D8F80C60FFF75CF90EAD034645F8240DC3
:10044000DA6C3068B1689042726805D15E6D8E4298
:1004500002D11E6D96420DD0D86459651A652046AA
:10046000F9F73BFE2846FFF751F920460521F8F73A
:100470007CFF37E0284633E02046FFF739F9059046
:1004800000282FD0D8F80C30C26C1A60426D9A60E8
:10049000026D5A6023E02046FFF72AF9C16D0590EE
:1004A00011B12046FFF73BFE059BDA6D196D002A5E
:1004B0001A6E05DD9142B4BF0021012106DD04E082
:1004C0009142CCBF0021012100DA1A6519B1204602
:1004D000FFF747FD03E0586E322100F085F905A8CB
:1004E000FFF714F94046FAF723FA0FB0BDE8F08F92
:1004F0000388994213B50C460ED2406850B1FFF7FD
:10050000F7F802AB50F8244043F8040D1846FFF703
:10051000FDF802E0044600E00024204602B010BDD1
:1005200013B5044640B1FFF7E3F802AB048843F883
:10053000040D1846FFF7EAF8204602B010BD2DE979
:10054000F743054600283DD04AB10846114602F05F
:100550004FFBD0F10104074638BF002401E01446E8
:1005600017462846FFF7C4F802AEB0F8008046F8F8
:10057000080DD0F804906846FFF7C8F824BB08F1CE
:1005800001014846890002F081F9814618B93846D0
:10059000FFF7E8F818E0FFF7ABF802AB43F8040DFB
:1005A00040F828701846FFF7B1F82846FFF7A0F882
:1005B000038800900133C0F8049003806846FFF779
:1005C000A5F802E0044600E00124204603B0BDE89F
:1005D000F08337B5054618B3FFF78AF800904068F6
:1005E000C0B1FFF785F800240190009B1B889C4256
:1005F00006DA019800EB8400FFF7D2FA0134F4E741
:1006000001A8FFF783F800980430FFF7C9FA009BB0
:1006100000221A806846FFF779F82846FFF7A2F80B
:1006200003B030BD73B50E46054658B1FFF760F80C
:1006300002AC314644F8040DFFF75AFF0546204648
:10064000FFF764F8284602B070BD0820FFF722BB10
:1006500030B585B0044610220D466846002107F0EB
:100660006BF92046FFF73AF803691BB10194009536
:100670006846984705B030BD70B50D4C2368132B04
:1006800006460D4612DCFFF729F803696E6043B198
:10069000226828460132226098472368013B236084
:1006A00070BD2846BDE87040FAF742B970BD00BF82
:1006B00034D9012038B5054600F00FF8044654B18E
:1006C000AC4207D02046FFF709F8036AAB4202D0DC
:1006D0001C46F4E70024204638BD08B5F8F71FFF94
:1006E00018B1FEF7FBFFC06908BD08BD1FB5044681
:1006F00000216846102207F01FF9606850B1FEF72C
:10070000EDFF40F21313406800936946636803935A
:10071000F9F78CFC04B010BD37B5054668B1FEF79B
:10072000E7FF02AC44F8040D0068FDF767FC2046C3
:10073000FEF7ECFF2846FFF715F803B030BD73B5A0
:10074000054601A8FDF7D8FB0446DCB1204601218F
:10075000FDF7AFFC019B83B178B11846FEF7BEFFF1
:100760004368AB4209D1204601A9019EFDF7DCFB9D
:1007700004463046FFF7D0FFE7E7204601A9FDF722
:10078000D3FBE1E702B070BD2DE9F34180460C20B8
:100790000F461646FFF77EFA0446F0B1FDF79EFCC1
:1007A0002246811901230F48FDF7DAFB0546204652
:1007B00085B1FEF79DFF034602A8C3F8048040F808
:1007C000043D9F601D60FEF7A1FF28463146FDF7FE
:1007D00049FC02E0FEF7C6FF2C46204602B0BDE809
:1007E000F08100BFED06010813B50C4680B1FEF79D
:1007F0007FFF01901CB100682146FDF733FC02AC7D
:1008000054F8043D1868FDF73BFC2046FEF77EFFD8
:1008100002B010BD2DE9E7410E4690460746D0B123
:10082000FEF766FF034602A8B3F90410B3F90020EF
:10083000B3F9065040F8043DB3F902308A1AED1AB4
:10084000D243ED4316444544FEF760FF3846314637
:100850002A46F8F70FFD03B0BDE8E08130B50A4D38
:100860000A4C2B6854F8230085B050B104A9182312
:1008700041F8103D6946FFF7FFFE2B68002244F85F
:10088000232005B030BD00BF2817022044170220E6
:10089000F8B5094B094A044618680F4652F820106B
:1008A000A14215461E4601D0FFF7D8FF336845F830
:1008B0002340034B1F70F8BD281702204417022065
:1008C0002C17022038B505460C4641B1F8F727FE33
:1008D00028B1A5602146BDE83840FFF7CDBE38BD40
:1008E0007FB50A4A03461068094A52F8200048B109
:1008F00000930E230191029302A900AB0593FFF729
:10090000BBFE012007B05DF804FB00BF28170220E2
:100910001817022010B50C4630B129B1FEF7DEFEE3
:10092000034603CB2060616010BD38B50546F8F77B
:100930007FFEFF28044603D0FE2808BFFF2400E006
:10094000FE242846F8F7EBFD2146BDE83840F8F7CD
:10095000ABBE02F00ABD0000024B1A6802601860CC
:10096000704700BF3C1702202DE9F043044687B0D2
:10097000002839D0FEF7BCFE0346019003C804AD41
:1009800085E8030001A81E6AD3F82890FEF7BEFE92
:100990002046FFF78FFE074630B32046F8F7BFFD2D
:1009A00019F0020F804604D0284641463246F9F736
:1009B00025FB2046FEF79CFE01904046FEF798FE80
:1009C00003903846FEF794FE039B019AD9690662AC
:1009D0000290116201A8DC61FEF798FE03A8FEF701
:1009E00095FE02A8FEF792FE07B0BDE8F0832DE960
:1009F000F84FDDF828B0DDF82CA005460E469046ED
:100A00001F461446894635F8020BD847D047013CAB
:100A100049F8040BF7D11F2F06D8304641463A4615
:100A2000BDE8F84F01F058BDBDE8F88F2DE9F84F4B
:100A3000DDF828B0DDF82CA005460E4690461F468E
:100A40008946044614F8010BD847D0472B1B434472
:100A500049F8040B002BF5D11F2F06D8304641462C
:100A60003A46BDE8F84F01F037BDBDE8F88F000009
:100A70002DE9F04F9DB006460F910D92002800F031
:100A80008683FEF735FE1CAB446943F81C0D1846FF
:100A9000FEF73CFE3046FAF787FF0828014602DDE4
:100AA000002C00F0C38101224FF0000830461B9259
:100AB0000B92CDF86880FEF71BFE0368DFF80CA6EA
:100AC0001B69B0F90A105B680E930DF1700BDAF830
:100AD00000304BF8140D04694569D0F80C90B0F95A
:100AE0000870587C1291FCF733F9DAF80030109056
:100AF000587CFCF74BF9034658460993FEF706FE6F
:100B0000082C51460B9A099B04D9102C8CBF042247
:100B1000022205E0012C03D111940DF1680800E0D8
:100B200011920E98984200F0E2800B68587CFCF716
:100B300035F91390B800FFF72FF80C90002800F05B
:100B400026833046FAF7CCF80646002D00F0BE802A
:100B50002846FEF7CDFDDDF834B018904FF0000ABE
:100B6000129A924580F2AE801898002319938368F8
:100B700019A95B6952469847B84205462FD10C988F
:100B8000FEF7B6FD082C0146169009D90E9A139B64
:100B90000092019330463A46109BFFF728FF08E089
:100BA0000E98139A0090019230463A46109BFFF738
:100BB0003DFF0123109802901CAD00220093019389
:100BC000039255F8182D04920F98CDF814805946C9
:100BD0003A46FCF7FFFA2846FEF798FD60E0012C44
:100BE0005CD1002D5CD019980F99CDF80C9008229B
:100BF00090FBF2F232440123049200F007020093CA
:100C0000084401930293069259462A46CDF814806F
:100C1000FCF704FA199B18981D44836819955B69C1
:100C200019A9524698470546DBE70C98FEF760FD88
:100C3000082C01461690199838D90E9A0092119AEC
:100C4000139B019300FB0260109B2A46FFF7CFFE27
:100C500001230DF1700C1098009300220193029073
:100C60000F99039219985CF8182D049208442A46AB
:100C70005946CDF81480CDF82CC0FCF7ABFADDF85E
:100C80002CC06046FEF742FD199B18981D448368EE
:100C900019955B6919A9524698470546002DC4D19C
:100CA0004E440AF1010A0BF1010B59E70E9B009328
:100CB000119B139A019200FB03602A46109BFFF7D9
:100CC000B5FEC5E718A8FEF721FD0EE0012300934D
:100CD000019304900294CDF80C90CDF814800F98F5
:100CE0000D99129B3A46FCF775FA0C984DE2304686
:100CF000F9F7F6FF0646002D00F08A802846FEF739
:100D0000F7FC00251890129B9D427DDA189800236D
:100D10001993836819A95B692A469847B8428246A5
:100D200024D1AA46189883680AF1010B5B6919A9B6
:100D30005A469847B84201D1DA46F3E7C5EB0A0BA9
:100D40000D99049601230BF1010B009301932944A3
:100D50000294CDF80C90CDF814800F983A465B467B
:100D6000FCF738FA09FB0B6655464BE0012C27D1FE
:100D7000BAF1000F22D019980F99CDF80C900822E3
:100D800090FBF2F23244049200F0070208440D99FD
:100D90000692012352460093019302932944CDF811
:100DA0001480FCF73BF9199B1898534419938368F6
:100DB00019A95B692A4698478246D9E74E4421E043
:100DC000BAF1000FFAD019981199029400FB016250
:100DD00004920D990F9ACDF80C90012310440093C2
:100DE000524601932944CDF81480FCF7F3F9199B7E
:100DF000189853441993836819A95B692A46984740
:100E00008246DDE701357EE718A8FEF77FFCBEE1EC
:100E100001230093019304900294CDF80C90CDF837
:100E200014800F980D99129B3A4641E030460A9182
:100E3000FEF75EFC82461CA8BAF80A2040F810AD06
:100E4000DAF800401092D4F81090BAF808709E4C6E
:100E500013B2DAF80C200B920993FEF757FCD9F87D
:100E600004000E9099480068407C54F820402569A1
:100E7000D5F80080FBF76CFF08280FFA87FB0A996A
:100E80000B9A099B04D910288CBF0424022400E08B
:100E90000124A9450FD1012003920AF11802009004
:100EA0000190029104920F980D99002205925A46E2
:100EB000FCF790F96BE1202940F08E800BFB04F0E9
:100EC000FEF76AFE0E90002800F06181FEF710FC2C
:100ED0001A903046FEF70CFC18902B6900F1180AA6
:100EE0004FEA8B064FEAC409002B2FD0DDF834807F
:100EF000022C03D0042C01D0012C06D150462F69BE
:100F00001A995A462346B847B244012300221A9937
:100F10000093019303920491059241465A46CDF8FD
:100F200008900F98FCF756F910990D9A08F10107EF
:100F300002FA81F3BB4207D118A8FEF7E7FB1AA813
:100F4000FEF7E4FB0E9820E1B846D1E70D9D022C98
:100F50001A9F0ED0042C18D0012C25D100235AF84A
:100F600023000993C047099BF85401339B45F6D1F0
:100F700019E000235AF823000993C047099B27F87A
:100F8000130001339B45F5D10DE05A4600235AF872
:100F900003000B920993C0470B9A099B013AF85042
:100FA00003F10403F3D1B244012300221A99009300
:100FB00001930392049105920F98CDF80890294669
:100FC0005A46FCF707F910980D996F1C01FA80F347
:100FD000BB42B1D03D46BAE7102940F0D8800FFAA5
:100FE00087FA0AFB04F0FEF7D7FD1290002800F004
:100FF000CE80FEF77DFB1A903046FEF779FB189005
:101000002B6900F1180613B1D9F814302BB9E2009E
:101010003FB211927F000D9D88E0B0F9080080007A
:10102000FEF7BAFD119018B1FEF762FB199001E0CE
:10103000119B1993199B002B00F0A0803FB27F00F9
:101040000E97E70013970D9F0C97022CDDF8688030
:1010500004D0042C07D0012C14D104E03046199997
:101060005246234603E01999304652460223D9F8E6
:101070001470B8472F691998414652462346B8471D
:101080000E9F3E440C9F1A9904910123002207F100
:101090000108139F009301930297039205920F9802
:1010A0000C995A46FCF796F8109F0D9800FA87F3B2
:1010B000434502D0CDF83080C7E719A8FEF726FBDC
:1010C0001198FEF74FFB59E08417022024010020FD
:1010D000042C41D0012C11D14A46314631F8020B83
:1010E0000A910B920E9B9847C0470B9A02F8010B8E
:1010F00009EB0A0082420A99F0D13E44012311987B
:101100001A99009300220193029003920491059290
:1011100029465A460F98FCF75DF810990D9A05F18B
:10112000010902FA81F34B4528D04D46022CDDF827
:101130006890CDD14B463146D94631F8020B0A9121
:1011400009930E9A9047C047099B0A9923F8020B0E
:10115000B9F10109F1D1D0E74B463146D94631F812
:10116000020B0A9109930E9A9047C047099B0A996E
:1011700043F8040BB9F10109F1D1BEE718A8FEF755
:10118000C5FA1AA8FEF7C2FA1298FEF7EBFA1DB0DC
:10119000BDE8F08F2DE9F04F91B00E4614460D904A
:1011A000FEF7A6FA024610A813685B4D1B6940F8CB
:1011B000082D5B68B2F808B0B2F80A900993FEF700
:1011C000A5FA2B68554F5B7C57F82300C3680821AC
:1011D0009B6A98472B685B7C57F82330D3F81080C4
:1011E000172888BF20200890D8F80410D8F80020CD
:1011F0000A9100200B92FCF787FC002840F08980C0
:101200002A680FFA8BF7F519B2F90C30013DED1A87
:10121000B2F90830002DCCBFC5EB07053D46B342FF
:10122000C3BFC6EB0301C1EB05051E460021002D1F
:101230006FDD0FFA89F3E018B2F90EC0B2F90A2097
:101240000138CCEB00000028C8BFC0EB0303944278
:10125000BDBFC4EB020ACAEB030314464FF0000AF9
:10126000002B56DD07FB0A1AE3184FEA8A0A0C9393
:101270000D98F9F735FD099B00930FAB00EB0A02BF
:101280000193304621462B46FCF758FB8146002847
:101290003FD0234B0A9999421ED02946089A4346CB
:1012A00001F0A4FAC0B9D8F810C0BCF1000F06D004
:1012B000484649460FFA8BF20423E0470CE04A46C1
:1012C0003B4610680B99069207938847079B069A3E
:1012D000013B42F8040BF4D1089A02920123002248
:1012E00004F1010C0093019303920592CDF8109044
:1012F000304621462A46CDF81CC0FBF76BFF04237D
:101300001BFB03AADDF81CC00C9B9C4501D0644666
:10131000AEE711B0BDE8F08F240100208417022051
:1013200047FE00087FB50C461546064630B3FEF76B
:10133000DFF9134A438901909442028904BFB0F94E
:101340000440B0F90650ADF80840013A013B224490
:101350002B4401A8ADF80C20ADF80A50ADF80E30C2
:10136000FEF7D4F902A8F9F7EFF838B13046214674
:101370002A46FAF77BFAF9F725F8F6E704B070BDCC
:1013800001F0FFFF01490A46FFF7CCBF01F0FFFF64
:10139000034610B533F9144B091BB0F9024000693C
:1013A000121B00FB0233C810802201F0070142FA31
:1013B00001F11A5C1143195410BD70B5B0F9064023
:1013C0000B688688A24241DA36B2B34204693DDA3C
:1013D000143004FB0202DD10701E5419C5EBE0004E
:1013E000555D03F0070205FA02F20134D2B23AB9B0
:1013F00068B3083314F8012B013823F00703F6E72C
:10140000150603D45200D2B20133F9E7FF2A1D4674
:1014100005D0560604D55200D2B20133F9E707339E
:1014200003F00702072A0DD101380BD414F8012B61
:10143000FF2A01D10833F7E7100603D55200D2B2D4
:101440000133F9E7581B0D60013070BD002070BDFD
:10145000FEF788B9B0F906300269002114305A430A
:1014600006F06ABAF8B5B0F90040091BB0F90440BB
:10147000A1422FDAB0F902500B4400F11404013BF1
:101480000069521BDE4300FB024201F00707CC104B
:1014900006F00706FF2141FA07F701FA06F6D4EB3A
:1014A000E30302EB0405FFB2F6B2105D03D13E4048
:1014B00030431055F8BD384310555C1E002C05F123
:1014C000010504DD2846224606F036FA25442B782D
:1014D0001E432E70F8BD00002DE9D34F02F10F0618
:1014E00036117600824606FB03F01430894690469A
:1014F0001F46FEF7CFFB834698B1FEF7F9F8044686
:101500000A4BA36002A8012340F8044DA4F804800C
:10151000A4F800A0A4F80290E780A3812661FEF75A
:10152000F5F8584602B0BDE8D08F00BF9CE6010830
:1015300037B50546FEF7DCF8024602A8948940F864
:10154000042D013CA4B29481FEF7E0F814B92846BA
:10155000FEF708F903B030BD2DE9F843054688468B
:1015600017469946A8684B46466841462846541C8B
:10157000B047089B3B44A34201D02246F2E7BDE8B6
:10158000F883000013B50C4618B9084B1B68186E99
:1015900050B1FEF7ADF8B0F90A3001909C42B8BFE7
:1015A000448101A8FEF7B2F802B010BD240100206A
:1015B00013B518B90D4B1B68186EA8B1FEF798F853
:1015C00002AB446943F8080D6846FEF79FF85CB12A
:1015D0002046FEF78DF802AC836844F8040D9B6842
:1015E00098472046FEF792F802B010BD2401002073
:1015F0000248012918BF0020704700BFF4E6010827
:101600000248162918BF0020704700BF710A010860
:10161000006808B510B1C3681B6A984708BD006828
:1016200008B518B1C3689B6A984708BD4FF0FF30F2
:1016300008BD37B580680C46FEF75AF8034602A885
:101640009988DA881D8940F8043D5B892180628091
:1016500029441A440139013AA180E280FEF756F884
:1016600003B030BD0E4B1B6873B50546186E0E46B1
:10167000FEF73EF8034602A8B3F9064040F8043DE1
:1016800003F11801361BDC68B3F9043004FB0614BF
:10169000ED1AFEF73BF804EB4504204602B070BD9E
:1016A0002401002008B508461146FFF7DBFF00883B
:1016B00008BD0000144B1B68F7B50746186E1546A9
:1016C0000E46FEF715F8294600903046FFF7CAFF90
:1016D0003B6904469B68984723885840009B2080BC
:1016E000586960B1FEF704F802AC836844F8040D51
:1016F0001B6831462A4698472046FEF707F8684699
:10170000FEF704F803B0F0BD2401002073B51C46B9
:10171000104B1B68186E0E461546FDF7E9FF29466B
:1017200000903046FFF79EFF009B0480586960B12F
:10173000FDF7DEFF02AC836844F8040D1B683146F8
:101740002A4698472046FDF7E1FF6846FDF7DEFF91
:1017500002B070BD240100202DE9F3472C4D1E4638
:101760002B688146186E0F461446FDF7C1FF0090A6
:101770004069AA4608B1FDF7BBFF019021463846F3
:10178000FFF770FF009BD3F80C80DAF800301A7C6A
:10179000D20705461FD5D9F810309B6898471FFA25
:1017A00080F8019820B1836839461B682246984723
:1017B0002B8888EA03032B80009B0134DB68B4424A
:1017C0001D44EEDD6846FDF7A1FF019BEBB101A8CA
:1017D000FDF79CFF19E0DB6BD3F80090019B63B130
:1017E0000198836822461B68394601349847B44201
:1017F000A5F800904544F3DDE4E7341B0134013CD7
:10180000A5F800904544FAD1DCE702B0BDE8F087C6
:10181000240100202DE9F04F2A4F14463A689846DB
:10182000D36B87B01B6802938246106E0E46FDF79D
:101830005FFF214604903046FFF714FF049A0546E7
:101840005069D3680393C6EB080909F10108BB4648
:1018500080B1FDF74DFF109A06AF131B47F8040D3A
:1018600001330093314622464346FFF775FE384662
:10187000FDF74CFF4FEA4906109B9C421CDCDBF84D
:1018800000301B7CDB070DD5DAF810309B689847D9
:10189000AA1980B2AB1E5988414023F8021F934217
:1018A000F9D105E0029B284699B24246FBF760FE5B
:1018B000039A01341544DFE704A8FDF727FF07B0BA
:1018C000BDE8F08F2401002007B50092FFF7A2FFCA
:1018D00003B05DF804FB00002DE9F04F814C93B09C
:1018E0009B4623680D90186E07920D46DDF87CA08C
:1018F000FDF7FEFE1090406908B1FDF7F9FE11906A
:1019000012A850F8083DDB680993FDF7FFFE209E02
:1019100011982E44049650B123681B7C990706D178
:101920001C9F00973146079A5B46FFF715FE049807
:101930000799FFF797FE1D9E102E044627D14FEA08
:101940004B0600251C9FDDF84480BD421ADABAF12F
:10195000000F11D084B120465146324606F088F877
:10196000B8F1000F08D0D8F80830079A5F680499DA
:1019700040462A445B46B8471E9FBA44099F01353A
:101980003C44DFE7B8F1000F40F01B831CE31D9ED1
:10199000172E38DD00261C9F119DBE4280F29D80CF
:1019A000079F3744BAF1000F27D034B33DB1AB687D
:1019B0000499D3F804C028463A465B46E047A31E84
:1019C000AAF104090393D846049B0D985B44C8EB25
:1019D0000301036959F8040F1B6802919847039BA0
:1019E000029923F8020F039325B1AB6828461B68C0
:1019F0003A469847B8F10108E6D11E9FBA44099FBC
:101A000001363C44C7E71D9E082E00F102046BD14D
:101A1000079E079F119DF31B1C9FBB42A4F1020070
:101A20005BDA304B219F1B681B7C67B313F0030309
:101A300004D0022B4BD1A046049F1DE01AF80320CE
:101A4000219F57F8222020F8132001335B45F5D160
:101A50003DE0219951F8233028F8023C2DB1AB68C4
:101A600028461B68394632469847049B01375B4439
:101A7000BB4208F102082AD00498C0EB0A03DB5DE0
:101A8000002BF2D0E5E713F0030304D0022B1ED1A4
:101A9000A046049F14E051465A4605F0E9FF16E0BF
:101AA00028F8023C2DB1AB6828461B6839463246FF
:101AB0009847049B01375B44BB4208F1020806D0FB
:101AC000049AC2EB0A03DB5D002BF2D0E8E71E9F0D
:101AD000BA44099F01363C449BE7002D40F07182D7
:101AE00072E200BF24010020219EAB4B209F08948E
:101AF000002E08BF1E462196209E76000E96BF003F
:101B0000079E0F970596089B059E079F9C1EF31B3B
:101B10001C9EB34280F253821D9F022F00F0D98099
:101B2000042F00F07881012F40F03F82DFF870929F
:101B3000D9F80030186EFDF7DBFD9AF80030974AAF
:101B40001090D55CD9F8003020981B7C119F03F0D1
:101B50000303022B5E46C0F1080845FA00F522D0C7
:101B6000032B62D0012B60D05246464538BFB046A9
:101B7000C8EB06064346214605F00100219F013BC4
:101B800057F8200021F8020B4FEA5505F4D104EB79
:101B90004804002E00F0998012F8013F7F494FF071
:101BA0000808CD5CE1E72198DDF81090B0F804C09A
:101BB000CDF818A0464538BFB046C8EB06062FB38F
:101BC0001DB904EB4804C14424E0EA070BD5BB6807
:101BD000059A1B68CDF808C0384649469847DDF895
:101BE00008C0A4F800C0B8F1010809F1010904F126
:101BF00002040FD06D08E3E7EB0748BFA4F800C06C
